:0200000480007A
:100000009705000093854506130540006B10B50069
:10001000EF004005130510006B0005001385411D1E
:10002000138601213306A64093050000EF104040DF
:1000300017150000130505B3EF00502EEF005038E0
:08004000EF00D0046F00D02E88
:10004800B70700009387070063880700371500800B
:10005800130505B66F00102C6780000013054000DB
:100068006B000500977101009381C1AFF326100260
:100078009396A601732600029315A6001316260070
:1000880037F1FF6F3301B1403301D1403301C10073
:10009800F326100263860600130500006B000500B6
:1000A80067800000D772850007E0051233055540C8
:1000B80093922200B38555008760061233065600D6
:1000C8005781000227E10602B3865600E31E05FCAD
:1000D80067800000130101FD232681021304010338
:1000E800232EA4FC232CB4FC232AC4FC8327C4FDA0
:1000F80083A707002326F4FE930744FD2322F4FE7A
:10010800832744FE03C707008327C4FE2380E70034
:100118008327C4FE93871700032744FE034717006D
:100128002380E7008327C4FE93872700032744FE24
:10013800034727002380E7008327C4FE93873700FF
:10014800032744FE034737002380E7008327C4FEC4
:10015800938747002326F4FE232404FE6F00400300
:10016800832784FE032784FDB307F70003C707002E
:100178008327C4FE2380E7008327C4FE93871700E4
:100188002326F4FE832784FE938717002324F4FE96
:10019800832744FD032784FEE344F7FC8327C4FE3A
:1001A8002320F4FE832704FE93F73700032704FE79
:1001B800B307F7002320F4FE832704FE2326F4FE6A
:1001C8008327C4FD0327C4FE23A0E7001300000013
:1001D8000324C1021301010367800000130101FC1D
:1001E800232E8102130401042326A4FC2324B4FC37
:1001F8008327C4FC83A707002326F4FE9307C4FDC6
:100208002322F4FE8327C4FE03C70700832744FE86
:100218002380E700832744FE938717000327C4FE43
:10022800034717002380E700832744FE93872700AE
:100238000327C4FE034727002380E700832744FEE3
:10024800938737000327C4FE034737002380E7005E
:100258008327C4FE938747002326F4FE232404FE45
:100268006F004003832784FE032784FCB307F7004D
:100278000327C4FE034707002380E7008327C4FE43
:10028800938717002326F4FE832784FE938717009D
:100298002324F4FE8327C4FD032784FEE344F7FCEC
:1002A8008327C4FE2320F4FE832704FE93F7370038
:1002B800032704FEB307F7002320F4FE832704FE78
:1002C8002326F4FE8327C4FC0327C4FE23A0E700EB
:1002D800130000000324C103130101046780000018
:1002E800130101FF232681001304010113000000FC
:1002F8000324C1001301010167800000130101FEFE
:10030800232E8100130401022326A4FE2324B4FE15
:10031800832784FE3727000023A2E7009307000005
:10032800138507000324C10113010102678000003F
:10033800130101FE232E1100232C81001304010256
:100348002326A4FEB747018013850750EF00C04F4E
:1003580093071000138507008320C101032481013E
:100368001301010267800000130101FD2326110219
:100378002324810213040103232EA4FC232CB4FCA0
:10038800232AC4FCB70700712326F4FEB7070072BE
:100398002324F4FE930730002322F4FE130744FEBF
:1003A8009307C4FE13064000930507001385070052
:1003B800EFF05FD21307C4FD9307C4FE1306400095
:1003C8009305070013850700EFF0DFD0130784FDBE
:1003D8009307C4FE13064000930507001385070022
:1003E800EFF05FCF130744FD9307C4FE13064000E8
:1003F8009305070013850700EFF0DFCD83A7C11B26
:10040800E7800700130704FE930784FE930507009F
:1004180013850700EFF09FDC832704FE1385070090
:100428008320C102032481021301010367800000B5
:10043800130101FD23261102232481021304010361
:10044800232EA4FC232CB4FC232AC4FCB707007178
:100458002324F4FEB70700722326F4FE9307400016
:100468002322F4FE130744FE930784FE130640007C
:100478009305070013850700EFF0DFC51307C4FDD8
:10048800930784FE130640009305070013850700B1
:10049800EFF05FC4130784FD930784FE1306400042
:1004A8009305070013850700EFF0DFC2130744FD2B
:1004B800930784FE13064000930507001385070081
:1004C800EFF05FC183A7C11BE7800700832744FDC6
:1004D800138507008320C10203248102130101034D
:1004E80067800000130101FD2326110223248102E5
:1004F80013040103232EA4FC232CB4FC232AC4FCDC
:10050800B70700712326F4FE930750002324F4FE56
:10051800130784FE9307C4FE1306400093050700E3
:1005280013850700EFF01FBB1307C4FD9307C4FE34
:10053800130640009305070013850700EFF09FB9E5
:100548009307C4FE032644FD832584FD1385070015
:10055800EFF05FB883A7C11BE7800700832744FD3E
:10056800138507008320C1020324810213010103BC
:1005780067800000130101FD232681021304010393
:10058800232EA4FC8327C4FD63D807008327C4FD5A
:10059800B307F040232EF4FC0327C4FDB73700004F
:1005A8009387078063D8E700B737000093870780F1
:1005B800232EF4FC83A7011C2326F4FE03A7011CA9
:1005C8008327C4FD3307F70023A0E11C8327C4FE5B
:1005D800138507000324C10213010103678000008B
:1005E800130101FE232E1100232C810013040102A4
:1005F8002326A4FE13050000EF00001E13000000D0
:100608008320C101032481011301010267800000D6
:10061800130101FD2326110223248102130401037F
:10062800232EA4FC232CB4FC232AC4FCB707007196
:100638002326F4FEB70700722324F4FE9307700004
:100648002322F4FE130744FE9307C4FE130640005A
:100658009305070013850700EFF0DFA71307C4FD14
:100668009307C4FE1306400093050700138507008F
:10067800EFF05FA6130784FD9307C4FE130640003E
:100688009305070013850700EFF0DFA4130744FD67
:100698009307C4FE1306400093050700138507005F
:1006A800EFF05FA383A7C11BE7800700130704FED1
:1006B800930784FE9305070013850700EFF01FB228
:1006C800832704FE138507008320C10203248102C7
:1006D8001301010367800000130101FF23261100A5
:1006E8002324810013040101B74701801385475172
:1006F800EF008015130000008320C100032481004F
:100708001301010167800000130101FF2326110076
:100718002324810013040101EF00800E93070500D4
:10072800138507008320C100032481001301010100
:1007380067800000130101FF232611002324810094
:1007480013040101B747018013858753EF00C00FD9
:10075800130000008320C10003248100130101015C
:1007680067800000130101FF232611002324810064
:1007780013040101B74701801385C755EF00C00C6A
:1007880083A7011E9386170023A0D11E1385070097
:100798008320C10003248100130101016780000048
:1007A800130101FF232611002324810013040101F2
:1007B800B747018013858758EF0000091300000030
:1007C8008320C10003248100130101016780000018
:1007D8006B10B500678000006B00050067800000A3
:1007E8006B40B500678000006B2005006780000043
:1007F8006B300000678000007325100267800000DE
:100808007325000267800000130540006B00050097
:10081800F32610029396F600732600029315A6009D
:100828001316260037F1FF6F3301B1403301D14071
:100838003301C100F3261002638606001305000089
:100848006B00050067800000130141FF23201100A1
:100858002322B1008345050063880500EF00C0012D
:10086800130515006FF01FFF832001008325410049
:100878001301C10067800000B702010023A0B20085
:1008880067800000130101FC232E1102232C810232
:100898001304010413051000EFF01FF49307500030
:1008A800232CF4FC832784FD9397270013850700E6
:1008B800EF00403A93070500232AF4FC832784FDC0
:1008C8009397270013850700EF00C03893070500AA
:1008D8002328F4FC832784FD9397270013850700BA
:1008E800EF004037930705002326F4FC232604FE77
:1008F8006F0080058327C4FE93972700032744FDD4
:10090800B307F7001307100023A0E7008327C4FEEE
:1009180093972700032704FDB307F7001307200068
:1009280023A0E7008327C4FE939727000327C4FC6E
:10093800B307F7001307500023A0E7008327C4FE7E
:10094800938717002326F4FE0327C4FE832784FD1C
:10095800E342F7FA832584FDB74701801385C75A18
:10096800EF00103F232404FE6F004003832784FE1A
:1009780093972700032744FDB307F70083A70700D1
:1009880093850700B74701801385075CEF00503C4B
:10099800832784FE938717002324F4FE032784FE0D
:1009A800832784FDE344F7FC832584FDB747018052
:1009B8001385475CEF00D039232204FE6F00400303
:1009C800832744FE93972700032704FDB307F70006
:1009D80083A7070093850700B74701801385075C45
:1009E800EF001037832744FE938717002322F4FE75
:1009F800032744FE832784FDE344F7FC832684FD14
:100A0800032684FD832584FDB74701801385075D90
:100A1800EF001034232004FE6F004003832704FEF8
:100A2800939727000327C4FCB307F70083A70700A1
:100A380093850700B74701801385075CEF005031A5
:100A4800832704FE938717002320F4FE032704FE60
:100A5800832784FDE344F7FC8326C4FC032604FDB6
:100A6800832544FD032584FDEFF0CFE3232E04FC0A
:100A78006F00C0068327C4FD939727000327C4FC93
:100A8800B307F70003A707008327C4FD9397270040
:100A9800832644FDB387F60083A607008327C4FD99
:100AA80093972700032604FDB307F60083A70700E2
:100AB800B387F600630EF7008325C4FDB7470180AE
:100AC8001385C75EEF00D028930710006F0040031E
:100AD8008327C4FD93871700232EF4FC0327C4FD46
:100AE800832784FDE348F7F8B747018013854761FA
:100AF800EF00102613050000EFF01FCE930700004B
:100B0800138507008320C103032481031301010413
:100B18006780000093050500930600001306000097
:100B2800130500006F309006130101FF93050000C4
:100B3800232481002326110013040500EF30900EB2
:100B480003A5811B8327C50363840700E78007008B
:100B580013050400EFF0DFA8130101FF232481002F
:100B68002322910037640180B7640180938744365B
:100B7800130444363304F44023261100135424404C
:100B880063020402931424009384C4FFB384F40022
:100B980083A704001304F4FF9384C4FFE7800700CD
:100BA800E31804FE8320C10003248100832441004C
:100BB8001301010167800000130101FF2324810054
:100BC80023202101376401803769018093070436A7
:100BD800130909363309F94023261100232291000D
:100BE80013592940630009021304043693040000D2
:100BF800832704009384140013044400E78007004B
:100C0800E31899FE37640180376901809307043639
:100C1800130949363309F940135929406300090279
:100C280013040436930400008327040093841400FB
:100C380013044400E7800700E31899FE8320C100ED
:100C480003248100832441000329010013010101C9
:100C5800678000009305050003A5811C6F00000153
:100C68009305050003A5811C6F40C002130101FD17
:100C780023229102232E31012326110223248102EB
:100C880023202103232C4101232A51012328610118
:100C98002326710123248101232291019384B50025
:100CA800930760019309050063E497069307000121
:100CB80063ECB720EF00100593040001930780014F
:100CC80013062000138981C2B307F90003A4470063
:100CD800138787FF6302E424832744008326C40024
:100CE8000326840093F7C7FFB307F40003A7470060
:100CF8002326D60023A4C60013671700138509000E
:100D080023A2E700EF005000130584006F00801C49
:100D180093F484FF63CA041A63E8B41AEF00807E70
:100D28009307701F63F8974693D79400638E071C48
:100D380013074000636CF73E93D76400138697034C
:100D48001385870393163600138981C2B306D90029
:100D580003A44600938686FF638C8602832744009B
:100D68009305F00093F7C7FF3387974063C0E50208
:100D7800635807340324C400638C86008327440027
:100D880093F7C7FF33879740E3D4E5FE13060500C2
:100D98000324090113088900630C041983254400FE
:100DA8001307F00093F5C5FFB3879540634AF740F2
:100DB800232A09012328090163D4073E9307F01F5A
:100DC80063E6B73093D535009387150093973700BE
:100DD80003254900B307F90083A6070093D52540EA
:100DE800130710003317B7003367A700938587FFF1
:100DF8002326B4002324D4002322E90023A087005B
:100E080023A686009357264093061000B396F60053
:100E1800636AD712B3F7E600639407029396160045
:100E28001376C6FFB3F7E60013064600639A070079
:100E380093961600B3F7E60013064600E38A07FE0A
:100E48001305F00093183600B308190193850800BC
:100E58001303060003A4C500639A85006F00402FA2
:100E6800635207300324C4006384852E832744001B
:100E780093F7C7FF33879740E354E5FE8326C40002
:100E88000326840093E514002322B4002326D60009
:100E980023A4C600B3049400232A990023289900A8
:100EA8009366170023A6040123A4040123A2D400F7
:100EB800B307F4001385090023A0E700EF00C0641E
:100EC800130584006F0000019307C00023A0F900F8
:100ED800130500008320C1020324810283244102F8
:100EE800032901028329C101032A8101832A4101BF
:100EF800032B0101832BC100032C8100832C4100AB
:100F08001301010367800000930600201306000404
:100F18001305F0036FF05FE303A4C7001306260070
:100F2800E39C87DA0324090113088900E31804E71E
:100F3800032749009357264093061000B396F600FE
:100F4800E37AD7EC03248900832A440013FCCAFF00
:100F580063689C00B3079C401307F000634EF712C8
:100F680083AAC11D03A7C11C9307F0FF330A84019C
:100F7800B38A54016308F732B71700009387F70064
:100F8800B38AFA00B7F7FFFFB3FAFA0093850A00AD
:100F980013850900EF00C0609307F0FF130B0500ED
:100FA800630AF52663664527938B411E83A70B00CA
:100FB800B387FA0023A0FB00138707006306AA384B
:100FC80083A6C11C9307F0FF638EF638330A4B41A2
:100FD8003307EA0023A0EB00937C7B0063860C2E8A
:100FE800330B9B41B7170000130B8B00138AF7FFD5
:100FF800B30A5B019387870033F74A01B3879741A8
:10100800B387E74033FA470193050A0013850900BF
:10101800EF0000599307F0FF6300F53A3305654187
:10102800B30A450183A70B002324690193EA1A0038
:10103800B307FA0023A0FB0023225B0163082433D3
:101048001306F000637886338326440013074CFFA9
:10105800137787FF93F61600B3E6E6002322D40041
:1010680093055000B306E40023A2B60023A4B600FB
:10107800636EE634832A4B0013040B0083A6811D9C
:1010880063F4F60023ACF11C83A6411D63F8F6183F
:1010980023AAF11C6F00801813E714002322E40030
:1010A800B30494002324990093E7170013850900DB
:1010B80023A2F400EF004045130584006FF09FE180
:1010C8008326C400032684006FF01FC293D79500BF
:1010D800130740006374F712130740016360F72297
:1010E8009386C7051387B70593963600B306D900CC
:1010F80083A70600938686FF638AF61A03A747002C
:101108001377C7FF63F6E50083A78700E398F6FE29
:1011180083A6C700032749002326D4002324F4000C
:1011280023A4860023A687006FF0DFCD13074001B4
:101138006378F710130740056360F71E93D7C40060
:101148001386F7061385E706931636006FF0DFBFA0
:10115800130313009377330093858500E39C07CE30
:101168006F00C00FB307F40003A747008326C4002D
:10117800032684001367170023A2E7002326D6005E
:101188001385090023A4C600EF0000381305840066
:101198006FF05FD413D63400938784006FF09FB24A
:1011A800B305B40083A745001385090093E717002A
:1011B80023A2F500EF004035130584006FF09FD19E
:1011C80013E714002322E400B3049400232A9900AF
:1011D8002328990013E7170023A6040123A4040178
:1011E80023A2E400B305B4001385090023A0F50089
:1011F800EF008031130584006FF0DFCD93D76500D1
:101208009386970313878703939636006FF01FEE34
:101218006302241303248900832A440093FACAFF33
:10122800B3879A4063E69A001307F000E346F7E6AF
:1012380013850900EF00402D130500006FF09FC9CA
:101248001386C7051385B705931636006FF0DFAF11
:1012580083A788001306F6FF6394171D937736005B
:10126800938888FFE39607FE0327490093C7F6FF94
:10127800B3F7E7002322F90093961600E3E4D7CCEE
:10128800E38206CC33F7F600631A0700939616003C
:1012980033F7F60013034300E30A07FE13060300BF
:1012A8006FF05FBA938A0A016FF05FCE0325490099
:1012B80093552740130710003317B7003367A7006B
:1012C8002322E9006FF05FE5B71700001387F7FFE7
:1012D800330A5B01337AEA00B387474133FAE70000
:1012E80093050A0013850900EF00802B9307F0FF90
:1012F800E316F5D2130A00006FF0DFD2130740059A
:101308006360F70893D7C5009386F7061387E70647
:10131800939636006FF09FDD130740156360F7085A
:1013280093D7F4001386870713857707931636003B
:101338006FF09FA1938B411E03A70B003387EA0030
:1013480023A0EB006FF0DFC793164A01E39A06C6A5
:1013580003248900B30A5C0193EA1A00232254018A
:101368006FF0DFD123A6611D6FF01FC713040B00B8
:101378006FF0DFD0930710002322FB006FF05FEBC4
:10138800130740156362F70693D7F500938687071E
:1013980013877707939636006FF05FD5130740558C
:1013A8006362F70693D724011386D7071385C70707
:1013B800931636006FF05F99938C8CFFB38A9A016D
:1013C800B38A6A41130A00006FF0DFC593058400F1
:1013D80013850900EF30100C0324890083A70B0044
:1013E800832A44006FF09FC9130740556364F702CE
:1013F80093D725019386D7071387C7079396360097
:101408006FF0DFCE9306803F1306F0071305E00761
:101418006FF09F939306803F1307E0076FF01FCD8F
:10142800832749006FF05FE51303F00013070500F9
:10143800637EC3029377F7006390070A63920508F7
:10144800937606FF1376F600B386E6002320B700EE
:101458002322B7002324B7002326B7001307070168
:10146800E366D7FE6314060067800000B306C34036
:101478009396260097020000B38656006780C60040
:101488002307B700A306B7002306B700A305B700D4
:101498002305B700A304B7002304B700A303B700CC
:1014A8002303B700A302B7002302B700A301B700C4
:1014B8002301B700A300B7002300B700678000002E
:1014C80093F5F50F93968500B3E5D500939605013E
:1014D800B3E5D5006FF0DFF693962700970200007A
:1014E800B386560093820000E78006FA93800200D4
:1014F800938707FF3307F7403306F600E378C3F610
:101508006FF0DFF36780000067800000130101FCC3
:101518002324C1022326D102232AF1022328E1022F
:10152800232C0103232E1103138605008325850030
:101538009307810293860700232E11002326F100CA
:10154800EF00C00B8320C101130101046780000074
:1015580003A3811C130101FC2324C1022326D10209
:10156800232AF1022322B1022328E102232C0103BA
:10157800232E1103832583009307410213060500D8
:101588009386070013050300232E11002326F1007C
:10159800EF00C0068320C101130101046780000029
:1015A800130101FF232481002322910093040500E5
:1015B800138505002326110023A60120EFE09FFBD9
:1015C8009307F0FF630CF5008320C100032481001A
:1015D80083244100130101016780000083A7C12013
:1015E800E38407FE8320C1000324810023A0F400C4
:1015F800832441001301010167800000130101E108
:101608002326111E2324811E2326711D2322B100A7
:10161800930B06002328D1002322911E2320211F8B
:10162800232E311D232C411D232A511D2328611DE2
:101638002324811D2322911D2320A11D232EB11BAC
:10164800130405002320A102EF60C064832705006E
:1016580013850700232AF102EF7010732326A102D5
:101668002328010E232A010E232C010E232E010EFE
:101678006306040083278403E3800754032641009C
:101688000317C6009317070193D7070193962701FD
:1016980063C6060283264606B7270000B367F7002D
:1016A80037E7FFFF1307F7FF33F7E6002316F600C7
:1016B800939707012322E60693D7070113F78700BC
:1016C800630E07160327410003270701630807165F
:1016D80093F7A7011307A0006386E7189307C110C3
:1016E800938C0B00938807002322F10E03C70C008C
:1016F800B7470180938747642326F1002326010E0C
:10170800B74701802324010E232E0100232801025C
:10171800232C01022320010423240104232E010287
:1017280023240100138C077C138D0800032A01026F
:101738006308073E930650026314D7006F10807742
:1017480013840C006F00C0006382D71413040900CF
:101758008347140013091400E39807FEB304994162
:101768006380043C8326C10E0327810E23209D013C
:10177800B38696001307170023229D002326D10E57
:101788002324E10E93067000130D8D0063C6E61046
:101798008327810003471400B38797002324F100AF
:1017A800630007381303F0FF93041900034E190070
:1017B800A303010C13040000130900009309A005FA
:1017C800130B9000930BA002930D03009384140055
:1017D800930A0E0093870AFE63EAF9220327C100E1
:1017E80093972700B387E70083A707006780070060
:1017F80013050A00EF60004A832745001385070098
:10180800232EF102EF7050582324A104930A0500F7
:1018180013050A00EF600048832785002320F104A0
:1018280063840A006F10804A03CE04006FF01FFA29
:101838001369090203CE04006FF05FF983254100A4
:1018480003250102EF20501E630405006F20004F9E
:10185800832741001307A00083D7C70093F7A70188
:10186800E39EE7E6832741008397E700E3C807E69E
:1018780083260101832541000325010213860B00FD
:10188800EF20900E2324A1006F008006B304994135
:10189800E38A04F06FF01FED832541001306410E23
:1018A80013050A00EFA01023631A0502130DC110D7
:1018B8006FF01FEE832541001306410E13050A0041
:1018C800EFA05021630E055283274101638807006A
:1018D8000325010293850700EF30C03B83274100B1
:1018E80083D7C70093F70704638407006F20004578
:1018F8008320C11E0324811E032581008324411EE9
:101908000329011E8329C11D032A811D832A411D24
:10191800032B011D832BC11C032C811C832C411C10
:10192800032D011C832DC11B1301011F67800000BB
:10193800B74701809387077E2328F102937709022E
:1019480013830D00638E070E8327010193877700A9
:1019580093F787FF83AB070083AD470013878700A2
:101968002328E1009377190063880700B3E7BB01D8
:10197800638407006F10C03E9379F9BF9307200076
:10198800A303010C1307F0FFE302E30A33E7BB01EB
:1019980013F9F9F7E31C077AE316032C639A072275
:1019A80013FB1900930C011B63040B006F1000302C
:1019B80093090B0063546B00930903000347710CF0
:1019C800232A01002324010223220102232C0100DF
:1019D800630E0732938919006F0040331304000027
:1019E80013870AFD938414009317240083CAF4FF15
:1019F800B3878700939717003304F70013870AFD0E
:101A0800E372EBFE93870AFEE3FAF9DC638A0A10B5
:101A180023065115A303010C93091000130B1000A2
:101A2800930CC1146F00402DB74701809387477FFF
:101A38002328F1029377090213830D00E39607F038
:101A48000327010193770901832B07001307470038
:101A58002328E100638407006F10C02693770904E8
:101A6800639407006F108025939B0B0193DB0B0198
:101A7800930D00006FF01FEF03CE040013694900B7
:101A88006FF0DFD483CA04009387140063947A014B
:101A98006F20806613870AFD93840700930D00006A
:101AA800E36AEBD29384140093972D0083CAF4FF62
:101AB800B387B70193971700B38DE70013870AFD23
:101AC800E372EBFE6FF01FD18326010193770902C1
:101AD80013874600638407006F10802693770901F7
:101AE800638407006F1040659377090463840700D7
:101AF8006F10502213790920631409006F10C06316
:101B0800832701012328E1000327810083A7070019
:101B1800938C04002380E70003C70C00E31C07C074
:101B28008327C10EE38C07DA8325410003250102D0
:101B38001306410EEFA0007A6FF05FDA03CE0400BF
:101B48009307C0066314FE006F10002C1369090187
:101B58006FF0DFC703CE0400930780066314FE000E
:101B68006F10802B136909046FF05FC69377090221
:101B780013830D00E39807048327010113770901F4
:101B880093874700630407006F20405913770904BF
:101B9800631407006F100067032701019309090008
:101BA8002328F100831B070093DDFB4113870D00F9
:101BB800634C07649307F0FFE304F308B3E7BB0142
:101BC80013F9F9F7E39C0706630403006F10505BF1
:101BD80013030000130B0000930C011B6FF05FDD73
:101BE8001369090803CE04006FF05FBE93770902FA
:101BF80013830D0093690901639C077E8327010104
:101C08009387470003270101930D00002328F10063
:101C1800832B0700930710006FF09FD683270101DD
:101C2800A303010C83AC0700938B470063940C005B
:101C38006F10801F1307F0FF6394ED006F10805141
:101C480013860D009305000013850C002328B101AD
:101C5800EF608034232AA1000323010163140500E7
:101C68006F10D07F83274101338B97410347710C55
:101C78009349FBFF93D9F94123287101232A0100D5
:101C88002324010223220102232C0100B3793B0102
:101C980013030000E31007D46F004007937709028D
:101CA80013830D00136909016396077683270101E1
:101CB8009387470003270101930D00002328F100B3
:101CC800832B07006F00C0761369890003CE0400D8
:101CD8006FF0DFAF03270101A303010C9309100084
:101CE80083270700130747002328E1002306F11480
:101CF800130B1000930CC114232A010013030000D6
:101D08002324010223220102232C010093722900BB
:101D18006384020093892900937B49080327C10E35
:101D280063960B0033083441E34600438346710C45
:101D3800638A06028326810E1306710C2320CD00C8
:101D48001307170013061000938616002322CD00F0
:101D58002326E10E2324D10E13067000130D8D00E7
:101D68006342D60C638A02028326810E1306810C15
:101D78002320CD00130727001306200093861600A2
:101D88002322CD002326E10E2324D10E1306700052
:101D9800130D8D00E348D64E93060008E386DB0654
:101DA800B30D6341E344B01793760910639A067044
:101DB8008327810E3307670123209D01938717002E
:101DC80023226D012326E10E2324F10E93067000D1
:101DD800130D8D00E3CEF62413794900630609003C
:101DE80033093441634820076354340113840900DC
:101DF80083278100B38787002324F100E31C07AA07
:101E0800832741012324010E6388070083254101AC
:101E180013050A00EF201068130DC110938C0400FD
:101E28006FF09FCF832541001306410E13050A006A
:101E38002326610423225104EFA0C049E31605A814
:101E48000327C10E130DC1100323C10483224104CB
:101E58006FF05FF1930600018327810E63C42601AA
:101E68006F10106DB7460180938D067B130B000130
:101E7800930B7000832A41006F00C000130909FF0B
:101E880063562B0513070701938717002320BD010D
:101E980023226D012326E10E2324F10E130D8D005C
:101EA800E3DEFBFC1306410E93850A0013050A00C6
:101EB800EFA04042E31A05A0130909FF0327C10E4A
:101EC8008327810E130DC110E34E2BFB3307270127
:101ED800938717002320BD0123222D012326E10E1D
:101EE8002324F10E93067000E3D0F6F08325410019
:101EF8001306410E13050A00EFA0C03DE316059C2A
:101F08000327C10E6FF05FEE1377890013830D006E
:101F1800E300075E8327010103A7070093874700B3
:101F28002328F1008325070003264700832687001E
:101F38000327C7002328B10E232AC10E232CD10E54
:101F4800232EE10E1305010F232A6100EF50D04D17
:101F58002326A10C13072000032341016314E50085
:101F68006F108015130710006314E5006F10402FE1
:101F7800130710066394EA006F101071130710041A
:101F88006394EA006F10C06293F7FAFD1307F0FF3D
:101F98002326F1046314E3006F10D0711307700453
:101FA8006394E7006F101070832EC10F232C210556
:101FB800136709108322010F032F410F832F810F0D
:101FC80063D40E006F10D027232E010413090700D5
:101FD800232A01000327C104930760046314F70050
:101FE8006F105030930750046314F7006F1090601F
:101FF8009309010B9307010D1307C10C9306030006
:102008001308C10D130620009385090013050A0063
:10201800232261042328510A23245102232AE10B95
:102028002322E103232CF10B232EF101232ED10BC4
:10203800232CD101EF40100E8327C104130770042D
:10204800930C0500832E8101832FC101032F4102C8
:1020580083228102032341046384E7006F20C00DBB
:102068008327810513F71700630407006F10D062F8
:102078000327C10DB3079741232EF1008327C10C15
:1020880013077004232CF1008327C1046394E7002D
:102098006F1090128327C104130760046394E7004C
:1020A8006F10903E832781019305100493F6FA0F71
:1020B8001387F7FF8327C1042326E10C13060000CA
:1020C8006398B7009386F60093F6F60F1306100090
:1020D800230AD10C635407006F10907B9306B0025B
:1020E800A30AD10C9306900063C4E6006F10D06673
:1020F8001308310E130608001305A0001303300659
:102108006F00C0001386050013870600B367A70297
:102118009305F6FF93870703A30FF6FEB346A702BE
:10212800E342E3FE138706031377F70F9306E6FFF0
:10213800A38FE5FE63E406016F10507F9305610DE0
:102148006F00800003C7060093851500938616006C
:10215800A38FE5FEE39806FF1307510E9307610D61
:102168003307C7403387E7009306410DB307D740CD
:10217800232CF1028327C101832681031307100052
:10218800338BD7006344F7006F1010728327C102A6
:10219800330BFB00832781059349FBFF93D9F94152
:1021A80013F9F7BF13690910B3793B01232401021E
:1021B80023220102232C01008327C1056394070011
:1021C8006F10D0061307D002A303E10C130300001D
:1021D800938919006FF09FB39377090213830D0059
:1021E800936909016392071E8327010193874700BA
:1021F800032701012328F100832B070093DDFB410E
:1022080013870D00E358079AB30B7041B337700179
:10221800B30DB041B38DFD409307D002A303F10C79
:102228001307F0FF930710006312E3F6130710007B
:102238006388E720130720006382E7249306011BC5
:102248006F00800093860C009397DD0113F77B00E5
:1022580093DB3B0013070703B3EB770193DD3D00E6
:10226800A38FE6FEB3E7BB01938CF6FFE39C07FC64
:1022780013F61900630E062213060003630AC72229
:102288009386E6FF9307011BA38FCCFE338BD740C1
:1022980013890900938C06006FF08FF10327010161
:1022A800B787FFFF93C707832314F10C93074700F1
:1022B8002328F100B74701809387077E13830D0019
:1022C8002328F102832B0700930D0000936929004E
:1022D80093072000930A80076FF08FEA8347710CF9
:1022E80003CE0400639407CE93070002A303F10C06
:1022F8006FF0CFCD9307B002A303F10C03CE040017
:102308006FF0CFCC8327010103CE040003A407009C
:10231800938747002328F100635A04CA3304804096
:10232800136949006FF08FCA1369190003CE0400BE
:102338006FF0CFC99377090213830D00639C070CD4
:1023480083260101137709019387460083AB0600B2
:10235800E312079613770904E308076C939B0B01B4
:1023680093DB0B01930D00002328F1006F00400C54
:102378009377090213830D00639A070683260101E8
:10238800137709019387460083AB060063040700AF
:102398006F10505913770904E304076A939B0B01E4
:1023A8002328F10093DB0B01930D0000930909002A
:1023B800930710006FF0CFDC03250102EF20807730
:1023C8006FF0CFAB9309090083270101938777004A
:1023D80093F787FF03A74700938687002328D10038
:1023E80083AB0700930D07006FF08FFC930909007A
:1023F800832701019387770093F787FF1387870067
:1024080083AB070083AD47002328E1009307100042
:102418006FF00FD7832701019387770093F787FF22
:1024280083AB070083AD4700138787002328E100AB
:102438009379F9BF930700006FF08FD493090900CF
:10244800E39C0D3693079000E3E87737938B0B03F3
:10245800A307711B13890900130B1000930CF11AC1
:102468006FF00FD5130710006394E7006F10405109
:102478001307200093090900E392E7DC8326010390
:10248800930C011B93F7FB00B387F60083C7070083
:102498001397CD0193DB4B00938CFCFFB36B770153
:1024A80093DD4D002380FC00B3E7BB01E39C07FCF0
:1024B8009307011B338B9741138909006FF04FCFA6
:1024C8009306500663D656398326010F9305010AF1
:1024D8001305010B2328D10A8326410F2322E10487
:1024E8002320010A232AD10A8326810F2322010AE5
:1024F8002324010A232CD10A8326C10F2326010A8B
:10250800232ED10AEFE0106D032741046312055A08
:102518008327810EB756018093860681130717001B
:102528002320DD0093871700930610002322DD0087
:102538002326E10E2324F10E13077000130D8D00DE
:10254800E344F7348327C10C0327C10163CAE700BA
:1025580093771900639607000327C10E6FF0DF8792
:10256800832741038326C1020327C10E2320FD00D0
:102578008327810E3387E6002322DD009387170027
:102588002326E10E2324F10E93067000130D8D000F
:10259800E3CAF6048327C101138BF7FFE35E608368
:1025A800930600018327810EE3D06631930B000167
:1025B800930A7000832C41006F00C000130B0BFFBF
:1025C800E3D46B2F130707019387170023208D018E
:1025D80023227D012326E10E2324F10E130D8D0005
:1025E800E3DEFAFC1306410E93850C0013050A007E
:1025F800EF90504E631A05AC0327C10E8327810E56
:10260800130DC1106FF09FFBB30B3441635A70F97F
:10261800130600018326810E6354760B232291044E
:1026280093070D0093840B00138D0C00938B090006
:10263800930C0B0093090400930E0001930D700096
:1026480003244100130B03006F00C000938404FFB0
:1026580063D89E04130707019386160023A08701F9
:1026680023A2D7012326E10E2324D10E93878700C6
:10267800E3DEDDFC1306410E9305040013050A0092
:10268800EF905045631205A4930E0001938404FF54
:102698000327C10E8326810E9307C110E3CC9EFA4F
:1026A8001384090093890B00938B0400832441044D
:1026B80013030B00138B0C00930C0D00138D0700F4
:1026C800330777019386160023208D0123227D018D
:1026D8002326E10E2324D10E13067000130D8D005E
:1026E8006350D6EC832541001306410E13050A00FA
:1026F80023226104EF90103E6318059C0327C10E46
:10270800130DC110032341046FF08FE91306000174
:102718008326810E6358B60993070D00130800013C
:10272800138D0C00930B7000930C0B00138B090096
:1027380093090400032441006F00C000938D0DFF2E
:102748006358B805130707019386160023A087016D
:1027580023A207012326E10E2324D10E93878700A5
:10276800E3DEDBFC1306410E9305040013050A00A3
:10277800EF905036631A059413080001938D0DFFEE
:102788000327C10E8326810E9307C110E34CB8FBC3
:102798001384090093090B00138B0C00930C0D0094
:1027A800138D07003307B7019386160023208D0188
:1027B8002322BD012326E10E2324D10E1306700027
:1027C800130D8D006352D6DE832541001306410E9A
:1027D80013050A00EF9010306318058E0327C10E09
:1027E800130DC1106FF04FDC937519006392050843
:1027F8002322DD002326B10F2324610F93077000E5
:1028080063CA675B930A2600130D0D0183268103B3
:102818009307410D23A0FB003387B60123A2DB00F9
:102828002326E10E2324510F9307700063D657DB4C
:10283800832541001306410E13050A00EF909029E5
:10284800631405880327C10E130DC1106FF0CFD88C
:102858000326810E8327C1019306100023209D01C2
:10286800930D1700130B1600930B8D00E3DEF6F69D
:10287800930610002322DD002326B10F2324610FC5
:102888009306700063CC66638327C1020327410364
:10289800130B1B00B38DFD0023A0EB0023A2FB004C
:1028A8002326B10F2324610F93067000938B8B00AE
:1028B80063CA66638326010F8327C10113081B00BF
:1028C8002328D10A8326410F9305010A1305010B1A
:1028D800232AD10A8326810F930A080023220103A1
:1028E800232CD10A8326C10F2320010A2322010A9F
:1028F800232ED10A9386F7FF232CD1002324010A23
:102908002326010AEFE0102D138D8B008326810109
:1029180003284102630E053093871C00B38DDD0048
:1029280023A0FB0023A2DB002326B10F2324510F91
:102938009307700063C0574993870B01930A2B00D4
:10294800930B0D00138D07006FF05FEC93090900DE
:102958006FF0DF8DB7470180130600018326810ED3
:10296800938D077B6354060D2326910423282105A4
:1029780093070D0013890D00130D0B00938D0C00A8
:10298800130F0001938C090093037000930904004E
:1029980023225104130B030083244100130408006D
:1029A8006F00C000130404FF635C8F041307070162
:1029B8009386160023A0270123A2E7012326E10E10
:1029C8002324D10E93878700E3DED3FC1306410E40
:1029D8009385040013050A00EF90D00F63040500E7
:1029E8006FE09FEE130F0001130404FF0327C10ECD
:1029F8008326810E9307C11093037000E3488FFA72
:102A08001308040083224104138409008324C104A9
:102A180093890C00938C0D00930D0900032901057F
:102A280013030B00130B0D00138D07003307070169
:102A3800938616002320BD0123220D012326E10ED3
:102A48002324D10E13067000130D8D006350D6AEEB
:102A5800832541001306410E13050A00232661044D
:102A680023225104EF901007630405006FE0DFE5AF
:102A78000327C10E130DC1100323C104832241048F
:102A88006FF0CFAA832541001306410E13050A00F3
:102A980023226104EF901004630405006FE0DFE275
:102AA8000327C10E130DC110032341046FF0CFAEED
:102AB8000326C10C635CC044832781018326C101BE
:102AC800138B070063CCF62A635660038326810EB6
:102AD8003307670123209D019386160023226D0189
:102AE8002326E10E2324D10E13067000130D8D004A
:102AF800E34ED61C9346FBFF8327810193D6F6410C
:102B0800337BDB00338B674163406035832781016A
:102B180093760940B38AFC00639C067A032BC10CA8
:102B28008327C1016346FB0093761900E386061CE0
:102B3800832641038327C102130670002320DD008A
:102B48008326810E3307F7002322FD0093861600A3
:102B58002326E10E2324D10E130D8D006354D600D5
:102B68006F10400D8326C101B387DC00338B6641AB
:102B7800B3875741930B0B0063D46701938B07000E
:102B8800635870038327810E3307770123205D0183
:102B98009387170023227D012326E10E2324F10EBB
:102BA80093067000130D8D0063D4F6006F10801427
:102BB80093C7FBFF93D7F741B3FBFB00330B7B4174
:102BC800635C60A1930600018327810E63DE664D76
:102BD800930B0001930A7000832C41006F00C00022
:102BE800130B0BFF63D26B4D130707019387170075
:102BF80023208D0123227D012326E10E2324F10EBB
:102C0800130D8D00E3DEFAFC1306410E93850C00CC
:102C180013050A00EF90006C630405006FE0DFCA3B
:102C28000327C10E8327810E130DC1106FF05FFBC0
:102C3800E35ED0BC9307000163C4D7006F10404B1C
:102C4800232C8100930C0001930A70001384060062
:102C5800032D4100130B08006F000001130404FF4B
:102C680063D48C12130B1B00938D0D0123A08B01D1
:102C780023A29B012326B10F2324610F938B8B0082
:102C8800E3DE6AFD1306410E93050D0013050A00E5
:102C9800EF904064630405006FE01FC3832DC10EED
:102CA800032B810E930BC1106FF05FFB930700039A
:102CB800A307F11A930CF11A6FE09FCF93770920BD
:102CC800E3980706930D00006FE0DFC9832701042E
:102CD80003CE0400639407006FE05FAF83C707006B
:102CE800639407006FE09FAE136909406FE01FAE61
:102CF800832701011305010B232AB101938777006C
:102D080093F787FF83A5070003A6470093878700EB
:102D18002328F100EF1041210327010B0323410170
:102D28002328E10E0327410B232AE10E0327810BF9
:102D3800232CE10E0327C10B232EE10E6FF08FA089
:102D48000326810083A706002328E1009356F64155
:102D580023A0C70023A2D700938C04006FE0DFDB19
:102D680093070003136929002304F10CA304510DF0
:102D78009379F9BF930720006FE09FC0138B06007B
:102D8800E34660D56FF01FD7930604000324810142
:102D9800930A1B0093878B00B38DDD0023A2DB0011
:102DA80023A08B012326B10F2324510F9306700013
:102DB80063DC566D832541001306410E13050A0096
:102DC800EF904051630405006FE01FB00326810EA9
:102DD800832DC10E130D4111930A1600930BC110D8
:102DE8006FF0DFA2832541001306410E13050A0088
:102DF800EF90404E630405006FE01FAD0327C10E3E
:102E0800130DC1106FF00FF903CE140013690902F6
:102E1800938414006FE09F9B03CE1400136909206C
:102E2800938414006FE09F9A93076000138B0D0042
:102E380063E0B76DB757018093090B002328710130
:102E4800938C87806FE05FEB130600018326810E69
:102E5800635C6643930D0001930A7000832B410065
:102E68006F00C000130B0BFF63D06D4313070701FE
:102E78009386160023208D012322BD012326E10E0F
:102E88002324D10E130D8D00E3DEDAFC1306410E68
:102E980093850B0013050A00EF90C04363040500F7
:102EA8006FE09FA20327C10E8326810E130DC11068
:102EB8006FF05FFB13890C006FE0DF8E8325410004
:102EC8001306410E13050A00EF90C0406304050085
:102ED8006FE09F9F832DC10E032B810E930BC110B2
:102EE8006FF09F9A832541001306410E13050A00CF
:102EF800EF90403E630405006FE01F9D832DC10ED7
:102F0800032B810E930BC1106FF0DF9A8326810E7D
:102F1800B7550180938505812320BD00130717004D
:102F280093051000938616002322BD002326E10E88
:102F38002324D10E93057000130D8D0063CED55454
:102F4800631206228327C10193761900B3E6F600BF
:102F5800639406006FE05FE8832641038327C1027C
:102F6800130670002320DD008326810E3307F70047
:102F78002322FD00938616002326E10E2324D10E7A
:102F880093088D00634ED65E8327C1019386160091
:102F980023A098013387E70023A2F8002326E10E37
:102FA8002324D10E93077000138D880063C4D700C3
:102FB8006FE09FE26FF0DF87930C011B930700001F
:102FC80013F90940232A9100232C3101130BF00F28
:102FD80093890C0023226102930C0A0083240104C4
:102FE800138A0D00930D0D00130D040013840700C0
:102FF8006F0040021306A0009306000013850B0023
:1030080093050A00EFC0D070E3000A2C930B05006B
:10301800138A05001306A0009306000013850B0011
:1030280093050A00EFD0003213050503A38FA9FE0C
:10303800130414009389F9FFE30E09FA83C6040008
:10304800E31AD4FAE30864FBE3100A249307900018
:10305800E3EC7723138A0C00938C09008329810100
:103068009307011B232E81002320910413040D00D4
:103078000323410283244101138D0D00338B9741B3
:10308800138909006FE0DF92832541001306410E82
:1030980013050A00EF900024630405006FE0DF8247
:1030A800130DC1106FF00FCA33076701938717001C
:1030B80023208D016FE0DFD08327010F9305010ADC
:1030C8001305010B2328F10A8327410F2320010A46
:1030D8002322010A232AF10A8327810F2324010AC4
:1030E8002326010A232CF10A8327C10F232EF10A74
:1030F800EFE0404FE340051E0347710C930770044F
:1031080063D0573DB7470180938C477D232A010040
:103118002324010223220102232C01001379F9F749
:1031280093093000130B30001303000063040700F9
:103138006FE05F8A6FE09FBD83270101938C0400D5
:1031480083A707002328E1000327810023A0E700C5
:103158006FE09F9C13850C00EF600043130B050084
:103168006FE0DFB0832641038327C1029305700017
:103178002320DD008326810E3307F7002322FD007C
:10318800938616002326E10E2324D10E93088D0082
:1031980063C8D53EE35A06DE930500FF330BC040F3
:1031A800E354B63A930B0001930A7000032D4100D3
:1031B8006F00C000130B0BFFE3D86B39130707012F
:1031C8009386160023A0880123A278012326E10E06
:1031D8002324D10E93888800E3DEDAFC1306410E1F
:1031E80093050D0013050A00EF90C00E6304050057
:1031F8006FE08FED0327C10E8326810E9308C1105F
:103208006FF05FFB13770920630A07340327010176
:10321800930909002328F100830B070093DDFB4184
:1032280013870D006FE0DF981377092063020732D8
:1032380093FBFB0F930D00002328F1006FF04F9FC5
:1032480013770920630C072E2328F10093FBFB0F4B
:10325800930D000093090900930710006FE04FF2E7
:103268008327C10F63DA07309307D002A303F10C59
:103278001307D00293077004E3D6572BB747018092
:10328800938CC77D6FF09FE833076701938616001C
:1032980023208D0123226D012326E10E2324D10E44
:1032A80013067000130D8D00E352D6868325410066
:1032B8001306410E13050A00EF90C00163040500D0
:1032C8006FE08FE00327C10E130DC1106FF01F844C
:1032D8008327C101832B4102232C9100B387FC0073
:1032E80023222105232681048324810223223103FA
:1032F8002324910393060D00130B7000930D000116
:10330800032981040324010483294100138D070044
:10331800638A0B08639A04081304F4FF938BFBFF7A
:103328008327C1033307270123A2260123A0F60020
:103338008327810E2326E10E938686009387170044
:103348002324F10E634CFB0E03460400B3055D41D4
:10335800930C060063D4C500938C05006356900354
:103368000326810E3307970123A056011306160082
:1033780023A296012326E10E2324C10E6342CB0E1D
:10338800034604009386860093C5FCFF93D5F54158
:10339800B3F7BC00B30CF640634C9001B38ACA0083
:1033A800E39A0BF66382045E9384F4FF6FF05FF791
:1033B8000326810E63C89D016F008005938C0CFF66
:1033C80063D89D05130707011306160023A086017D
:1033D80023A2B6012326E10E2324C10E938686007C
:1033E800E35ECBFC1306410E9385090013050A0022
:1033F800EF80506E630405006FE00FCD938C0CFFD7
:103408000327C10E0326810E9306C110E3CC9DFB52
:10341800330797011306160023A0860123A29601FD
:103428002326E10E2324C10E634ACB62034604001F
:1034380093868600B38ACA006FF09FF61306410E82
:103448009385090013050A00EF80D068630405001E
:103458006FE08FC70327C10E9306C1106FF0DFEE30
:103468001306410E9385090013050A00EF80906644
:10347800630405006FE04FC5034604000327C10E2F
:103488009306C1106FF05FF0938A1A00138D8700BE
:10349800938B07006FF08FB7832541001306410E09
:1034A80013050A00EF801063630405006FE0CFC1C5
:1034B8000326C10C0327C10E130DC1106FF05FA8BE
:1034C800B7470180938C077D6FF05FC48325410067
:1034D8001306410E13050A00EF80D05F6304050050
:1034E8006FE08FBE0327C10E130DC1106FF08FE080
:1034F800130B60006FF01F948326C101B387DC00B3
:10350800338B6641B38B574163547BEB930B0B00B2
:103518006FF00FEA832701012328E10003278100C8
:1035280083A70700938C04002390E7006FE0CFDEA9
:1035380093FBFB0F930D00006FE0CFC22328F1002F
:10354800930D000093090900930710006FE04FC323
:10355800930D00002328F1006FE09FED0327010180
:10356800930909002328F100832B070093DDFB4111
:1035780013870D006FE0CFE30347710C6FF09FCF07
:10358800832541001306410E13050A00EF8090546D
:10359800630405006FE04FB30326C10C0327C10E77
:1035A8008326810E9308C110E350069E6FF0DFBE9C
:1035B800930700032304F10C93078005A304F10C7F
:1035C8009367290013073006232CF104232A0100EE
:1035D800930CC114E3486708832EC10F93F7FAFDD3
:1035E8002326F104232E0104136929108322010FD5
:1035F800032F410F832F810F63C80E441307100652
:10360800E384EA18130710046384EA006FE09F9CC0
:103618009309010B13850900232A61042328510A01
:10362800232AE10B232CF10B232ED10BEF00913031
:103638001306C10CEF50D02313860500930505002F
:1036480013850900EF00510E0327010B93070109A9
:10365800930B010A2328E1080327410B13060108ED
:1036680093850700232AE1080327810B13850B00A4
:10367800232EF100232CE1080327C10B2328C104C2
:1036880023200108232EE1083707FC3F2326E10801
:103698002322010823240108EFE000098327010AF7
:1036A8000328410A832E810A032FC10A93850B0040
:1036B800138509002328F10A2322F104232A010B88
:1036C80023240103232CD10B2322D103232EE10B26
:1036D800232CE1012320010A2322010A2324010AC1
:1036E8002326010AEFD0104F032F8101832E4102B8
:1036F800032881028327410403234105631605003B
:10370800130710002326E10C374701801307477F72
:103718002322E104130BF3FF232C910123209106AC
:1037280023225107232AA107232C4107232E91077F
:10373800232421072326810623286106930C0B00E6
:10374800138D0700930D0800138A0E00930A0F00CB
:103758008324C1016F00400593850B001385090080
:103768002324C1022322F103232E5100232A510AC4
:10377800232CF10B232EC10A2328210B2320010A15
:103788002322010A2324010A2326010AEFD09044A8
:10379800938CFCFF8322C101832F410203268102FF
:1037A8006304050E232C6101B70703401386040048
:1037B80093850B0013850900232EF1082320A10B04
:1037C8002322B10B2324410B2326510B2328010864
:1037D800232A0108232C0108EFD01075138509004E
:1037E800EF00014793050500130405001385090040
:1037F800032BC10B832A010B032A410B0329810BDD
:10380800EF00015A8327010B032601059385040065
:103818002320F1088327410B13850B00232E610910
:103828002322F1088327810B23285109232A4109E0
:103838002324F1088327C10B232C21092326F1080F
:10384800EFE0106F83274104032781010329010A50
:10385800B387870083C707008322410A832F810A21
:103868000326C10A130B1700A30FFBFE232A910599
:103878009307F0FF130D0900938D0200138A0F00C0
:10388800930A0600E39AFCEC03230107930309005B
:10389800B706FE3F93850B001385090023226102BA
:1038A800232E810083240106832A41062328710AD6
:1038B80023227106232A510A23205106232CF10BB7
:1038C8002328F105232EC10A2324C1022320010A3B
:1038D8002322010A2324010A2326D10AEFD0503CCF
:1038E800032D41070324C106930D0B00032A81070A
:1038F800832CC1070329810603234102634CA04896
:103908008323410683220106832F010503268102B2
:10391800B706FE3F93850B00138509002328710A1B
:10392800232A510A232CF10B232EC10A2320010A32
:103938002322010A2324010A2326D10AEFD0902941
:1039480003234102631805008327C10113FB1700F5
:1039580063120B448327410513060003938617005F
:10396800B386DD0063C80700938D1D00A38FCDFECD
:10397800E39CB6FFB3879D41232EF1006FE00FF063
:10398800930909006FE09FAC832C81028327C10152
:1039980023208104138D0600B386FC008324810153
:1039A800032941040324C1048329410263F856977B
:1039B800938A06006FF08F96832781011307D0FF43
:1039C80063C4E700635AF300938AEAFF93F7FAFDAA
:1039D8002326F1046FE00FED0327C101832781013E
:1039E80063C2E72E03278105138B0700137717009F
:1039F800630607000327C102338BE700832781058D
:103A080013F7074063060700832781016348F04ADC
:103A18009349FBFF93D9F941B3793B01930A7006A7
:103A280023240102232201026FE00FF90347710CDE
:103A380013030000630407006FD0DFF96FE00FADD8
:103A4800232A010013090700370700809307D002D3
:103A5800B34ED701232EF1046FF05FBA1306410E5F
:103A68009385090013050A00EF80D006630405005A
:103A78006FD09FE5034604000327C10E9306C110CB
:103A8800B38ACA006FF0DF91832781048325C103BD
:103A980013040000B389F940138607001385090051
:103AA800EF50503703C814001306A0009306000017
:103AB8003338000113850B0093050A00B384040111
:103AC800EFC000456FF08FD49307900063E077D57F
:103AD8006FF04FD89307D002A303F10C1307D0025D
:103AE8006FF0CFE19309010B930603001307C10C94
:103AF8001308C10D9307010D1306300093850900C3
:103B080013050A00232261042328510A23245102A1
:103B1800232AE10B2322E103232CF10B232EF101AD
:103B2800232ED10B232CD101EF20D05E8346050034
:103B380013070003930C0500832E8101832FC10115
:103B4800032F41028322810203234104930B010ABC
:103B5800638CE6060327C10C330B6700338B6C01BB
:103B680093850B0013850900232C61002328510A33
:103B7800232AE10B232CF10B232ED10B2320010A3E
:103B88002322010A2324010A2326010AEFD09004E4
:103B980013070B0003238101631405006FE08FCD29
:103BA8000327C10D13060003636467016FE08FCC20
:103BB80093071700232EF10C2300C7000327C10D1C
:103BC800E36867FF6FE00FCB930B010A93850B0047
:103BD80013850900232261042328510A2324510252
:103BE800232AE10B2322E103232CF10B232EF101DD
:103BF800232ED10B232CD1012320010A2322010AD1
:103C08002324010A2326010AEFD0C07C832E8101D8
:103C1800832FC101032F4102832281020323410420
:103C2800E30A05F213071000330767402326E10C67
:103C38006FF09FF2832541001306410E13050A0019
:103C4800EF804069630405006FD01FC8032BC10CC7
:103C58000327C10E130DC1106FE0DFF00347710C8D
:103C6800232871012324010223220102232C0100AD
:103C780093090300130B03001303000063040700F8
:103C88006FD05FD56FE08F888327810513F7170002
:103C980083278101336767006352F0426314072A60
:103CA800032B8101930A60068327810513F70740D8
:103CB800631807209349FBFF93D9F941B3793B0176
:103CC8006FF01FD68327C1010327C102930A70062C
:103CD800338BE70083278101E348F0FC330BFB407B
:103CE800130B1B009349FBFF93D9F941B3793B01AF
:103CF8006FF01FD3832541001306410E13050A00F8
:103D0800EF80405D630405006FD01FBC032BC10C1E
:103D18008327C1010327C10E130DC110338B6741DF
:103D28006FE01FE9B7470180938C877D6FF00FBE66
:103D3800B7460180938D067B6FE04F999307F0FF9C
:103D48002324F1006FD0DFBA33076701938616008A
:103D580023A0880123A268012326E10E2324D10E83
:103D680013067000938888006350D6A2832541000B
:103D78001306410E13050A00EF80C05563040500C1
:103D88006FD09FB40327C10E8326810E9308C110FC
:103D98006FF08F9F8327810193860D00232EF10CEE
:103DA8008327410403C6FDFF83C5F7006310B602ED
:103DB80013050003A38FA6FE8326C10D9387F6FF84
:103DC800232EF10C03C6F6FFE386C5FE9305160005
:103DD8001305900393F5F50F6306A600A38FB6FEAF
:103DE8006FF05FB98327410483C5A700A38FB6FE90
:103DF8006FF05FB8130B13009309010B1308C10D83
:103E08009307010D1307C10C93060B00130620003E
:103E18009385090013050A00232261042328510A07
:103E280023245102232AE10B2322E103232CF10B43
:103E3800232EF101232ED10B232CD101EF20902D1D
:103E4800832E8101832FC101032F41028322810226
:103E580003234104930C0500338B6C01930B010A77
:103E68006FF01FD09305130013050A00232A610081
:103E7800EFC0DFDF930C0500032341016302052C2B
:103E8800232AA1006FF04FF5930700032304F10CD8
:103E9800930780076FF08FF2338B6C00930B010A46
:103EA8006FF01FCC630403006FE00F901303100042
:103EB8006FE08F8F130360006FE00F8F930A700617
:103EC80083250104832781012324010203C70500F8
:103ED800232201021306F00F630EC702635CF70288
:103EE80083C61500B387E740638E060003274102A7
:103EF80093851500130717002322E1021387060094
:103F08006FF09FFD83268102938616002324D10239
:103F18006FF09FFC232CF1000327810283274102C5
:103F28002320B1043387E700832781043307F7028E
:103F3800330B67019349FBFF93D9F941B3793B01EF
:103F48006FE08FA70327C102930A6006338BE7004F
:103F5800330B6B006FF05FD59306610D6318060095
:103F680093060003230BD10C9306710D9307011BD5
:103F78003386F640130707039307D60D2380E60020
:103F8800232CF1026FE00F9F9309010B13850900A1
:103F9800232A61042328510A232AE10B232CF10B3D
:103FA800232ED10BEF0001191306C10CEF50400C62
:103FB800138605009305050013850900EFF0D076F8
:103FC8000327010B93070109930B010A2328E10832
:103FD8000327410B1306010893850700232AE108EC
:103FE8000327810B13850B00232EF100232CE108F6
:103FF8000327C10B2328C10423200108232EE1082D
:104008003707FC3F2326E10823220108232401085F
:10401800EFD080718327010A0328410A832E810A81
:10402800032FC10A93850B00138509002328F10A81
:104038002322F104232A010B23240103232CD10B6F
:104048002322D103232EE10B232CE1012320010A93
:104058002322010A2324010A2326010AEFD08037EC
:10406800032F8101832E4102032881028327410403
:104078000323410563160500130710002326E10CEE
:10408800374701801307077E2322E1046FF08FE88A
:1040980083278101130710009306D0023307F740E6
:1040A800A30AD10C6FE00F848327810513F717004B
:1040B800631407006FE00F8E6FE04F8D631A0700DF
:1040C80093091000930A6006130B10006FF05F95B8
:1040D8008327C102930A6006138B1700330B6B000A
:1040E8009349FBFF93D9F941B3793B016FF05F9393
:1040F80093070D006FE05FCA03270101832D0700B6
:104108001307470063D40D00930DF0FF03CE14008E
:104118002328E100938407006FD04FEB930909002F
:104128006FE00F8D930909006FD0DFAD9307200072
:10413800232CF1026FE00F84130B03006FF0DFD123
:10414800032741008357C70093E707042316F700A6
:104158006FD0CFF893060600138605009305050077
:1041680003A5811C6FD08FC983D7C50003AE450650
:1041780003D3E50083A8C50103A84502130101B8CC
:1041880093F7D7FF13070040232C8146231AF10029
:10419800138405009307010793058100232A91469C
:1041A80023282147232E1146130905002326C1077A
:1041B800231B610023221103232601032324F1007A
:1041C800232CF1002328E100232EE1002320010203
:1041D800EFD0CFC293040500635C05028357410109
:1041E80093F70704638807008357C40093E707041D
:1041F8002316F4008320C147032481471385040054
:1042080003290147832441471301014867800000BF
:104218009305810013050900EF000058E30005FC31
:104228009304F0FF6FF09FFB83A7811C130101FF2C
:1042380023248100232291002326110093040500E2
:10424800138405006386070003A78703630607082E
:104258000317C4009317070193D7070193F6870044
:10426800638A060883260401638A060A13F717007F
:104278006308070283274401232404001305000070
:10428800B307F040232CF400638A06028320C100A0
:104298000324810083244100130101016780000089
:1042A80093F72700130700006394070003274401CE
:1042B8002324E40013050000E39A06FC8317C400D6
:1042C80013F70708E30407FC93E707042316F40031
:1042D8001305F0FF6FF09FFB13850700EF009005B3
:1042E8000317C4009317070193D7070193F68700B4
:1042F800E39A06F693F60701638E060693F74700DE
:104308006390070483260401936787002316F4004B
:104318009397070193D70701E39A06F413F7072841
:1043280013060020E304C7F4930504001385040072
:10433800EF30902D8357C400832604016FF01FF3DC
:1043480083250403638E0500930704046388F5003E
:1043580013850400EF0010140317C4002328040277
:10436800832604011377B7FD232204002320D400F9
:104378006FF09FF99307900023A0F40013670704D8
:104388002316E4001305F0FF6FF05FF003A7811B0D
:1043980083278714638C070403A747001308F001D9
:1043A800634EE806131827006306050233830701E6
:1043B8002324C30883A88718130610003316E600C1
:1043C800B3E8C80023A417192324D31093062000A8
:1043D8006304D5021307170023A2E700B387070178
:1043E80023A4B70013050000678000009307C714D3
:1043F8002324F7146FF05FFA83A6C7181307170072
:1044080023A2E70033E6C60023A6C718B38707012F
:1044180023A4B70013050000678000001305F0FF10
:1044280067800000130101FD2324810103AC811B77
:10443800232E3101232C4101232A51012328610114
:1044480023261102232481022322910223202103FF
:1044580023267101930A0500138B0500130A100027
:104468009309F0FF03298C14630809028324490087
:104478001384F4FF6342040293942400B304990064
:1044880063040B0483A74410638067051304F4FFD7
:104498009384C4FFE31634FF8320C10203248102FE
:1044A80083244102032901028329C101032A8101CE
:1044B800832A4101032B0101832BC100032C8100B6
:1044C80013010103678000008327490083A6440085
:1044D8009387F7FF638A870423A20400E38806FA18
:1044E8008327891833178A00832B4900B377F7008D
:1044F800639E0700E780060083274900E39477F767
:1045080083278C14E38427F96FF0DFF58327C91814
:1045180083A544083377F700631C070013850A0056
:10452800E78006006FF05FFD232289006FF01FFB14
:1045380013850500E78006006FF01FFC8397C50010
:10454800130101FE232C810013970701135707015C
:1045580023263101232E1100232A9100232821012B
:10456800937687001384050093090500639A061063
:10457800371700001307078083A64500B3E7E70055
:104588002396F5006350D01803278402630A070CAA
:104598009397070193D7070183A4090093963701DE
:1045A80023A009008325C40163C4061693061000DE
:1045B8001306000013850900E70007009307F0FFC2
:1045C8006308F5188357C400032784028325C401B0
:1045D80093F74700638E070083264400832704036C
:1045E8003305D540638607008327C4033305F540A8
:1045F800130605009306000013850900E70007006D
:104608009307F0FF631AF51003A709008317C40086
:10461800630407169306D0016306D700930660016A
:104628006310D70C8326040137F7FFFF1307F77FC2
:10463800B3F7E7002316F400232204002320D40054
:104648008325040323A09900638C050093070404C1
:104658006386F50013850900EF00C0632328040270
:10466800130500008320C101032481018324410133
:10467800032901018329C100130101026780000099
:1046880003A90501E30E09FC83A40500137737008D
:1046980023A02501B3842441930700006314070075
:1046A80083A745012324F400634890006FF05FFB63
:1046B8003309A900E35690FA832744028325C401ED
:1046C800938604001306090013850900E780070094
:1046D800B384A440E34EA0FC8357C4001305F0FF45
:1046E80093E707042316F4008320C1010324810102
:1046F80083244101032901018329C1001301010217
:104708006780000003A7C503E340E0E86FF05FF5AA
:10471800032504056FF0DFEB8357C40037F7FFFF6D
:104728001307F77FB3F7E700832604019397070180
:1047380093D707412316F400232204002320D40032
:1047480013973701E35E07EE2328A4046FF05FEFA9
:1047580083A70900E38807E61307D0016388E70207
:10476800130760016384E7028357C40093E70704D3
:104778002316F4006FF01FEF37F7FFFF1307F77FDB
:1047880083260401B3F7E7006FF0DFFA23A099004E
:10479800130500006FF01FED130101FE232C8100AB
:1047A800232E1100130405006306050083278503E3
:1047B800638007028397C500639607028320C101BF
:1047C8000324810113050000130101026780000022
:1047D8002326B100EF0000368325C1008397C5006A
:1047E800E38E07FC13050400032481018320C10123
:1047F800130101026FF09FD49305050063060500BD
:1048080003A5811C6FF05FF903A5811BB7450080E4
:104818009385057A6F001002130500006780000079
:10482800B7E500809385C5826F00D000130101FEB3
:10483800B7570080232E1100232C8100232A9100D2
:104848002328210123263101232441012322510158
:10485800232061010324450093878782232EF502D4
:104868001307C52E930730002324E52E2322F52EA7
:104878002320052E93074000130905002326F40082
:104888001306800093050000232204062320040059
:10489800232204002324040023280400232A0400DC
:1048A800232C04001305C405EFC01FB8379B0080F4
:1048B80083248900B79A0080379A0080B7990080CE
:1048C800130B8B20938ACA26130A4A2F9389C9355A
:1048D800B70701002320640323225403232444033D
:1048E80023263403232E84009387970023A6F400FD
:1048F800130680009305000023A2040623A00400E9
:1049080023A2040023A4040023A8040023AA04006B
:1049180023AC04001385C405EFC01FB10324C900EC
:10492800B707020023A0640323A2540323A444036B
:1049380023A6340323AE9400938727012326F4008B
:104948002322040623200400232204002324040035
:1049580023280400232A0400232C04001305C4057B
:104968001306800093050000EFC01FAC8320C1012F
:1049780023206403232254032324440323263403DB
:10498800232E84000324810193071000232CF902AD
:1049980083244101032901018329C100032A8100DD
:1049A800832A4100032B01001301010267800000E4
:1049B8001305000067800000130101FF2322910006
:1049C800130680069384F5FFB384C40223202101D3
:1049D80013890500232481002326110093854407A9
:1049E800EFC0CFA813040500630005021305C50036
:1049F80023200400232224012324A40013868406F0
:104A080093050000EFC05FA2130504008320C100D6
:104A180003248100832441000329010013010101BB
:104A280067800000130101FE2328210103A9811BCF
:104A380023263101232E110083278903232C81008B
:104A4800232A9100930905006386070A1309092E92
:104A58009304F0FF83274900032489009387F7FF15
:104A680063DA07006F0000089387F7FF13048406D2
:104A7800638A97060317C400E31807FEB707FFFF0A
:104A8800938717002322040623200400232204000E
:104A9800232404002326F40023280400232A0400E6
:104AA800232C040013068000930500001305C40599
:104AB800EFC09F9723280402232A04022322040418
:104AC80023240404130504008320C1010324810165
:104AD80083244101032901018329C1001301010233
:104AE8006780000003240900630C04001309040014
:104AF8006FF05FF613050900EFF05FD36FF01FF555
:104B08009305400013850900EFF01FEB2320A9004F
:104B180013040500E31C05FC9307C00023A0F9005B
:104B28006FF05FFA03A5811BB7E500809385C58206
:104B38006F00405083278503638407006780000067
:104B48006FF0DFCE6780000067800000678000009C
:104B58006780000003A5811CB755008093850582F6
:104B68006F00404203A5811CB75500809385859B43
:104B78006F004041130101FE23282101232C8100ED
:104B8800232A91002326310113840500232E1100C6
:104B980093090500138981C2EFC0DF968326890037
:104BA800371700009307F7FE83A446003384874035
:104BB80093F4C4FF330494001354C4001304F4FFA3
:104BC8001314C400634EE400930500001385090024
:104BD800EFC01F9D83278900B38797006306F502FE
:104BE80013850900EFC05F928320C101032481016E
:104BF80083244101032901018329C1001305000011
:104C08001301010267800000B30580401385090085
:104C1800EFC01F999307F0FF6304F50483A7411EB3
:104C280083268900B384844093E414003384874046
:104C38001385090023A2960023A2811EEFC0DF8CF2
:104C48008320C10103248101832441010329010137
:104C58008329C100130510001301010267800000B9
:104C68009305000013850900EFC09F93032789006F
:104C78009306F000B307E540E3D4F6F683A6C11C1B
:104C880093E717002322F7003305D54023A2A11E7E
:104C98006FF01FF563860512130101FF23248100BD
:104CA8002322910013840500930405002326110094
:104CB800EFC05F850325C4FF130784FF9377E5FFE3
:104CC8003306F700938581C28326460003A8850032
:104CD80093F6C6FF630EC8182322D6001375150075
:104CE8003308D6006310050A032384FF032848000D
:104CF8003307674083288700138501C3B38767009C
:104D0800137818006380A8140323C70023A668003B
:104D1800232413016306081C93E617002322D700F7
:104D28002320F6009306F01F63E8F60A93D73700AE
:104D3800938617009396360003A84500B386D500DE
:104D480003A5060013D6274093071000B397C700A2
:104D5800B3E70701138686FF2326C7002324A7008D
:104D680023A2F50023A0E6002326E5000324810002
:104D78008320C1001385040083244100130101012D
:104D88006FC08FF80325480013751500631C0502D2
:104D9800B387D700138501C38326860093E81700DD
:104DA8003308F700638AA6140326C60023A6C600A4
:104DB8002324D600232217012320F8006FF09FF642
:104DC8006780000093E61700232ED4FE2320F60008
:104DD8009306F01FE3FCF6F493D697001306400001
:104DE800636ED60C93D667001385960313868603E5
:104DF800131535003385A50083260500130585FFA7
:104E0800630AD51003A646001376C6FF63F6C700EB
:104E180083A68600E318D5FE03A5C6002326A700AF
:104E28002324D700032481002324E5008320C10024
:104E3800138504008324410023A6E6001301010121
:104E48006FC08FEC63180812832586000326C600FE
:104E5800B387F60093E6170023A6C5002324B600FF
:104E68002322D7003307F7002320F7006FF01FF045
:104E780013751500B387D70063100502032584FF57
:104E88003307A7408326C70003268700B387A700F8
:104E98002326D60023A4C60013E6170083A6011D07
:104EA8002322C70023A4E500E3E2D7EC83A5C11DB4
:104EB80013850400EFF01FCC6FF05FEB1306400181
:104EC8006374D602130640056364D60693D6C700FA
:104ED8001385F6061386E606131535006FF09FF165
:104EE800B387D7006FF05FEB1385C6051386B60549
:104EF800131535006FF01FF023AAE50023A8E5007D
:104F08002326A7002324A700232217012320F80023
:104F18006FF0DFE503A845001356264093071000FD
:104F28003396C7003366060123A2C5006FF01FEF52
:104F380013064015636CD60093D6F70013858607D1
:104F480013867607131535006FF0DFEA1306405510
:104F5800636CD60093D627011385D6071386C60738
:104F6800131535006FF01FE91305803F1306E0079E
:104F78006FF05FE893E617002322D7002320F6009E
:104F88006FF0DFDE130101FE23225101232E1100F1
:104F9800232C8100232A9100232821012326310173
:104FA8002324410123206101930A052E63800A0806
:104FB800138B0500130A0000930910001309F0FF72
:104FC80083A44A0003A48A009384F4FF63C60402FE
:104FD8008357C4009384F4FF63FCF9008317E4004B
:104FE8001305040063862701E7000B00336AAA0053
:104FF80013048406E39E24FD83AA0A00E3920AFCB4
:105008008320C1010324810113050A00832441017F
:10501800032901018329C100032A8100832A410051
:10502800032B01001301010267800000130A00002E
:105038006FF01FFD130101FD232A510123261102E0
:10504800232481022322910223202103232E3101CC
:10505800232C41012328610123267101930A052E7F
:1050680063860A08938B0500130B0500130A0000DA
:10507800930910001309F0FF83A44A0003A48A00CF
:105088009384F4FF63C804028357C4009384F4FF35
:1050980063FEF9008317E4009305040013050B0071
:1050A80063862701E7800B00336AAA00130484068D
:1050B800E39C24FD83AA0A00E3900AFC8320C10232
:1050C8000324810213050A008324410203290102F3
:1050D8008329C101032A8101832A4101032B01018C
:1050E800832BC1001301010367800000130A00002D
:1050F8006FF0DFFC93064500930700001305A50138
:105108003788FFFF6F00C001939717002390E600D0
:10511800939707019386260093D70701630ED5025C
:1051280003D70600137617006304060093E71700F9
:105138001357170013F62700B3650701E30606FCAB
:10514800939717002390B60093970701938626003C
:1051580093D70701E316D5FC678000009306850105
:1051680013070000130525006F00C001131717006F
:105178002390F600131707019386E6FF13570701DC
:105188006304D50483D70600139607011356064116
:105198009397170063540600136717009397070146
:1051A80093D707011376270093E51700E30006FC61
:1051B800131717002390B600131707019386E6FF0D
:1051C80013570701E310D5FC67800000130101FEA7
:1051D800370E0100231D0100231E01009385850160
:1051E8009307C10113088100130EFEFF03D70500C2
:1051F8009387E7FF9385E5FF63180702239F07FE60
:10520800E39607FF130646009306E10103D707005C
:105218001306260093872700231FE6FEE398D7FE90
:1052280013010102678000003307A70283D8270013
:1052380003D30700B376C701B386160113570701D6
:1052480093D80601330767003307170193580701FE
:105258002391D7002390E700239F17FFE39807F9CE
:105268006FF05FFA13072501130525008357E5FF43
:1052780063980700E31AA7FE130500006780000083
:105288001305100067800000130101FF232481002B
:105298000354250123229100232611009347F4FF8C
:1052A800139717019304050063160700EFF09FFB9F
:1052B80063180500B787FFFF3344F400239984007F
:1052C8008320C100032481008324410013010101CC
:1052D80067800000130101FF232481000354250186
:1052E800232611009347F4FF13971701631807004B
:1052F800EFF05FF793070000631405009357F4007D
:105308008320C100032481001385070013010101D4
:105318006780000083172501130101FF2326110070
:1053280023248100232291002320210163C0070642
:105338002390050083572501378700001307F7FFDF
:10534800B377F7002391F500130405016382E7069C
:1053580093876500239205001305E5FF1304E4FF16
:105368000357240093872700239FE7FEE31885FE51
:10537800239C05008320C10003248100832441006D
:105388000329010013010101678000009307F0FF62
:105398002390F50083572501378700001307F7FF8F
:1053A800B377F7002391F50013040501E392E7FAB8
:1053B80003572501138905009304050033F7E70017
:1053C8006318F702EFF01FEA630405021307690088
:1053D800231209009387C4FF1304E4FF83562400B3
:1053E80013072700231FD7FEE39887FE6FF09FF867
:1053F800930749009305A90193872700239F07FE78
:10540800E39CF5FE8320C10003248100832441002E
:10541800032901001301010167800000835725015A
:10542800130101FB2324810493C7F7FF232291046E
:10543800232611041397170193040500138405000C
:1054480063160700EFF01FE2631205088357240173
:1054580093C7F7FF139717016304070693058100A5
:1054680013850400EFF01FEB9305410213050400B8
:10547800EFF05FEA8355810083574102638CB704DC
:105488009307A100130761021306010283D60700E0
:10549800938727006396060883560700130727009B
:1054A80063900608E394C7FE130500008320C10437
:1054B800032481048324410413010105678000004B
:1054C80013050400EFF01FDAE30A05F81305E0FFFF
:1054D8006FF0DFFD13051000639C07041307A1009C
:1054E8009307610293872700130727000356E7FFF6
:1054F80083D6E7FF9305C103631ED600E386B7FA98
:1055080093872700130727000356E7FF83D6E7FF93
:10551800E306D6FEE3ECC6F83305A0406FF01FF9AA
:1055280013051000E38405F81305F0FF6FF01FF86A
:105538001305F0FF6FF09FFA130101FF23261100F6
:10554800EFF05FD28320C10013351500130101016C
:1055580067800000130101FF23248100232021011B
:105568002326110023229100138905001304050046
:1055780063C2050A9307F00013860500130545006A
:10558800930684019305F00063D42703930705006D
:105598009387270003D70700239FE7FEE39AD7FEE8
:1055A800231C0400130606FFE3C2C5FE1379F900A5
:1055B8009307700063D82703930784019305240099
:1055C8001307000083D607009387E7FF139686002A
:1055D8003367C7002391E70013D78600E394B7FE2B
:1055E800130989FF630A09001309F9FF1305040069
:1055F800EFF0DFB6E31A09FE8320C100032481001F
:10560800832441000329010013050000130101014F
:1056180067800000930710FFB304B04063D4F50C13
:105628009305850113090000930645001306F00051
:1056380003578401938705003369E9009387E7FFDF
:1056480003D707002391E700E39AD7FE231204004B
:10565800938404FFE34E96FC9307700063D6970487
:105668001319090113590941834784019305A401BA
:10567800130700003369F9001319090113590901C7
:1056880083D706009386260013D687003367C700A2
:1056980093978700239FE6FE139707011357070187
:1056A800E390B6FE938484FF6380040283578401E9
:1056B8009384F4FF1305040093F7170033E92701D7
:1056C800EFF05FA3E39404FE8320C100032481006C
:1056D800333520018324410003290100130101010E
:1056E80067800000930790FF63C6F5001309000068
:1056F8006FF0DFFB13090000930644006FF0DFF63C
:1057080083574500130101FF23229100232611002E
:10571800232481002320210193040500639C070CA6
:1057280003576500130400009317070193D7074137
:1057380063C4070A9306A5011306000A6318070243
:10574800938764006F00800003D7070093872700C2
:10575800239EE7FEE39AF6FE239C0400130404014B
:10576800630CC40603D76400E30C07FC937707F0C7
:1057780063900704138584019385240013070000B0
:105788009307050083D607009387E7FF13968600E3
:105798003367C7002391E70013D78600E394F5FE2B
:1057A80003D7640013048400937707F0E38807FCA9
:1057B8001309000A6F00400113041400EFF01F9A48
:1057C800634C890003D76400131707011357074177
:1057D80013850400E35207FE130504008320C1006B
:1057E80003248100832441000329010013010101DE
:1057F8006780000013F707F0130400006310070424
:105808001309F0F66F0040011304F4FFEFF09F8EC8
:10581800E30424FD83D7440013850400E39607FEC0
:10582800130504008320C100032481008324410060
:105838000329010013010101678000009306450058
:105848009305A501130700006F00800083D70600A9
:1058580013D687003367C700939787002390E60025
:10586800139707019386260013570701E390B6FEA6
:1058780083D74400130480FF6FF09FF8130101FEE3
:10588800232C8100232A910023282101232631017A
:105898002324410123225101138906009384070020
:1058A800232E11001304050093890500130A06002E
:1058B800930A0700EFF0DFE4930700093309A940D2
:1058C80063DEA706B78700009387E7FF63DE27211B
:1058D80063880A1E03A5440083A70400638EA70EED
:1058E8001387A4019387440313072700231F07FE88
:1058F800E31CF7FE930780036304F53663D2A7061B
:1059080093070004630EF52E930710076310F53212
:10591800B78700409387F7FF1307A00023AAF40076
:10592800B787FFFF23A4E400239CF40023A6E40028
:105938009307A000378700006F0080066356091E92
:10594800930700F7635EF91A930724001304A40170
:1059580093872700239F07FEE39C87FE6F000014B0
:10596800930780016308F526930750036310F52C0D
:10597800B70700049387F77F1307600023AAF40092
:10598800B71700009387078023A4E40023A6E40048
:1059980037170000239CF400130707809307600063
:1059A8009387870093971700B387F4002395E70040
:1059B80023A0A40063422003930700096308F51E8F
:1059C800835784011305040093F71700B3E9F9001E
:1059D800EFF04FF203A5440083A5840083D7440168
:1059E8001308F008139615003306C4000357060081
:1059F800B376F700634AA8021308B0006346B802FA
:105A08001307060093058401835727006384070062
:105A180093E616002311070013072700E396E5FE17
:105A28000357060083D7440193C7F7FFB3F7E7008E
:105A38002310F60083D7640133F7D7006300070407
:105A48006382D71213862403130784019384C40145
:105A58009306000083570600835507001307E7FFE6
:105A68001306E6FFB387B700B387D7002311F70003
:105A780093D7070193F61700E31E96FC635620118F
:105A880083574400639C070AB7870000231C04005F
:105A98009387E7FF63C82703231124018320C101EB
:105AA8000324810183244101032901018329C100C1
:105AB800032A8100832A4100130101026780000044
:105AC800231C0400B787FFFF93C7F7FF2311F400D7
:105AD8009307440013048401239007009387270049
:105AE800E31CF4FE6FF09FFB930724001304A4014A
:105AF80093872700239F07FEE39C87FE6FF01FFA1A
:105B08009305090013050400EFF0DFA46304050002
:105B180093091000638A0A0A03A5440083A70400B6
:105B2800E390A7DC6FF05FE9E3800AF603A5440081
:105B380083A70400E316F5DA6FF0DFE71305040026
:105B4800EFF04FDBB787000013091900231C04008E
:105B58009387E7FFE3C827F7E35009F4231104000C
:105B68006FF0DFF3639A090E83A7C40003D784019B
:105B780093971700B307F40083D70700B3F7E7003C
:105B8800E39207ECE34E20EF930700096306F50064
:105B980013050400EFF08FDC83574400E39007FA05
:105BA800231C0400E34C09FA6FF01FEF03A68400DE
:105BB80083D74401131616003306C40003570600A2
:105BC800B3F6E7006FF05FE6231C0400231104001E
:105BD8006FF0DFECB70780009387F70F13074000DB
:105BE80023AAF4009307001023A4E400239CF400E4
:105BF80023A6E40093074000130700106FF05FDA54
:105C08009307700023A4F400B70701809387F7FF78
:105C180023AAF40093071000239CF4009307600064
:105C280023A6F400130710006FF09FD79307C00056
:105C380023A4F400B70701809387F7FF23AAF40091
:105C480093071000239CF4009307B00023A6F400E8
:105C5800130710006FF0DFD4E3060ADE6FF01FE2CF
:105C6800B70780009387F70F1307600023AAF40093
:105C78009307001023A4E400239CF40023A6E40067
:105C880093076000130700106FF09FD1130101FD07
:105C9800232E310183592500232291029384050084
:105CA800232611022324810223202103232C4101CE
:105CB80013090600232A51012328610123267101B3
:105CC80023248101232291012320A101130A050025
:105CD800EFF01FA303D42400B389A940138504005F
:105CE800EFF01FA2930A49033304A4401307E90401
:105CF80093870A0093872700239F07FEE39CE7FE0C
:105D0800634A3409930B4A00138B44009389F9FFC3
:105D1800930CAA01138C240013070B0093870B0024
:105D2800938727001307270003D6E7FF8356E7FF6B
:105D3800631AD60AE39697FF93068A0113878401AC
:105D4800130600008357070083D506001307E7FFF3
:105D5800B387C740B387B7402311F70093D707012C
:105D68009386E6FF13F61700E31EECFC130D1000F4
:105D780013850A00EFF08FBE8357C9041304F4FF9C
:105D880013850400336DFD002316A905EFF00FBD40
:105D9800E31434F993060400032481028320C1022A
:105DA8008329C101032A8101832A4101032B0101AF
:105DB800832BC100032C8100832C4100032D01009B
:105DC8009307090013850400032901028324410273
:105DD80013070000130600009305000013010103D8
:105DE8006FF0DFA9130D0000E3E4C6F86FF0DFF4ED
:105DF8000357050083572500630207043787FFFF11
:105E0800B3E7E7002399F50003572500B78700009B
:105E18009387F7FF630EF7029307650093850501E3
:105E2800130585019387270003D7E7FF9385E5FFCF
:105E38002391E500E398A7FE678000002399F50009
:105E480003572500B78700009387F7FFE316F7FC91
:105E5800930765001305A50103D70700938727005B
:105E6800631A0702E39AA7FE1387250193870500A3
:105E780093872700239F07FEE31CF7FE83D725019E
:105E8800378700001307F7FFB3E7E7002399F5000A
:105E98006780000013870501938705009387270013
:105EA800239F07FEE39CE7FEB7C7FF7F23A8F50003
:105EB80067800000130101F7232A5107835A25013F
:105EC800B78700009387F7FF2324810823229108CE
:105ED80023202109232E31072328610723261108AF
:105EE800232C4107232671072324810723229107A6
:105EF80033FB5701930405001389050013040600BA
:105F0800938906006318FB0AEFF0CFB5631A0520E2
:105F1800035A2901B3774B016392672313050900DC
:105F2800EFF04FB46314050A13850400EFF0CFE0D7
:105F3800631C0520B78700009387F7FF33FA4701F2
:105F4800131A0A01135A0A016312FA2C13050900DD
:105F5800EFF08FDE631E053083D72401B377FA0094
:105F680063824721138504009305C100EFF08FBABF
:105F78001305090093058102EFF0CFB98354E100BE
:105F88000359A102639A0408930701019306410289
:105F9800638CF62A9387270003D7E7FFE30A07FEF7
:105FA8001305C100EFF0CFF5B304A0400357A102D9
:105FB8006F00C00603DA250133F74701E314F7FA47
:105FC80013850500EFF00FAAE30605F6130749014C
:105FD800130929008357E9FF13042400231FF4FE43
:105FE800E31827FF8320C10803248108832441087C
:105FF800032901088329C107032A8107832A410746
:10600800032B0107832BC106032C8106832C410631
:10601800130101096780000013070900130B090029
:106028009307C10293060104631207026388F622EC
:106038009387270003D7E7FFE30A07FE13058102CA
:10604800EFF00FEC0357A102330BA94083578102ED
:10605800938A8903239BE902239AF9021387E904A7
:1060680093870A002390070093872700E31CF7FE15
:10607800938BC904130A000013094102930C010110
:10608800130C6104035509001309E9FF631E051287
:1060980003D7C90493870B00336AEA009387E7FFA5
:1060A80003D707002391E700E39A57FF239C0902CF
:1060B800E31A99FD13874903930781029306210484
:1060C800035607009387270013072700239FC7FE5F
:1060D800E398F6FEB7C6FFFFB384640193862600F3
:1060E8009387090013070004B386D4001306000041
:1060F80093050A0013058102EFF04FF80357C1001A
:1061080083578102630CF71A9307F0FF2314F102F7
:106118009305040013058102EFF09FCD6FF09FEC0B
:10612800138744019384240083D7E4FF13042400D5
:10613800231FF4FEE398E4FE6FF0DFEA1385040002
:10614800EFF08FBF6306050CB75501809385458135
:1061580013050900EFF08FAC630E0512035A2901ED
:106168006FF05FDD13850400EFF00FBD63180500C5
:1061780013050900EFF04FBCE30605DE13850400A4
:10618800EFF04F959304050013050900EFF08F9485
:106198006382A412B787FFFF2319F40013072401B1
:1061A8009307040093872700239F07FEE39CE7FEDD
:1061B80083572401378700001307F7FFB3E7E70089
:1061C8002319F4006FF01FE21306410493058102BE
:1061D800EFE0DFFF13860B00930500001307C105EE
:1061E80003550600835707001306E6FF1307E7FF6A
:1061F800B387A700B387B7002311F60093D7070129
:1062080093F51700E31E87FD6FF09FE883DA2401FA
:10621800B78700009387F7FFB3FA5701939A0A01EB
:1062280093DA0A01E390FAD413850400EFF0CFB0B3
:10623800E31605F48357290193C7F7FF139717014E
:10624800E31207D26FF0DFF293074401130424002E
:10625800231F04FEE39C87FE6FF0DFD893074401F9
:1062680013042400231F04FEE31CF4FE6FF09FD7E1
:10627800B75501809385458113850400EFF00F9A87
:10628800630A050083D72401B377FA00E38E47F940
:106298006FF05FFA13070401930704009387270040
:1062A800239F07FEE39CE7FEB7C7FF7F2328F40080
:1062B8006FF05FD3231904006FF05FEE231401021F
:1062C8006FF01FE583572501130101F52324810A87
:1062D80093C7F7FF2322910A2320210B2328610962
:1062E8002326110A232E3109232C4109232A510977
:1062F8002326710923248109232291092320A10936
:10630800232EB1071397170193040500138905007D
:1063180013040600138B060063160700EFE09FF4D2
:10632800631A05368357290193C7F7FF1397170197
:10633800630E0708B75901809385498113850400C6
:10634800EFF0CF8D6304051083D924010357290189
:10635800B78700009387F7FFB3F9370133FAE700EF
:10636800639AF90813850400EFF00F9D6308051080
:1063780063183A0113050900EFF00F9C6310050E2E
:106388009307440113042400231F04FEE31CF4FEB6
:106398008320C10A0324810A8324410A0329010AAC
:1063A8008329C109032A8109832A4109032B010989
:1063B800832BC108032C8108832C4108032D010875
:1063C800832DC1071301010B678000001305090025
:1063D800EFE05FE9E30005F6130749011309290017
:1063E8008357E9FF13042400231FF4FEE31827FF53
:1063F8006FF01FFA6306FA08138504009305C101BC
:10640800EFE05FF19305810313050900EFE09FF0CA
:10641800835BA1038354E10163900B0C9307C103D1
:10642800930B01056380FB349387270083D6E7FF2E
:10643800E38A06FE13058103EFF08FACB307A04093
:106448002326F1000357E1016F00800993854981F4
:1064580013050900EFE09FFCE31805EE130704019C
:106468009307040093872700239F07FEE39CE7FE1A
:10647800B7C7FF7F2328F4006FF09FF1E31E3AF7B8
:1064880013050900EFF04F8BE30805F613850400A8
:10649800EFE05FE49304050013050900EFE09FE3D4
:1064A8006384A432B787FFFF2319F400130724017C
:1064B8009307040093872700239F07FEE39CE7FECA
:1064C80083572401378700001307F7FFB3E7E70076
:1064D8002319F4006FF0DFEB232671011387040002
:1064E80023249100930701029306410363120702D4
:1064F8006384F6289387270003D7E7FFE30A07FE9C
:106508001305C101EFF0CF9FB387A4402324F10006
:1065180003278103130D8B0393070D00232AEB0236
:106528009304EB0493872700239F07FEE39C97FEC1
:1065380013058103EFE01FBC035C2102B7090100CA
:10654800930B0105131A0C01330A8A41930AA1031C
:106558009389F9FF930CE106130961050355C103FB
:106568008357E103938D0900131505013305F500E1
:106578006368AA0033558503931D050193DD0D015A
:10658800130641059305C10113850D00EFE01FC4F3
:106598001306C10393078105938727001306260076
:1065A80003D5E7FF8355E6FF6314B510E39697FF1D
:1065B800130500009305C10613860B0083570600D8
:1065C80003D805001306E6FFB387A740B387074142
:1065D8002311F60093D707019385E5FF13F51700FC
:1065E800E31E56FD2310BD019307C10393872700BF
:1065F80003D60700239FC7FEE39A77FF23180104F9
:10660800130D2D00E39CA4F5930500009307C10327
:10661800930621059387270003D7E7FFB3E5E50035
:10662800E39AD7FEB335B00013074B0393078103F2
:10663800035607009387270013072700239FC7FEE9
:10664800E398F6FE8327C10003278100B7460000C0
:106658009386F6FFB38BE740B386DB0093070B0006
:10666800130700041306000013058103EFF00FA1C0
:106678000357C101835781036300F7149307F0FFA1
:10668800231CF1029305040013058103EFF04FF674
:106698006FF01FD0138744019384240083D7E4FF4D
:1066A80013042400231FF4FEE398E4FE6FF05FCE8A
:1066B800E3F0A5F09387FDFF9398070193D80801AD
:1066C80013050000930541031306C106835706000E
:1066D80003D805001306E6FFB387A740B387074131
:1066E8002311F60093D707019385E5FF13F51700EB
:1066F800E31E26FD1306C103930781059387270030
:106708001306260003D5E7FF8355E6FF6318B50097
:10671800E39697FF938D08006FF09FE9E3FCA5FED1
:10672800938DEDFF939D0D0193DD0D011305000081
:10673800930541031306C1068357060003D80500D5
:106748001306E6FFB387A740B38707412311F60076
:1067580093D707019385E5FF13F51700E31E26FD80
:106768006FF01FE59307440113042400231F04FE60
:10677800E39C87FE6FF0DFC10357C1018357810394
:106788006300F704B787FFFF2319F40013072401F8
:106798009307040093872700239F07FEE39CE7FEE7
:1067A80083572401378700001307F7FFB3E7E70093
:1067B8002319F4006FF0DFBD231C01026FF09FEC7A
:1067C800231904006FF09FFC231904006FF01FCEFB
:1067D800130101FD232481022326110213840500DD
:1067E800930741001307E10193872700239F07FEC2
:1067F800E39CE7FE0356E5009317060193D707418C
:1068080063CA0706B78700009387F7FF23120100C2
:106818003376F600630CF6069307E5002313C100F0
:106828001307A1009387E7FF83D607001307270004
:10683800231FD7FEE318F5FE631206022314010096
:106848009305040013054100EFF08FDA8320C1029D
:1068580003248102130101036780000093071000DD
:106868009305F0FF130541002314F100EFE09FCEDC
:106878006FF01FFD9307F0FF2312F100B7870000A8
:106888009387F7FF3376F600E318F6F893070500C9
:106898009306E50003D7070093872700631C0704C6
:1068A800E39AF6FE13074401930704009387270031
:1068B800239F07FEE39CE7FE1307240193070400C8
:1068C80093872700239F07FEE39CE7FE8357240155
:1068D800378700001307F7FFB3E7E7002319F40031
:1068E8008317E500E3D407F613050400EFE0DF990A
:1068F8006FF0DFF51307040193070400938727005F
:10690800239F07FEE39CE7FEB7C7FF7F2328F40019
:106918006FF0DFF383AE050003AE450003A38500E7
:1069280083A5C500130101E183280504232EB102C4
:106938009305F0FF2320B116930500092324811E37
:106948002326711D2326111E2322911E2320211F79
:10695800232E311D232C411D232A511D2328611D5F
:106968002324811D2322911D2320A11D232EB11B29
:106978002328D103232AC103232C61022322B11621
:106988002320C1002324D1002326E100232C010168
:10699800930B05001384070063820802032745044C
:1069A8009307100093850800B397E70023A2E80037
:1069B80023A4F800EF10807623A00B04130A010625
:1069C8001305010393050A00EFF09FE013050A0081
:1069D800EFE05F90630C0520032701009307100088
:1069E8002320F40093073000630AF720930740013F
:1069F8002322F100E31E076083572107032741166E
:106A080093C7F7FF232AE1001397170163180700BC
:106A180013050A00EFE01F85E312054493070009F8
:106A28002322F1161307C10793070A00130641072B
:106A38009387270083D6E7FF13072700231FD7FE76
:106A4800E398C7FE0356E1082328010093170601BF
:106A580093D7074163DE070013161601B707010035
:106A6800135616019387F7FF2317C1082328F1004F
:106A7800375B0180130D4B81930D4D019306000088
:106A88009307810913870D00930CC10A6F008000DA
:106A98008356070093872700239FD7FE13072700F5
:106AA800E39897FF63080616B78700009387F7FFF8
:106AB800E30CF6588317C108E3D207629305C107B0
:106AC80013850D00EFE09F9563020516E348051056
:106AD8008357E108E39E07688317C1089304000001
:106AE8009309011663C4070213048D111306C10725
:106AF800938609009305060013050400EFF08FBB89
:106B08008317C1089384F4FFE3D207FE1304010D31
:106B1800130C810E130704009307C107130601091C
:106B28009387270083D6E7FF13072700231FD7FE85
:106B3800E398C7FE930600009307810913870D00A9
:106B48006F0080008356070093872700239FD7FE96
:106B580013072700E39897FF930A8D02930CCD1231
:106B680037F9FFFF130D8D116F00C000938C4C0196
:106B7800938A4A019305040013850D00EFE01F8AEC
:106B8800930504006356A00413850C00EFE01F89E9
:106B98009386090013060400930504006342050266
:106BA80013850A00EFF00FB11306810993860900D7
:106BB8009305060013850A00EFF0CFAFB3842401D4
:106BC8009357F901B387270113D91740E390AAFB1C
:106BD800130681099386090093850D0013050600A5
:106BE800EFF04FEE130941126F00800503270100F3
:106BF8002320040093073000E31AF7DE8324810082
:106C0800232291009307A002E3D897DE2322F10004
:106C18006FF09FDE9307C1079306E10803D70700CB
:106C280093872700E31C07E8E39AF6FE9304000025
:106C380013094112930901161304010D130C810E57
:106C48009305040013058109EFE0CFEC13078109D0
:106C5800930704009387270083D6E7FF13072700CD
:106C6800231FD7FEE39887FF930504001305C10788
:106C78002318010AEFE00FEA9307C1071304240061
:106C88000357E4FF93872700239FE7FEE31884FF59
:106C980013058109138609009305C107231A010802
:106CA800EFE0DFFE0355C11A6314051C930C41097C
:106CB8001304E107930A610B93054B811305C10780
:106CC800EFE0CFF56306051A1307000093860C0062
:106CD8006F00C001131717002390F6001317070160
:106CE8009386E6FF135707016384860483D706005B
:106CF800139607011356064193971700635406002D
:106D0800136717009397070193D707011376270096
:106D180093E51700E30006FC131717002390B6004D
:106D2800131707019386E6FF13570701E39086FCC4
:106D38001307410B9307C1079387270083D6E7FF03
:106D480013072700231FD7FEE39897FF2316010C8C
:106D5800130700009306C10C6F00C001131717003A
:106D68002390F600131707019386E6FF13570701D0
:106D78006384560583D70600139607011356064108
:106D8800939717006354060013671700939707013A
:106D980093D707011376270093E51700E30006FC55
:106DA800131717002390B600131707019386E6FF01
:106DB80013570701E39056FD130700009306C10C13
:106DC8006F00C001131717002390F600131707016F
:106DD8009386E6FF135707016384560583D7060099
:106DE800139607011356064193971700635406003C
:106DF800136717009397070193D7070113762700A6
:106E080093E51700E30006FC131717002390B6005C
:106E1800131707019386E6FF13570701E39056FD02
:106E28001306000093860C001307C10C83D50600D7
:106E3800835707009386E6FF1307E7FFB387B7007A
:106E4800B387C7002391F60093D7070113F61700FD
:106E5800E31E57FD13058109138609009305C10731
:106E6800EFE0DFE20355C11A9384F4FFE30605E47B
:106E78008327010163820704032701009307D002D7
:106E88002302F11293073000032441006302F70440
:106E98009307A000E304F520130505039307E00218
:106EA800A302A1122303F1126342047A9307711219
:106EB8002328F1006F00C004032701009307000294
:106EC8002302F1129307300003244100E312F7FC78
:106ED800330494009307A002E3DC87FA9307A00029
:106EE800E308F5189307E002130505032303F112DD
:106EF80093077112A302A1121304A0022328F10020
:106F0800930C0000930A410B232E910093840C00EC
:106F1800938C0A00938A090083290101930D410982
:106F2800130CE107130D610B9306000013860D0087
:106F38006F00C001939616002310F6009396060181
:106F48001306E6FF93D606016304860583570600F9
:106F58009395070193D505419397170063D40500CE
:106F680093E616009397070193D7070193F5260038
:106F780013E51700E38005FC939616002310A6007E
:106F8800939606011306E6FF93D60601E31086FDE5
:106F980093860C009307C1079387270003D6E7FF62
:106FA80093862600239FC6FEE398B7FF2316010C9D
:106FB800930600001306C10C6F00C00193961600DB
:106FC8002310F600939606011306E6FF93D60601F2
:106FD8006304A605835706009395070193D50541D9
:106FE8009397170063D4050093E61600939707015B
:106FF80093D7070193F5260013E51700E38005FCF6
:10700800939616002310A600939606011306E6FF32
:1070180093D60601E310A6FD930600001306C10CE3
:107028006F00C001939616002310F6009396060190
:107038001306E6FF93D606016304A60583570600E8
:107048009395070193D505419397170063D40500DD
:1070580093E616009397070193D7070193F5260047
:1070680013E51700E38005FC939616002310A6008D
:10707800939606011306E6FF93D60601E310A6FDD4
:107088009305000013860D009306C10C03550600F6
:1070980083D706001306E6FF9386E6FFB387A700AB
:1070A800B387B7002311F60093D7070193F51700AC
:1070B800E39EA6FD13860A009305C10713058109FF
:1070C800EFE0DFBC8357C11AB3869900938414009C
:1070D800138607032380C600E35894E403270101BD
:1070E8008324C10193091400B3093701B30C870045
:1070F80013074000635EF70613075000E380E700BC
:1071080083C7E9FF1387E9FF93F7F7076340047C18
:107118009306E0026382D704938617002300D70002
:1071280093068003930500031306E002130580030A
:1071380063C8F6006F00C0032300D700637AF50226
:107148002300B7001307F7FF8347070093F7F707F4
:1071580093861700E392C7FE8347F7FF93068003E1
:10716800E3F2F6009307100393841400A30FF7FECD
:10717800B7550180138604009385C5A813850C00B4
:10718800EF20800083572107032741012328911608
:1071980093C7F7FF2322E11613971701631E070011
:1071A80013050A00EFE04FB96310052213050A0022
:1071B800EFE04F8B631A05208326C10083474112F5
:1071C8001387140023A0E600E380070C1307E002EE
:1071D8006380E706930709009306E0026F008000CA
:1071E800630AD7049387170003C70700E31A07FE4B
:1071F800930650046366F9006F0040016388270115
:107208009387F7FF03C70700E31AD7FE2380070019
:1072180093070900930600021306D00203C707006C
:107228006304D700631AC702938717006FF01FFF24
:107238009307090003C7170093871700A38FE7FE7A
:10724800E30807FA03C7170093871700A38FE7FE21
:10725800E31207FE6FF0DFF9130409006F00C000A6
:1072680003C70700138406002300E40093061400F4
:1072780093871700E31607FE832601009307200073
:107288000347F4FF6386F6128327410093860700BD
:1072980063D4970093860400930700036316F702EC
:1072A800B307244163D2F602130600036F0080007F
:1072B80063DCE6001304F4FF8347F4FF23000400B3
:1072C80033072441E386C7FE0327010093073000F4
:1072D8006302F70A8327810023A20B041386970011
:1072E8009307700163F2C70C13071000930740005F
:1072F8009397170093864701930507001307170014
:10730800E378D6FE23A2BB0413850B00EF0090564A
:1073180023A0AB049305090093040500EF20C01BCC
:107328008327810163880700330424413384840060
:1073380023A087008320C11E0324811E1385040017
:107348000329011E8324411E8329C11D032A811D8F
:10735800832A411D032B011D832BC11C032C811C77
:10736800832C411C032D011C832DC11B1301011FFC
:107378006780000083274100B384970063C0044AF4
:107388008327C1000327810083A70700B307F700FD
:107398002324F1008327810023A20B0413863700DE
:1073A80093077001E3E2C7F4930500006FF0DFF57F
:1073B80093070003E310F7F2B30724419306100084
:1073C800E3C4F6EE6FF01FF10327C100B7270000F2
:1073D8009387F7702320F7006FF09FE3930A410B20
:1073E80013870A009307C10713060109938727002B
:1073F80083D6E7FF13072700231FD7FEE398C7FEAE
:10740800B74700009387E7082313F10CB7870000FC
:107418009387F7FF232EF100B7C7FFFF1309411227
:107428001304010D130E000113038D0C938727001D
:107438002324710323222103930400001309040069
:1074480093090116130CA10A2320F102930B0E00D5
:1074580013040300938609001306810993850A0023
:1074680013050400EFE01FE61307C1049307810921
:107478009387270083D6E7FF13072700231FD7FE2C
:10748800E39897FF8327C1018355E10533F6F5009B
:10749800832701023305F600635CA0381306000950
:1074A8003306A640130709009307C10493872700F2
:1074B80083D6E7FF13072700231FD7FEE39847FF6C
:1074C8006354C0069307F0001307090063DCC70282
:1074D800130606FF93564600138716001317170066
:1074E8003307E9009307090093872700239F07FEC6
:1074F800E39CE7FE130600083306A6409396460071
:107508003306D640131616003306CD0083570700FE
:1075180083560623B3F7D7002310F7009395050188
:1075280093D5054163CC0514930781091307090016
:1075380003D6070083560700938727001307270001
:107548006314D602E316FCFE13870A009307810929
:107558009387270083D6E7FF13072700231FD7FE4B
:10756800E39897FFB3847401130444019307CD1281
:1075780093DB1B00E310F4EE8357610C0357E1081B
:1075880013040900832B8102B387E70037C7FFFF85
:10759800130727F703294102B387E7002313F10CE8
:1075A8001307C10793870A001306810C93872700E6
:1075B80083D6E7FF13072700231FD7FEE398C7FEEC
:1075C80013070000930781096F00800003D70D009F
:1075D80093872700239FE7FE938D2D00E39897FF5D
:1075E800930C8D02371C0000130D8D116F000001E4
:1075F800135C1C006388AC2D938C4C0193850A00A6
:1076080013050D00EFD09FE193850A00634CA02A73
:1076180013850C00EFD09FE0E34CA0FC9386090093
:1076280013860A0093850A0013850C00EFE09FC9B2
:1076380013068109938609009305060013850C003B
:10764800EFE05F87B38484016FF09FFA8357C11A14
:10765800930C6112930971126FF09FA913094112DB
:10766800B7550180938585A613050900B724000046
:10767800EF1090319384F4706FF0DFB09307C1047A
:10768800130709006F00C0009306E105E38EF6E8D2
:1076980003D60700835607009387270013072700A0
:1076A800E304D6FE8357210E0327C101B377F70001
:1076B800639EE70013050900EFD0DFBAE31605E67D
:1076C80013050900EFD05FE7E31005E69305C10E47
:1076D80013850D00EFD01FC4930581101305090011
:1076E800EFD05FC30356C10E0355A1108358E10EB6
:1076F8001346F6FF13160601135606012316C10E8C
:10770800B385A84093060500635EB0068326410250
:107718001307811093070112130727008355E7FF0A
:1077280093862600239FB6FEE318F7FE231E011258
:10773800130781109306C10E6F00800003D6060060
:1077480013072700231FC7FE93862600E318F7FEBA
:1077580083274102231001121307C10E1306C11318
:107768009387270083D6E7FF13072700231FD7FE39
:10777800E398C7FE8356A110B305154123120110E3
:1077880013850600638A05302326D1029307F0F695
:1077980063C8F5061305C10EEFD0DFDB8326C102EF
:1077A8009305050093070112130541100356C10EF6
:1077B80003578110630EE632130700001306070013
:1077C80003D70700035805009387E7FF3307C7402F
:1077D800330707412391E700135707011376170072
:1077E8001307A1101305E5FFE39CE7FC130610003F
:1077F800938709001307000413058110EFE00F8831
:107808009305090013058110EFE08FDE6FF0DFD1DB
:10781800832781009384F7FF6FF08FBE8327C10011
:10782800230201121304090023A007006FF09FB67A
:10783800930709001307410E93872700239F07FE2C
:10784800E39CE7FE6FF09FCD8327010113094112E6
:10785800638C070EB7550180938505A713050900AA
:10786800B7240000EF1050129384F4706FF09F91CA
:1078780093071003A302F1129307E0022303F11206
:10788800938414001304900293070003A303F112D6
:10789800930781122328F1006FF08FE693071003F6
:1078A800A302F1129307E0022303F1129384140058
:1078B8006340801E930C7112E31C048A23289101F3
:1078C8006FF00FE4130C810E6FF08FB7930710035E
:1078D800238FF9FE938414006FF09F8913094112D6
:1078E800B7550180938585A813050900B7240000C2
:1078F800EF1090099384F4706FF0DF889305810985
:107908001305C107EFE0CFCE93054B81130581091D
:10791800EFD0DFB0631605FEE34C048483C7E9FFAC
:10792800138727FD133717001347F7FF3387EC003A
:107938000347070013771700E30C07821387E9FF53
:1079480093F7F7076FF0CFFCB75501809385C5A76C
:1079580013050900B7240000EF1010039384F47096
:107968006FF05F8293871700A30FF7FE6FF05F80B9
:107978001304010D930504001305C107B74A00005D
:10798800EFD05F9993040000130C810E1309C10C0A
:107998009309210D938AEAFF8357810E93F77700A5
:1079A800639A070C1307410B93070400938727007A
:1079B80083D6E7FF13072700231FD7FEE39887FF27
:1079C8001305410B2316010CEFD0CFF21305410B21
:1079D800EFD04FF2130600009306090013070C00BE
:1079E80083D50600835707009386E6FF1307E7FF52
:1079F800B387B700B387C7002391F60093D7070171
:107A080013F61700E31E37FD8357610B0357810BED
:107A180093873700231BF10A630007021305410B04
:107A2800EFD04FED8357610B0357810B93871700F6
:107A3800231BF10AE31407FE8357C10C639C07025A
:107A48008357610B63E8FA02130704009307410B9D
:107A58009387270083D6E7FF13072700231FD7FE46
:107A6800E39827FF2314010E9384F4FF930750FD36
:107A7800E394F4F29305C10713050400EFE04FB750
:107A8800930901166FF00F89930709006FF00FF83B
:107A98001304F4FF6FF05FDF1307C1109307010FA2
:107AA800938727001307270083D8E7FF0356E7FFCC
:107AB8006398C80213066110E394C7FE0357C10E0A
:107AC800835781106302F706930709001307410ED5
:107AD80093872700239F07FEE39CE7FE6FF0DFA450
:107AE8006366160D93070112130541106FF01FCC42
:107AF800130700001303E10E03D80700035605001F
:107B08009387E7FF1305E5FF330606013307E60011
:107B18002391E7001357070113771700E31E65FC4D
:107B2800130600006FF0DFCC138706006392060689
:107B38008317E11063CE0704930601126F00000259
:107B48002390F60013171700131707019386E6FF13
:107B58009307A11013570701E384F6CA83D70600D9
:107B680013960701135606419397170063540600AE
:107B7800136717009397070193D707011376270018
:107B880093E51700E30E06FA2390B6006FF09FFB0B
:107B98001306C11093070112631207086382C7080E
:107BA80003570600130626006FF01FFF0326410245
:107BB8001307811093070112130727000355E7FFE6
:107BC80013062600231FA6FEE318F7FE231E011244
:107BD800130681101307C10E130541101307270060
:107BE8000358E7FF13062600231F06FFE318A7FE26
:107BF80003274102231001129308C10E1306C11373
:107C0800130727000358E7FF93882800239F08FFDE
:107C1800E318C7FE231201106FF05FB91385160031
:107C28002315A1106FF0DFBD032785008327C5004A
:107C38000326050083264500130101FC13050100F6
:107C4800930541012324E1002326F100232E11028C
:107C58002320C1002322D100EFE09FB783576102A0
:107C68001305000093C7F7FF13971701631A07005E
:107C780013054101EFD00FDF13351500130515006B
:107C88008320C10313010104678000001305050F59
:107C980067800000138501126780000013850112B8
:107CA80067800000130101FF2326110023248100AF
:107CB80023229100630C0602B7550180938545A9DC
:107CC8001305060093040600EF104069375401803D
:107CD80063120502130504A98320C100032481004F
:107CE800832441001301010167800000375401809B
:107CF8006FF05FFE930504A913850400EF1000667A
:107D0800E30A05FCB7550180938545801385040077
:107D1800EF10C064E30005FC130500006FF0DFFB03
:107D280003C58115678000001386050093050500CB
:107D380003A5811C6FF01FF7130101F923248106A5
:107D4800138405008395E50023229106232021074B
:107D580023261106930406001389060063CA050446
:107D680013068100EF50505B634405040327C100EC
:107D7800B7F700008320C106B3F7E70037E7FFFF36
:107D8800B387E70093B71700032481062320F9007F
:107D98009307004023A0F400371500008324410610
:107DA80003290106130505801301010767800000F8
:107DB8008357C4002320090093F707086384070248
:107DC8008320C106032481069307000423A0F4003E
:107DD8000329010683244106130500001301010746
:107DE800678000008320C1060324810693070040B2
:107DF80023A0F4000329010683244106130500008B
:107E0800130101076780000003D7C500130101FEB5
:107E1800232C8100232E1100232A910023282101DD
:107E280013772700138405006308070213873504B6
:107E380023A0E50023A8E5001307100023AAE50006
:107E48008320C10103248101832441010329010105
:107E580013010102678000009306C1001306810028
:107E680093040500EFF05FED8325810013090500F9
:107E780013850400EF809FDF8317C400630805049F
:107E8800375700801307878223AEE4020327810057
:107E98008326C10093E707082316F4002320A400D3
:107EA8002328A400232AE40063980604B3E72701E3
:107EB8002316F4008320C101032481018324410196
:107EC80003290101130101026780000013F707204D
:107ED800E31807F693F7C7FF93E72700130734045F
:107EE8002316F400930710002320E4002328E4005D
:107EF800232AF4006FF0DFF48315E40013850400EF
:107F0800EF60C012631605008317C4006FF01FFAF4
:107F18008357C40093F7C7FF93E7170093970701A8
:107F280093D707416FF09FF803A34111670003003F
:107F3800638005026302060463880604834706001B
:107F480023A0F500034506003335A0006780000034
:107F5800130101FF9305C10063040602638A060248
:107F68008347060023A0F500034506003335A0002B
:107F780013010101678000001305000067800000FD
:107F8800130500006FF0DFFE1305E0FF67800000B7
:107F98001305E0FF6FF0DFFD9377350013F8F50F59
:107FA8006386070C9307F6FF630E06040347050074
:107FB800630C07059306F0FF6F0040019387F7FFF6
:107FC8006382D704034705006300070513051500FE
:107FD80013773500E31407FE130730006368F702D0
:107FE800638207020347050063000703B307F50030
:107FF8006F00C0000347050063080701130515005B
:10800800E39AA7FE13050000678000003707010008
:10801800939885001307F7FFB3F8E80093F5F50F79
:10802800B3E5B80093980501B3E8B80037868080B7
:10803800B705FFFE9385F5EF130606081303300016
:108048000327050033C7E800B306B7001347F7FF57
:1080580033F7E6003377C700E31607F89387C7FFBF
:1080680013054500E36EF3FC6FF09FF793070600D6
:108078006FF09FF68327C504130101FF23248100B5
:108088002322910023261100232021011304050037
:1080980093840500638E070213972400B387E700D3
:1080A80003A50700630605040327050023A0E700CE
:1080B80023280500232605008320C100032481000E
:1080C8008324410003290100130101016780000096
:1080D8001306100293054000EF5000642326A40401
:1080E80093070500E31A05FA130500006FF0DFFC9B
:1080F80013091000331999001306590013162600A6
:108108009305100013050400EF500061E30E05FC11
:1081180023229500232425016FF09FF9638005022F
:1081280003A745008327C50413172700B387E70073
:1081380003A7070023A0E50023A0B700678000007D
:10814800130101FD37080100232481022322910233
:10815800232021039384050003A4050113090500C6
:1081680023261102232E31019385450113050000B2
:108178001308F8FF83A7050093854500130515002C
:1081880033F707013307C70293D70701B387C7023D
:10819800B306D70093D8060133F70601B386170153
:1081A800939706013387E70023AEE5FE93D60601D1
:1081B800E34285FC6382060283A78400635EF402BF
:1081C8009307440093972700B387F40023A2D700AE
:1081D8001304140023A884008320C102032481020D
:1081E8001385040003290102832441028329C10164
:1081F800130101036780000083A5440013050900EB
:108208002326D10093851500EFF0DFE603A60401CD
:10821800930905009385C400130626001305C500BD
:1082280013162600EF50D06C03A744008327C90417
:108238008326C10013172700B387E70003A70700A9
:1082480023A0E40023A09700930744009384090027
:1082580093972700B387F40023A2D70013041400D0
:1082680023A884006FF05FF7130101FE232C81001F
:10827800232A9100232821012326310123244101A7
:10828800138906009307900093868600232E110019
:10829800232251019309050013840500130A0600DF
:1082A80093040700B3C6F60263D2270D93071000A4
:1082B800930500009397170093851500E3CCD7FE2C
:1082C80013850900EFF01FDB930710002328F50042
:1082D800232A95009307900063D44709930A9400D2
:1082E80093840A00330444019384140083C6F4FF82
:1082F800930505001306A000938606FD1385090063
:10830800EFF01FE4E31294FE13048AFF33848A001B
:1083180063562A03B3044941B304940013041400B8
:108328008346F4FF930505001306A000938606FD17
:1083380013850900EFF0DFE0E39284FE8320C1019A
:108348000324810183244101032901018329C100F8
:10835800032A8100832A410013010102678000007B
:108368001304A400130A90006FF09FFA930500000D
:108378006FF01FF53707FFFF3377E5009307050018
:108388001305000063160700939707011305000102
:10839800370700FF33F7E70063160700130585006A
:1083A80093978700370700F033F7E7006316070055
:1083B8001305450093974700370700C033F7E700D8
:1083C80063160700130525009397270063C8070065
:1083D8001397170013051500635407006780000002
:1083E80013050002678000008327050013F7770054
:1083F8006306070293F6170013070000639C060044
:1084080013F727006304070893D717002320F50004
:1084180013071000130507006780000093960701F3
:1084280093D60601130700006396060093D7070149
:108438001307000193F6F70F6396060013078700EA
:1084480093D7870093F6F700639606001307470053
:1084580093D7470093F63700639606001307270063
:1084680093D7270093F617006398060093D7170051
:1084780013071700638807002320F500130507007A
:1084880067800000130700026FF0DFF893D727001A
:10849800130720002320F50013050700678000005C
:1084A800130101FF232481001384050093051000A4
:1084B80023261100EFF01FBC232A85008320C1006A
:1084C80003248100130710002328E500130101018C
:1084D80067800000130101FE232631012324410196
:1084E80083A90501032A0601232A910023282101D3
:1084F800232E1100232C8100938405001309060004
:1085080063CC490113070A0013890500138A09007F
:1085180093040600930907008327890083254900EF
:1085280033043A01B3A78700B385F500EFF09FB491
:10853800130E45011313240033036E0093070E0036
:1085480063786E0023A0070093874700E3EC67FE7B
:1085580093854401939E29001306490193182A0024
:1085680037080100B38ED501B30816011308F8FFC8
:1085780063EED5016F00C01093DF0F0163960F08FB
:1085880093854500130E4E0063FCD50F83AF05009D
:10859800B3F30F01E38203FE930F0E00930206006C
:1085A8009304000003A7020003AF0F00938F4F004E
:1085B800B3760701B38676029357070133770F0125
:1085C800135F0F0193824200B3877702B386E600F8
:1085D800B386960013D70601B3F60601B387E70101
:1085E800B387E70013970701B366D70023AEDFFE12
:1085F80093D40701E3E812FB23A09F0083AF050093
:1086080093DF0F01E38E0FF603270E00130F0E0002
:1086180093060600930307009302000083A7060051
:1086280013D9030133770701B3F70701B387F703BA
:10863800130F4F009386460083230F00B3F4030102
:10864800B3872701B38757009392070133E7E20006
:10865800232EEFFE03D7E6FF93D707013307F7036F
:10866800330797003307F70093520701E3E816FB37
:108678002320EF0093854500130E4E00E3E8D5F163
:10868800635480028327C3FF1303C3FF6388070073
:108698006F00800183270300639807001304F4FF29
:1086A8001303C3FFE31804FE232885008320C101B8
:1086B8000324810183244101032901018329C10085
:1086C800032A81001301010267800000130101FEE3
:1086D800232C81002326310123244101232E11005C
:1086E800232A9100232821019377360013040600DA
:1086F80093090500138A05006394070C135424405A
:1087080013090A006308040683A48904638E040C11
:108718009377140013090A00639007021354144056
:10872800630A040403A5040063080506930405000E
:1087380093771400E38407FE138604009305090069
:1087480013850900EFF01FD96308090603274900BC
:1087580083A7C9041354144013172700B387E700ED
:1087680003A707002320E90023A027011309050018
:10877800E31A04FA8320C1010324810113050900C7
:1087880083244101032901018329C100032A8100AF
:10879800130101026780000013860400938504001A
:1087A80013850900EFF01FD323A0A40023200500A0
:1087B800930405006FF0DFF7130905006FF01FF64B
:1087C8009387F7FF37570180130707AA9397270066
:1087D800B307F70003A6070093060000EFF05F96C3
:1087E800130A05006FF09FF1930510001385090027
:1087F800EFF05F8893071027232AF50093071000EE
:108808002328F50023A4A9049304050023200500C8
:108818006FF01FF0130101FE2324410103AA050193
:10882800232A910083A7850093545640338A440134
:10883800232C8100232821012326310123225101E1
:10884800232E110013041A0093890500130906004A
:10885800930A050083A5450063D8870093971700FE
:1088680093851500E3CC87FE13850A00EFF09F80FF
:108878001307450163549002938454009394240091
:10888800B3069500930707009387470023AE07FEBA
:10889800E39CF6FE9384C4FE3307970003A80901FE
:1088A800938749011376F9011318280033880701C3
:1088B8006302060893080002B388C84093050000C5
:1088C80083A607001307470093874700B396C6009F
:1088D800B3E6B600232ED7FE83A6C7FFB3D516018D
:1088E800E3E007FF2320B70063840500130A0400B0
:1088F80003A7490083A7CA048320C10113172700CF
:10890800B387E70003A70700232845010324810153
:1089180023A0E90023A03701832441010329010191
:108928008329C100032A8100832A4100130101021F
:10893800678000009387470083A6C7FF1307470097
:10894800232ED7FEE3F607FB9387470083A6C7FFCE
:1089580013074700232ED7FEE3EE07FD6FF05FF9FC
:108968001306050083A70501032505013305F54016
:10897800631E0502139727001306460193854501D8
:10898800B307E600B385E5006F0080006370F60268
:108998009387C7FF9385C5FF83A6070003A7050034
:1089A800E386E6FE1305F0FF63F4E6006780000047
:1089B8001305100067800000130101FE2328210120
:1089C8000327060103A90501232C8100232A91000E
:1089D8002326310123244101232E11003309E940C4
:1089E80093890500130A0600138445019304460180
:1089F8006318090413172700B307E4003387E4005A
:108A08006F0080006372F4169387C7FF1307C7FFD0
:108A180083A5070083260700E386D5FE63F6D50203
:108A280013070400938709001384040093090A00BC
:108A380093040700138A0700130910006F00C00091
:108A4800E34009FE1309000083A54900EFF08FE217
:108A580003A30901832E0A0137060100131E230010
:108A6800939E2E0023262501330EC401B38ED40114
:108A780013084501930700001306F6FF6F008000F6
:108A8800138808000327040083A5040093084800FE
:108A9800B376C700B386F600B3F7C500B386F640D1
:108AA80093D5050193570701B387B74013D70641FC
:108AB800B387E70013970701B3F6C600B366D7007C
:108AC8009384440023AED8FE1304440093D707418F
:108AD800E3E8D4FB637EC405B70E010013880800E1
:108AE80093050400938EFEFF03A7050013084800B2
:108AF800938545003376D7013306F6009356064131
:108B080093570701B387D700939607013376D601A9
:108B1800B3E6C600232ED8FE93D70741E3E6C5FD8A
:108B28001308FEFF330888401378C8FF338808010C
:108B3800639A06001308C8FF832708001303F3FF8E
:108B4800E38A07FE8320C1010324810123286500ED
:108B580083244101032901018329C100032A8100DB
:108B6800130101026780000093050000EFF08FD029
:108B78008320C10103248101930710002328F500F5
:108B8800232A050083244101032901018329C10007
:108B9800032A81001301010267800000B707F07FF4
:108BA800B3F5B700B707C0FCB385F5006358B0004C
:108BB800930700001385070067800000B305B040E5
:108BC80093D545419307300163C8B700B70708003C
:108BD800B3D5B7406FF0DFFD1387C5FE9306E001FC
:108BE8009305000093071000E3C6E6FCB707008072
:108BF800B3D7E7001385070067800000130101FE63
:108C0800232C810003240501232A910093044501A4
:108C18001314240033848400232821010329C4FF6A
:108C2800232631012324410113050900138A050075
:108C3800232E1100EFF00FF413070002B307A7402B
:108C48002320FA009307A0009309C4FF63D0A70864
:108C5800130555FF63F03405832784FF630005047B
:108C68003306A74033D7C700B316A900B3E6E6001A
:108C7800930584FF3707F03FB3E6E600B397A700F4
:108C880063F2B402032744FF3357C700B3E7E70092
:108C98006F00400193070000631405063707F03F93
:108CA800B366E9008320C1010324810183244101C3
:108CB800032901018329C100032A810013850700C4
:108CC8009385060013010102678000001306B000B7
:108CD8003306A6403357C900B706F03FB366D7003E
:108CE8001307000063F63401032784FF3357C700D6
:108CF800130555013315A900B367E5006FF09FFA16
:108D08003315A9003707F03FB366E5009307000065
:108D18006FF05FF9130101FD232A5101938A0500C1
:108D2800930510002324810223229102232021038A
:108D380093040600232E3101232C4101232611021E
:108D4800138A060093090700EFF0CFB23706100028
:108D580013D444019307F6FF1374F47F1309050035
:108D6800B3F7970063040400B3E7C7002326F100B4
:108D7800638E0A081305810023245101EFF0CFE622
:108D8800930705000327C1006310050683268100A9
:108D9800232AD900B334E00093841400232CE9007B
:108DA80023289900630604081304D4BC3304F40090
:108DB8001307500323208A00B307F74023A0F900C4
:108DC8008320C10203248102130509008324410280
:108DD800032901028329C101032A8101832A410150
:108DE8001301010367800000930600020326810037
:108DF800B386A640B316D700B3E6C6003357A7001C
:108E0800232AD9002326E1006FF0DFF81305C100FB
:108E1800EFF08FDD930710002328F9008327C100A6
:108E280093041000232AF90093070502E31E04F6B1
:108E3800139724003307E900032507019387E7BC4C
:108E48002320FA00EFF00FD393945400B384A44086
:108E580023A099006FF0DFF6130101FD2320210301
:108E6800138905009305810023261102232481021A
:108E780023229102232E310193090500EFF01FD818
:108E88009304050013840500130509009305C10028
:108E9800EFF0DFD68327090103A7090183268100A4
:108EA8003307F7408327C10013175700B386F640EE
:108EB800B307D700635EF0029397470133848700B6
:108EC8001306050093860500138504009305040026
:108ED800EF7050088320C1020324810283244102D9
:108EE800032901028329C1011301010367800000DE
:108EF80013974701B385E5406FF09FFC130101FF0D
:108F0800232481002326110023222101232031015B
:108F1800930770011304050063D4A704B777018091
:108F280003A587D083A5C7D0B777018003A907D148
:108F380083A947D11304F4FF130609009386090097
:108F4800EF70D06DE31804FE8320C1000324810074
:108F580003294100832901001301010167800000F2
:108F6800B757018013143500938707AA3384870005
:108F780003250401832544018320C10003248100C3
:108F880003294100832901001301010167800000C2
:108F9800832606019385F5FF93D5554093851500E3
:108FA800930746019396260093952500B386D7002C
:108FB800B305B50063F8D702130705009387470088
:108FC80003A8C7FF13074700232E07FFE3E8D7FED0
:108FD800B387C6409387B7FE93F7C7FF93874700C9
:108FE8003305F5006378B50013054500232E05FE0B
:108FF800E36CB5FE678000000327050113D65540D2
:1090080093064501635AC70293172700B387F600F2
:1090180063FCF60403A5C7FF9387C7FF631A05001F
:1090280063F2F6049387C7FF03A70700E30A07FE66
:10903800130510006780000093172600B387F60019
:10904800E358E6FC93F5F501E38405FC03A6070065
:10905800130510003357B600B315B700E30AB6FA84
:10906800678000006780000013050000678000002B
:10907800130101FF2324810037040080232291007B
:10908800232611001344F4FF93040600232006004E
:109098003377B4003706F07F938705009306050001
:1090A8006350C706B368A700638C080433F6C5008D
:1090B800138805009308000063120602B777018041
:1090C80083A6C7D103A687D1EF7050559306050034
:1090D800138805003377B4009308A0FC1357474161
:1090E800B70710809387F7FF130727C03378F80076
:1090F80033071701B707E03FB367F80023A0E40080
:109108008320C100032481008324410013850600C5
:10911800938507001301010167800000130101F620
:10912800130EC108232AF10837030080B707FFFF91
:10913800938E05001343F3FF2326D10893878720D6
:109148009305810093060E00232E1106232AF100B1
:109158002328E108232C0109232E11092324D101F6
:10916800232CD101232E6100232861002322C10171
:10917800EF00005783278100238007008320C10761
:109188001301010A67800000930E0500130101F620
:1091980003A5811C130E8108232AF10837030080D8
:1091A800B707FFFF1343F3FF2324C1082326D10881
:1091B800938787201386050093060E009305810088
:1091C800232E1106232AF1002328E108232C010964
:1091D800232E11092324D101232CD101232E610030
:1091E800232861002322C101EF00804F83278100DB
:1091F800238007008320C1071301010A678000004C
:10920800130101FF23248100138405008395E500E1
:1092180023261100EF5080116340050283270405BF
:109228008320C100B387A7002328F4040324810006
:1092380013010101678000008357C40037F7FFFF5F
:109248001307F7FFB3F7E7002316F4008320C100E4
:109258000324810013010101678000001305000049
:10926800678000008397C500130101FE232C81004D
:10927800232A91002328210123263101232E1100BE
:1092880013F707101384050093040500130906005B
:10929800938906008395E500631E070237F7FFFFF1
:1092A8001307F7FFB3F7E7002316F400032481013F
:1092B8008320C10193860900130609008329C10090
:1092C80003290101138504008324410113010102CC
:1092D8006F40003E9306200013060000EF40D05A6E
:1092E8008317C4008315E4006FF05FFB130101FFCF
:1092F80023248100138405008395E50023261100AB
:10930800EF4090589307F0FF6304F5028357C400B9
:10931800371700002328A404B3E7E7002316F40056
:109328008320C1000324810013010101678000002C
:109338008357C40037F7FFFF1307F7FFB3F7E700BA
:109348002316F4008320C1000324810013010101C6
:10935800678000008395E5006F4000473367B500DC
:109368009303F0FF1377370063100710B7877F7FE9
:109378009387F7F70326050083A60500B372F60066
:109388003363F600B382F200B3E2620063927210B4
:109398006316D6080326450083A64500B372F60077
:1093A8003363F600B382F200B3E26200639E720C8C
:1093B8006316D6060326850083A68500B372F600D9
:1093C8003363F600B382F200B3E262006398720C72
:1093D8006316D6040326C50083A6C500B372F6003B
:1093E8003363F600B382F200B3E262006392720C58
:1093F8006316D6020326050183A60501B372F6009B
:109408003363F600B382F200B3E26200639C720A2F
:109418001305450193854501E30ED6F4131706019C
:1094280093970601631EF7001357060193D70601A9
:109438003305F7409375F50F6390050267800000C8
:109448001357070193D707013305F7409375F50FB5
:1094580063940500678000001377F70F93F7F70F01
:109468003305F740678000000346050083C6050002
:1094780013051500938515006314D600E31606FE40
:109488003305D640678000001305450093854500E5
:10949800E31CD6FC13050000678000001305850057
:1094A80093858500E312D6FC130500006780000051
:1094B8001305C5009385C500E318D6FA1305000007
:1094C800678000001305050193850501E31ED6F8A2
:1094D8001305000067800000B367B50093F73700F5
:1094E8006392070803A70500B7867F7F9386F6F780
:1094F800B377D700B387D700B3E7E700B3E7D70060
:109508001306F0FF639EC706130605001308F0FF55
:109518001306460093854500232EE6FE03A70500A3
:10952800B377D700B387D700B3E7E700B3E7D7002F
:10953800E38007FF83C7050003C7150083C625001E
:109548002300F600638A0700A300E600630607000D
:109558002301D6006394060067800000A30106007B
:10956800678000009307050003C70500938717006D
:1095780093851500A38FE7FEE31807FE67800000B8
:10958800130605006FF01FFB9377350013070500DE
:10959800639C0704B7867F7F9386F6F79305F0FFF1
:1095A800130747000326C7FFB377D600B387D70052
:1095B800B3E7C700B3E7D700E384B7FE8346C7FF26
:1095C800B307A7400346D7FF0345E7FF63800604B8
:1095D800630A06023335A0003305F5001305E5FFDD
:1095E80067800000E38806FA83470700130717001F
:1095F80093763700E39807FE3307A7401305F7FF74
:10960800678000001385D7FF678000001385C7FFB8
:1096180067800000B3E7A50093F73700639A070651
:10962800930730001307050063E8C70663000606C2
:1096380003C805009306F6FF93851500230007016C
:1096480093071700630808023306C700B306D7005C
:109658006F00400103C7F5FF93871700A38FE7FE4C
:10966800630C0700938515003388F640E394C7FE22
:109678006780000013880600338707016300080627
:1096880093871700A38F07FEE39CE7FE678000001F
:10969800130705006FF09FF93703FFFEB788808036
:1096A8001303F3EF93880808130E300083A6050010
:1096B800B387660013C8F6FFB3F70701B3F71701BE
:1096C800E39807F6130747001306C6FF232ED7FEB5
:1096D80093854500E36CCEFC6FF05FF56780000072
:1096E800130101E12326111E2324811E2326711D47
:1096F800138405002324B100930B0600232AD1000C
:109708002322911E2320211F232E311D232C411D8E
:10971800232A511D2328611D2324811D2322911DE5
:109728002320A11D232EB11B2324A102EFE08FD6F5
:109738008327050013850700232AF102EFF0DFE4F1
:109748008357C4002326A1022328010E232A010ED1
:10975800232C010E232E010E93F7070863880700B8
:1097680083270401639407006F1000709307C110EA
:10977800938C0B00938807002322F10E03C70C007B
:10978800B7570180938787BC2326F1002326010E53
:10979800B75701802324010E232E0100232801023C
:1097A800232C01022320010423240104232E010277
:1097B80023220100138C47D4138D0800032A810249
:1097C800630E0738930650026314D7006F100054D5
:1097D80013840C006F00C000638AD70E13040900BD
:1097E8008347140013091400E39807FEB304994152
:1097F800638604368326C10E0327810E23209D012C
:10980800B38696001307170023229D002326D10E46
:109818002324E10E93067000130D8D0063CEE60A33
:109828008327410003471400B38797002322F100E0
:10983800630607321303F0FF93041900034E19005F
:10984800A303010C13040000130900009309A005E9
:10985800130B9000930BA002930D03009384140044
:10986800930A0E0093870AFE63E2F91E0327C100DC
:1098780093972700B387E70083A70700678007004F
:1098880013050A00EFE00FC1832745001385070081
:10989800232EF102EFF05FCF2324A104930A0500E1
:1098A80013050A00EFE00FBF832785002320F1048A
:1098B80063840A006F10005403CE04006FF01FFA8F
:1098C8001369090203CE04006FF05FF9B3049941EC
:1098D800E38204F66FF01FF2832581001306410E20
:1098E80013050A00EF500008631A0502130DC11092
:1098F8006FF01FF3832581001306410E13050A003C
:10990800EF504006E304050483270101638807003C
:109918008325010103258102EFB0CFB7832781009A
:1099280083D7C70093F70704638407006F20805E1E
:109938008320C11E0324811E032541008324411E68
:109948000329011E8329C11D032A811D832A411D64
:10995800032B011D832BC11C032C811C832C411C50
:10996800032D011C832DC11B1301011F67800000FB
:10997800B74701809387077E2328F102937709026E
:1099880013830D00638E070E8327410193877700A9
:1099980093F787FF83AB070083AD470013878700E2
:1099A800232AE1009377190063880700B3E7BB0116
:1099B800638407006F1040429379F9BF9307200032
:1099C800A303010C1307F0FFE30CE30E33E7BB011D
:1099D80013F9F9F7E31C077AE316032E639A076273
:1099E80013FB1900930C011B63040B006F108037E5
:1099F80093090B0063546B00930903000347710C30
:109A0800232801002322010223200102232C010024
:109A180063040764938919006F000064130400004D
:109A280013870AFD938414009317240083CAF4FF54
:109A3800B3878700939717003304F70013870AFD4D
:109A4800E372EBFE93870AFEE3F2F9E263880A10F9
:109A580023065115A303010C93091000130B1000E2
:109A6800930CC1146F00005EB74701809387477F4E
:109A78002328F1029377090213830D00E39607F078
:109A88000327410193770901832B07001307470038
:109A9800232AE100638407006F10402E937709049E
:109AA800639407006F10002D939B0B0193DB0B0150
:109AB800930D00006FF01FEF03CE040013694900F7
:109AC8006FF0DFD99377090213830D00E39C071425
:109AD80083264101137709019387460083AB06006B
:109AE8006312074C13770904631407006F10101CE6
:109AF800939B0B0193DB0B01930D0000232AF100CC
:109B08006F001014832641019377090213874600DA
:109B1800638407006F10402A937709016384070064
:109B28006F10100493770904638407006F10D02521
:109B380013790920631409006F10900283274101EB
:109B4800232AE1000327410083A70700938C040020
:109B58002380E70003C70C00E31607C68327C10E5E
:109B6800E38E07DA03248100032581021306410EE0
:109B780093050400EF40105F8357C4006FF09FDA2D
:109B880003CE04009307C0066314FE006F10C02BB9
:109B9800136909016FF09FCC03CE04009307800678
:109BA8006314FE006F10402B136909046FF01FCB7C
:109BB80003274101B787FFFF93C707832314F10CDD
:109BC80093074700232AF100B74701809387077E50
:109BD80013830D002328F102832B0700930D000047
:109BE8009369290093072000930A80076FF05FDDCF
:109BF8001377890013830D00630407006F10801822
:109C0800832741011305010B2328B10193877700AE
:109C180093F787FF83A5070003A64700938787006C
:109C2800232AF100EFA040300327010B0323010191
:109C38002328E10E0327410B232AE10E0327810B7A
:109C4800232CE10E0327C10B232EE10E1305010F70
:109C580023286100EFD05FFD2326A10C1307200005
:109C6800032301016314E5006F10806713071000D8
:109C78006314E5006F101005130710066394EA00DB
:109C88006F204028130710046394EA006F105053A4
:109C980093F7FAFD1307F0FF2326F1046314E3009A
:109CA8006F105018130770046394E7006F20402763
:109CB800832EC10F232C2105136709108322010F5E
:109CC800032F410F832F810F63D40E006F20400CA8
:109CD800232E010413090700232801000327C104C8
:109CE800930760046314F7006F10502B9307500418
:109CF8006314F7006F2040129309010B9307010DBD
:109D08001307C10C930603001308C10D13062000A6
:109D18009385090013050A00232261042328510AA8
:109D280023225102232AE10B2320E103232CF10BE8
:109D3800232EF101232ED10B232CD101EFC09FBD7F
:109D48008327C10413077004930C0500832E810137
:109D5800832FC101032F01028322410203234104FF
:109D68006384E7006F2080438327810513F717007A
:109D7800630407006F2040180327C10DB3079741FC
:109D8800232EF1008327C10C13077004232CF10044
:109D98008327C1046394E7006F10D00C8327C104A4
:109DA800130760046394E7006F101037832781015D
:109DB8009305100493F6FA0F1387F7FF8327C1045E
:109DC8002326E10C130600006398B7009386F6007B
:109DD80093F6F60F13061000230AD10C63540700FC
:109DE8006F2040329306B002A30AD10C930690006C
:109DF80063C4E6006F2040241308310E13060800E0
:109E08001305A000130330066F00C0001386050079
:109E180013870600B367A7029305F6FF9387070326
:109E2800A30FF6FEB346A702E342E3FE1387060339
:109E38001377F70F9306E6FFA38FE5FE63E40601A9
:109E48006F2000359305610D6F00800003C7060081
:109E58009385150093861600A38FE5FEE39806FF09
:109E68001307510E9307610D3307C7403387E70087
:109E78009306410DB307D740232CF1028327C10174
:109E88008326810313071000338BD7006344F70040
:109E98006F20C0288327C102330BFB00832781056D
:109EA8009349FBFF93D9F94113F9F7BF13690910D7
:109EB800B3793B012322010223200102232C010054
:109EC8008327C105639407006F1010011307D002A0
:109ED800A303E10C13030000938919006F00C01756
:109EE8009377090213830D0093690901639207565A
:109EF800832741019387470003274101930D000001
:109F0800232AF100832B0700930710006FF05FAB43
:109F180083274101A303010C83AC0700938B4700FF
:109F2800E38C0C761307F0FF6394ED006F10004587
:109F380013860D009305000013850C00232AB10138
:109F4800EFE08F852328A100032341016314050056
:109F58006F10D01983270101338B97410347710C88
:109F68009349FBFF93D9F941232A71012328010062
:109F78002322010223200102232C0100B3793B0193
:109F880013030000E31807A86F00000D9377090278
:109F980013830D001369090163960748832741015C
:109FA8009387470003274101930D0000232AF100FE
:109FB800832B07006F00C0481369890003CE040093
:109FC8006FF0DF899377090213830D009369090104
:109FD8006394074A83274101938747000327410178
:109FE800232AF100832B070093DDFB4113870D0023
:109FF8006346072A9307F0FF6304F34AB3E7BB01FC
:10A0080013F9F9F7639C0748630403006F100062B3
:10A0180013030000130B0000930C011B6FF05F9DEE
:10A0280003274101A303010C9309100083270700AC
:10A0380013074700232AE1002306F114130B10002D
:10A04800930CC114232801001303000023220102EA
:10A0580023200102232C010093722900638402004B
:10A0680093892900937B49080327C10E63960B0047
:10A0780033083441E34000138346710C638A0602B7
:10A088008326810E1306710C2320CD0013071700B9
:10A0980013061000938616002322CD002326E10E16
:10A0A8002324D10E13067000130D8D006342D60CC5
:10A0B800638A02028326810E1306810C2320CD00B9
:10A0C8001307270013062000938616002322CD00CD
:10A0D8002326E10E2324D10E13067000130D8D00E4
:10A0E800E342D61E930600086380DB58B30D634134
:10A0F8006340B06993760910639406428327810E02
:10A108003307670123209D019387170023226D01E0
:10A118002326E10E2324F10E93067000130D8D0003
:10A12800E3C4F6041379490063060900330934418E
:10A1380063482007635434011384090083274100CE
:10A14800B38787002322F100631607FA83270101EA
:10A158002324010E638807008325010113050A00E3
:10A16800EFA05FB3130DC110938C04006FF09F9E96
:10A17800832581001306410E13050A002326610476
:10A1880023225104EF40007E631005F80327C10E17
:10A19800130DC1100323C104832241046FF05FF142
:10A1A800930600018327810E63C426016F101040B7
:10A1B800B7560180938D46D3130B0001930B7000A3
:10A1C800832A81006F00C000130909FF63562B051D
:10A1D80013070701938717002320BD0123226D0170
:10A1E8002326E10E2324F10E130D8D00E3DEFBFC84
:10A1F8001306410E93850A0013050A00EF40807686
:10A20800631405F0130909FF0327C10E8327810E84
:10A21800130DC110E34E2BFB33072701938717005B
:10A228002320BD0123222D012326E10E2324F10E34
:10A2380093067000E3D0F6F0832581001306410EE3
:10A2480013050A00EF400072631005EC0327C10EE6
:10A258006FF05FEE9377090213830D00639C07206C
:10A268008327410113770901938747006304070097
:10A278006F10D07613770904631407006F10C01E9F
:10A2880003274101232AF10093090900831B0700D2
:10A2980093DDFB4113870D00E35E07D4B30B7041D8
:10A2A800B3377001B30DB041B38DFD409307D002B1
:10A2B800A303F10C1307F0FF930710006318E3F0F2
:10A2C80013071000638EE71C130720006388E7203C
:10A2D8009306011B6F00800093860C009397DD01A5
:10A2E80013F77B0093DB3B0013070703B3EB7701FE
:10A2F80093DD3D00A38FE6FEB3E7BB01938CF6FF29
:10A30800E39C07FC13F619006304062013060003F8
:10A318006300C7209386E6FF9307011BA38FCCFE3B
:10A32800338BD74013890900938C06006FF04FECEC
:10A338009307B002A303F10C03CE04006FF00FD211
:10A348008327410103CE040003A407009387470035
:10A35800232AF100635404D0330480401369490070
:10A368006FF0CFCF1369090803CE04006FF00FCF49
:10A3780083CA04009387140063947A016F10105FF6
:10A3880013870AFD93840700930D0000636CEBCCE0
:10A398009384140093972D0083CAF4FFB387B70101
:10A3A80093971700B38DE70013870AFDE372EBFE5E
:10A3B8006FF04FCB1369190003CE04006FF00FCA7A
:10A3C8008347710C03CE0400639A07C89307000201
:10A3D800A303F10C6FF08FC89377090213830D0064
:10A3E8006396070683264101137709019387460080
:10A3F80083AB0600630407006F10D05D1377090470
:10A40800631407006F108008939B0B01232AF10047
:10A4180093DB0B01930D00009309090093071000CB
:10A428006FF00FDA832741019387770093F787FF4F
:10A4380083AB070083AD470013878700232AE10019
:10A448009379F9BF930700006FF08FD7930909003C
:10A45800832741019387770093F787FF1387870046
:10A4680083AB070083AD4700232AE1009307100060
:10A478006FF00FD59309090083274101938777006F
:10A4880093F787FF03A7470093868700232AD10005
:10A4980083AB0700930D07006FF09FB59309090080
:10A4A800E39C0D5093079000E3E87751938B0B03DF
:10A4B800A307711B13890900130B1000930CF11AE1
:10A4C8006FF00FD3130710006394E7006F100016A6
:10A4D8001307200093090900E39CE7DE83260103A4
:10A4E800930C011B93F7FB00B387F60083C70700A3
:10A4F8001397CD0193DB4B00938CFCFFB36B770173
:10A5080093DD4D002380FC00B3E7BB01E39C07FC0F
:10A518009307011B338B9741138909006FF04FCDC7
:10A528009306500663D456338326010F9305010A18
:10A538001305010B2328D10A8326410F2322E104A6
:10A548002320010A232AD10A8326810F2322010A04
:10A558002324010A232CD10A8326C10F2326010AAA
:10A56800232ED10AEF6010670327410463120558B0
:10A578008327810EB756018093860681130717003B
:10A588002320DD0093871700930610002322DD00A7
:10A598002326E10E2324F10E13077000130D8D00FE
:10A5A800E344F74E8327C10C0327C10163CAE700C0
:10A5B80093771900639607000327C10E6FF09FB6C3
:10A5C800832741038326C1020327C10E2320FD00F0
:10A5D8008327810E3387E6002322DD009387170047
:10A5E8002326E10E2324F10E93067000130D8D002F
:10A5F800E3CAF6028327C101138BF7FFE35460B364
:10A60800930600018327810EE3D0664B930B00016C
:10A61800930A7000832C81006F00C000130B0BFF9E
:10A62800E3D46B49130707019387170023208D0193
:10A6380023227D012326E10E2324F10E130D8D0024
:10A64800E3DEFAFC1306410E93850C0013050A009D
:10A65800EF404031631A05AA0327C10E8327810EF4
:10A66800130DC1106FF09FFBB30B3441E35070A979
:10A67800130600018326810E6354760B232291046E
:10A6880093070D0093840B00138D0C00938B090026
:10A69800930C0B0093090400930E0001930D7000B6
:10A6A80003248100130B03006F00C000938404FF90
:10A6B80063D89E04130707019386160023A0870119
:10A6C80023A2D7012326E10E2324D10E93878700E6
:10A6D800E3DEDDFC1306410E9305040013050A00B2
:10A6E800EF404028631205A2930E0001938404FFF3
:10A6F8000327C10E8326810E9307C110E3CC9EFA6F
:10A708001384090093890B00938B0400832441046C
:10A7180013030B00138B0C00930C0D00138D070013
:10A72800330777019386160023208D0123227D01AC
:10A738002326E10E2324D10E13067000130D8D007D
:10A74800E356D69A832581001306410E13050A00A5
:10A7580023226104EF4000216318059A0323410472
:10A768000327C10E130DC110B30D6341E354B09913
:10A77800130600018326810E6358B60993070D005E
:10A7880013080001138D0C00930B7000930C0B0041
:10A79800138B090093090400032481006F00C00093
:10A7A800938D0DFF6358B8051307070193861600AC
:10A7B80023A0870123A207012326E10E2324D10E1B
:10A7C80093878700E3DEDBFC1306410E9305040044
:10A7D80013050A00EF4000196318059213080001D9
:10A7E800938D0DFF0327C10E8326810E9307C11099
:10A7F800E34CB8FB1384090093090B00138B0C007E
:10A80800930C0D00138D07003307B70193861600CC
:10A8180023208D012322BD012326E10E2324D10EFE
:10A8280013067000130D8D00E356D68C8325810026
:10A838001306410E13050A00EF40C0126316058C7B
:10A848000327C10E130DC1106FF0DF8A0326810E96
:10A858008327C1019306100023209D01930D170043
:10A86800130B1600930B8D0063D0F640930610006F
:10A878002322DD002326B10F2324610F93067000E5
:10A8880063CA66498327C10203274103130B1B00D0
:10A89800B38DFD0023A0EB0023A2FB002326B10FFC
:10A8A8002324610F93067000938B8B0063C866495D
:10A8B8008326010F8327C10113081B002328D10A0F
:10A8C8008326410F9305010A1305010B232AD10A98
:10A8D8008326810F930A080023200103232CD10A21
:10A8E8008326C10F2320010A2322010A232ED10A1D
:10A8F8009386F7FF232CD1002324010A2326010A7B
:10A90800EF60502D138D8B008326810103280102EF
:10A918006300053893871C00B38DDD0023A0FB007E
:10A9280023A2DB002326B10F2324510F93077000C5
:10A9380063C2577993870B01930A2B00930B0D0081
:10A94800138D0700832681039307410D23A0FB0085
:10A958003387DD0023A2DB002326E10E2324510FD9
:10A968009307700063D057FD832581001306410EBD
:10A9780013050A00EF30107F630405006FE0DFF86D
:10A988000327C10E130DC1106FF0CFF99309090009
:10A998006FF01F93B7570180130600018326810EBD
:10A9A800938D47D36354060D23269104232821054C
:10A9B80093070D0013890D00130D0B00938D0C00E8
:10A9C800130F0001938C090093037000930904008E
:10A9D80023225104130B030083248100130408006D
:10A9E8006F00C000130404FF635C8F0413070701A2
:10A9F8009386160023A0270123A2E7012326E10E50
:10AA08002324D10E93878700E3DED3FC1306410E7F
:10AA18009385040013050A00EF30D0746304050021
:10AA28006FE09FEE130F0001130404FF0327C10E0C
:10AA38008326810E9307C11093037000E3488FFAB1
:10AA48001308040083224104138409008324C104E9
:10AA580093890C00938C0D00930D090003290105BF
:10AA680013030B00130B0D00138D070033070701A9
:10AA7800938616002320BD0123220D012326E10E13
:10AA88002324D10E13067000130D8D006356D6DEF5
:10AA9800832581001306410E13050A00232661044D
:10AAA80023225104EF30106C630405006FE0DFE5EA
:10AAB8000327C10E130DC1100323C10483224104CF
:10AAC8006FF08FDB832581001306410E13050A0002
:10AAD80023226104EF301069630405006FE0DFE2B0
:10AAE8000327C10E130DC110032341046FF08FDF3C
:10AAF8000326C10C6358C05E8327C10183268101E8
:10AB0800138B070063CAF630635660038326810EF1
:10AB18003307670123209D019386160023226D01C8
:10AB28002326E10E2324D10E13067000130D8D0089
:10AB3800E348D6209346FBFF8327810193D6F6414D
:10AB4800337BDB00338B67416348603783278101A0
:10AB580093760940B38AFC006396063C032BC10C2C
:10AB68008327C1016346FB0093761900E380062022
:10AB7800832641038327C102130670002320DD00CA
:10AB88008326810E3307F7002322FD0093861600E3
:10AB98002326E10E2324D10E130D8D00E34CD63C61
:10ABA8008326C101B387DC00338B6641B3875741E5
:10ABB800930B0B0063D46701938B070063567003F4
:10ABC8008327810E3307770123205D0193871700C0
:10ABD80023227D012326E10E2324F10E9306700023
:10ABE800130D8D00E3C6F65A93C7FBFF93D7F741C1
:10ABF800B3FBFB00330B7B41635660D39306000124
:10AC08008327810E63D2666B930B0001930A700051
:10AC1800832C81006F00C000130B0BFF63D66B6998
:10AC2800130707019387170023208D0123227D0135
:10AC38002326E10E2324F10E130D8D00E3DEFAFC2A
:10AC48001306410E93850C0013050A00EF3090514E
:10AC5800630405006FE05FCB0327C10E8327810ED5
:10AC6800130DC1106FF05FFB93751900E39005C0D9
:10AC78002322DD002326B10F2324610F93077000E0
:10AC880063CA6743930A2600130D0D016FF09FCB2B
:10AC9800E35AD0CA9307000163C4D7006F10804CF1
:10ACA800232C8100930C0001930A70001384060082
:10ACB800032D8100130B08006F000001130404FF2B
:10ACC80063D68C76130B1B00938D0D0123A08B018B
:10ACD80023A29B012326B10F2324610F938B8B00A2
:10ACE800E3DE6AFD1306410E93050D0013050A0005
:10ACF800EF305047630405006FE01FC1832DC10E7C
:10AD0800032B810E930BC1106FF05FFB13890C00AE
:10AD18006FE05FB2832581001306410E13050A0018
:10AD2800EF305044630405006FE01FBE832DC10E51
:10AD3800032B810E930BC1106FF0DFB483258100C4
:10AD48001306410E13050A00EF30D04163040500D5
:10AD58006FE09FBB832DC10E032B810E930BC11097
:10AD68006FF01FB593070003A307F11A930CF11AAC
:10AD78006FE01FC893770920E3960702930D000040
:10AD88006FE05FC28327410103A70700938747004D
:10AD9800232AF1008325070003264700832687001E
:10ADA8000327C7002328B10E232AC10E232CD10E56
:10ADB800232EE10E6FE09FE90326410083A70600DA
:10ADC800232AE1009356F64123A0C70023A2D70007
:10ADD800938C04006FE01FD89307000313692900C0
:10ADE8002304F10CA304510D9379F9BF93072000B4
:10ADF8006FE01FBD8327010403CE0400639407009E
:10AE08006FE0DFA583C70700639407006FE01FA505
:10AE1800136909406FE09FA4138B0600E34860CFD5
:10AE28006FF05FD1832581001306410E13050A00D8
:10AE3800EF305033630405006FE01FAD0327C10EE8
:10AE4800130DC1106FF00FFB03CE14001369090234
:10AE5800938414006FE09FA003CE140013690920A7
:10AE6800938414006FE09F9F0325810293050004DB
:10AE7800EF50DFDF8327810023A0A70023A8A700C6
:10AE8800631405006F1080330327810093070004C3
:10AE9800232AF7006FE09F8D93076000138B0D0046
:10AEA80063E2B76DB757018093090B00232A71013C
:10AEB800938C87806FF00F99130600018326810E0B
:10AEC80063566663930D0001930A7000832B81001B
:10AED8006F00C000130B0BFF63DA6D6113070701E6
:10AEE8009386160023208D012322BD012326E10E1F
:10AEF8002324D10E130D8D00E3DEDAFC1306410E78
:10AF080093850B0013050A00EF30D0256304050074
:10AF18006FE09F9F0327C10E8326810E130DC1107A
:10AF28006FF05FFB8327C101832B0102232C910063
:10AF3800B387FC00232221052326810483244102B0
:10AF4800232031032322910393060D00130B700075
:10AF5800930D00010329810403240104832981003E
:10AF6800138D0700638A0B08639A04081304F4FF1F
:10AF7800938BFBFF8327C1033307270123A22601F5
:10AF880023A0F6008327810E2326E10E93868600F0
:10AF9800938717002324F10E634CFB0E034604002D
:10AFA800B3055D41930C060063D4C500938C05007E
:10AFB800635690030326810E3307970123A0560199
:10AFC8001306160023A296012326E10E2324C10EA0
:10AFD8006344CB2E034604009386860093C5FCFF8A
:10AFE80093D5F541B3F7BC00B30CF640634C900120
:10AFF800B38ACA00E39A0BF6638E04629384F4FF63
:10B008006FF05FF70326810E63C89D016F0080050E
:10B01800938C0CFF63D89D051307070113061600D0
:10B0280023A0860123A2B6012326E10E2324C10E04
:10B0380093868600E35ECBFC1306410E93850900D8
:10B0480013050A00EF301012630405006FE0DF8B70
:10B05800938C0CFF0327C10E0326810E9306C110A3
:10B06800E3CC9DFB330797011306160023A0860146
:10B0780023A296012326E10E2324C10E6348CB6642
:10B088000346040093868600B38ACA006FF09FF6D1
:10B098001306410E9385090013050A00EF30900C42
:10B0A800630405006FE05F860327C10E9306C11095
:10B0B8006FF0DFEE832581001306410E13050A00A9
:10B0C800EF30500A630405006FE01F840326810EE9
:10B0D800832DC10E130D4111930A1600930BC11055
:10B0E8006FF05F868326810EB755018093850581B1
:10B0F8002320BD0013071700930510009386160040
:10B108002322BD002326E10E2324D10E93057000CF
:10B11800130D8D0063CED506631A06268327C10159
:10B1280093761900B3E6F600639406006FE09FFF7C
:10B13800832641038327C102130670002320DD0004
:10B148008326810E3307F7002322FD00938616001D
:10B158002326E10E2324D10E93088D00634CD64894
:10B168008327C1019386160023A098013387E7003F
:10B1780023A2F8002326E10E2324D10E93077000A2
:10B18800138D880063C4D7006FE0DFF96FF0CFFD3F
:10B19800832581001306410E13050A00EF30807CD9
:10B1A800630405006FE04FF60326C10C0327C10EA8
:10B1B800130DC1106FF05FF6930C011B930700008D
:10B1C80013F9094023289100232C3101130BF00FA8
:10B1D80093890C0023206102930C0A008324010444
:10B1E800138A0D00930D0D00130D0400138407003E
:10B1F8006F0040021306A0009306000013850B00A1
:10B2080093050A00EF40D05063080A54930B0500D9
:10B21800138A05001306A0009306000013850B008F
:10B2280093050A00EF50001213050503A38FA9FE2A
:10B23800130414009389F9FFE30E09FA83C6040086
:10B24800E31AD4FAE30864FB63180A4C93079000E6
:10B2580063E4774D138A0C00938C090083298101DC
:10B268009307011B232E81002320910413040D0052
:10B278000323010283240101138D0D00338B9741B1
:10B28800138909006FE0CFF6832581001306410E6C
:10B2980013050A00EF30006D630405006FE0CFE688
:10B2A800130DC1106FF00FB03307670193871700B4
:10B2B80023208D016FE09FE51306410E9385090059
:10B2C80013050A00EF30006A630405006FE0CFE35E
:10B2D800034604000327C10E9306C1106FF01FD068
:10B2E8008327010F9305010A1305010B2328F10A8F
:10B2F8008327410F2320010A2322010A232AF10A66
:10B308008327810F2324010A2326010A232CF10A0B
:10B318008327C10F232EF10AEF60C02C6344054434
:10B328000347710C9307700463D65721B747018010
:10B33800938C477D23280100232201022320010248
:10B34800232C01001379F9F793093000130B30000F
:10B3580013030000630407006FE0CFEB6FE0DFCF5B
:10B3680083274101938C040083A70700232AE10067
:10B378000327410023A0E7006FE0CFFD13850C00F1
:10B38800EFE08FA0130B05006FE05FBD832641033C
:10B398008327C102930570002320DD008326810ED8
:10B3A8003307F7002322FD00938616002326E10EBB
:10B3B8002324D10E93088D0063CED522E35206DAFA
:10B3C800930500FF330BC040E352B62E930B0001E8
:10B3D800930A7000032D81006F00C000130B0BFF50
:10B3E800E3D66B2D130707019386160023A0880167
:10B3F80023A278012326E10E2324D10E9388880006
:10B40800E3DEDAFC1306410E93050D0013050A006E
:10B41800EF304055630405006FE00FCF0327C10EDE
:10B428008326810E9308C1106FF05FFB930604001A
:10B4380003248101930A1B0093878B00B38DDD00E1
:10B4480023A2DB0023A08B012326B10F2324510F55
:10B4580093067000E3C056C7938A1A00138D8700BD
:10B46800938B07006FF00FCE13770920630207163E
:10B478000327410193090900232AF100830B0700E0
:10B4880093DDFB4113870D006FE09FB6137709200A
:10B4980063060712232AF10093FBFB0F930D0000AC
:10B4A80093090900930710006FE08FD113770920E3
:10B4B8006300071093FBFB0F930D0000232AF10094
:10B4C8006FE01FF88327C10F63D207129307D002DA
:10B4D800A303F10C1307D0029307700463D4574BEE
:10B4E800B7470180938CC77D6FF0DFE433076701AE
:10B4F8009386160023208D0123226D012326E10E59
:10B508002324D10E13067000130D8D006350D6E46A
:10B51800832581001306410E13050A00EF3080448D
:10B52800630405006FE04FBE0327C10E130DC11061
:10B538006FF0CFE1B7470180938C077D6FF09FDFF5
:10B54800832581001306410E13050A00EF30804160
:10B55800630405006FE04FBB0327C10E130DC11034
:10B568006FF04FDD130B60006FF0DF938326C1018E
:10B57800B387DC00338B6641B38B574163567BE757
:10B58800930B0B006FF04FE683274101232AE1005C
:10B598000327410083A70700938C04002390E7004A
:10B5A8006FE04FDB93FBFB0F930D00006FE08FBF45
:10B5B800930D0000232AF1006FE09FE8232AF10091
:10B5C800930D000093090900930710006FE04FBF27
:10B5D8000327410193090900232AF100832B07005F
:10B5E80093DDFB4113870D006FE09FA00347710CAB
:10B5F8006FF09FEE832581001306410E13050A00A4
:10B60800EF304036630405006FE00FB00326C10C2D
:10B618000327C10E8326810E9308C110E35206B496
:10B628006FF01FDA130360006FE08FE893090900D9
:10B638006FE0DFE7832C41028327C10123208104C7
:10B64800138D0600B386FC0083248101032941047D
:10B658000324C1048329010263F256D1938A0600A8
:10B668006FF0CFCF832781011307D0FF63C4E700B2
:10B67800635AF300938AEAFF93F7FAFD2326F1044D
:10B688006FE0CFF20327C1018327810163C4E72C50
:10B6980003278105138B070013771700630607003C
:10B6A8000327C102338BE7008327810513F707407F
:10B6B8006306070083278101E348F01A9349FBFFDB
:10B6C80093D9F941B3793B01930A70062322010209
:10B6D800232001026FE0CFFE0347710C1303000023
:10B6E800630407006FE00FB36FE01F971306410E66
:10B6F8009385090013050A00EF30C026630405008E
:10B708006FE08FA0034604000327C10E9306C11003
:10B71800B38ACA006FF01F8E832781048325C10373
:10B7280013040000B389F940138607001385090044
:10B73800EFD05FEE03C814001306A00093060000C4
:10B748003338000113850B0093050A00B384040104
:10B75800EF40007C6FF09FAB93079000E3E877AB76
:10B768006FF05FAF9307D002A303F10C1307D00269
:10B778006FF05FBB832581001306410E13050A0095
:10B78800EF30401E630405006FE00F98032BC10CD7
:10B798000327C10E130DC1106FF08FC09309010B61
:10B7A800930603001307C10C1308C10D9307010D7D
:10B7B800130630009385090013050A00232261044B
:10B7C8002328510A23225102232AE10B2320E103D3
:10B7D800232CF10B232EF101232ED10B232CD10185
:10B7E800EFB04F938346050013070003930C050041
:10B7F800832E8101832FC101032F0102832241027D
:10B8080003234104930B010A638CE6060327C10C4A
:10B81800330B6700338B6C0193850B00138509008C
:10B82800232C61002328510A232AE10B232CF10B36
:10B83800232ED10B2320010A2322010A2324010AE3
:10B848002326010AEF50103913070B000323810147
:10B85800631405006FE08FD20327C10D13060003A0
:10B86800636467016FE08FD193071700232EF10CF3
:10B878002300C7000327C10DE36867FF6FE00FD0FF
:10B88800930B010A93850B00138509002322610499
:10B898002328510A23225102232AE10B2320E10302
:10B8A800232CF10B232EF101232ED10B232CD101B4
:10B8B8002320010A2322010A2324010A2326010A3C
:10B8C800EF505031832E8101832FC101032F0102D4
:10B8D8008322410203234104E30A05F213071000FF
:10B8E800330767402326E10C6FF09FF20347710C82
:10B8F800232A71012322010223200102232C0100A3
:10B9080093090300130B03001303000063040700EB
:10B918006FE04F906FE04FF48327810513F717000E
:10B928008327810133676700E354F0006312077CC3
:10B93800032B8101930A60068327810513F70740CB
:10B94800631607729349FBFF93D9F941B3793B0119
:10B958006FF0DFD78327C1010327C102930A70065E
:10B96800338BE70083278101E348F0FC330BFB406E
:10B97800130B1B009349FBFF93D9F941B3793B01A2
:10B988006FF0DFD4B7470180938C877D6FF09F9A63
:10B99800832581001306410E13050A00EF20907CD1
:10B9A800630405006FD05FF6032BC10C8327C10128
:10B9B8000327C10E130DC110338B67416FF0CFA25F
:10B9C800930700032304F10C93078005A304F10CEB
:10B9D8009367290013073006232CF104232801005C
:10B9E800930CC1146342674A832EC10F93F7FAFD83
:10B9F8002326F104232E0104136929108322010F41
:10BA0800032F410F832F810F63C80E3813071006C9
:10BA18006380EA52130710046384EA006FE00FACF6
:10BA28009309010B13850900232A61042328510A6D
:10BA3800232AE10B232CF10B232ED10BEF80806FEF
:10BA48001306C10CEFD0CFE213860500930505005D
:10BA580013850900EF80404D0327010B9307010967
:10BA6800930B010A2328E1080327410B1306010859
:10BA780093850700232AE1080327810B13850B0010
:10BA8800232EF100232CE1080327C10B2328C1042E
:10BA980023200108232EE1083707FC3F2326E1086D
:10BAA8002322010823240108EF5010488327010AA4
:10BAB8000328410A832E810A032FC10A93850B00AC
:10BAC800138509002328F10A2322F104232A010BF4
:10BAD80023220103232CD10B2320D103232EE10B96
:10BAE800232CE1012320010A2322010A2324010A2D
:10BAF8002326010AEF50100E032F8101832E010225
:10BB080003284102832741040323410563160500E6
:10BB1800130710002326E10C374701801307477FDE
:10BB28002322E104130BF3FF232C91012320910618
:10BB380023225107232AA107232C4107232E9107EB
:10BB4800232421072326810623286106930C0B0052
:10BB5800138D0700930D0800138A0E00930A0F0037
:10BB68008324C1016F00400593850B0013850900EC
:10BB78002322C1022320F103232E5100232A510A34
:10BB8800232CF10B232EC10A2328210B2320010A81
:10BB98002322010A2324010A2326010AEF509003D5
:10BBA800938CFCFF8322C101832F010203264102EB
:10BBB8006304050E232C6101B707034013860400B4
:10BBC80093850B0013850900232EF1082320A10B70
:10BBD8002322B10B2324410B2326510B23280108D0
:10BBE800232A0108232C0108EF501034138509007B
:10BBF800EF8000069305050013040500138509006E
:10BC0800032BC10B832A010B032A410B0329810B48
:10BC1800EF8000198327010B032601059385040093
:10BC28002320F1088327410B13850B00232E61097C
:10BC38002322F1088327810B23285109232A41094C
:10BC48002324F1088327C10B232C21092326F1087B
:10BC5800EF60102E83274104032781010329010A7D
:10BC6800B387870083C707008322410A832F810A8D
:10BC78000326C10A130B1700A30FFBFE232A910505
:10BC88009307F0FF130D0900938D0200138A0F002C
:10BC9800930A0600E39AFCEC0323010793030900C7
:10BCA800B706FE3F93850B00138509002320610228
:10BCB800232E810083240106832A41062328710A42
:10BCC80023227106232A510A23205106232CF10B23
:10BCD8002328F105232EC10A2322C1022320010AA9
:10BCE8002322010A2324010A2326D10AEF50407B8C
:10BCF800032D41070324C106930D0B00032A810776
:10BD0800832CC10703298106032301026346A00A85
:10BD18008323410683220106832F0105032641025E
:10BD2800B706FE3F93850B00138509002328710A87
:10BD3800232A510A232CF10B232EC10A2320010A9E
:10BD48002322010A2324010A2326D10AEF508068FE
:10BD580003230102631805008327C10113FB1700A1
:10BD6800631C0B0483274105130600039386170001
:10BD7800B386DD0063C80700938D1D00A38FCDFE39
:10BD8800E39CB6FFB3879D41232EF1006FD09FFF40
:10BD98002328010013090700370700809307D00202
:10BDA800B34ED701232EF1046FF05FC6B75601805A
:10BDB800938D46D36FE04FC68327810193860D008C
:10BDC800232EF10C8327410403C6FDFF83C5F7002A
:10BDD8006310B60213050003A38FA6FE8326C10DC8
:10BDE8009387F6FF232EF10C03C6F6FFE386C5FE04
:10BDF800930516001305900393F5F50F6306A60047
:10BE0800A38FB6FE6FF01FF88327410483C5A700F0
:10BE1800A38FB6FE6FF01FF7130B13009309010BE6
:10BE28001308C10D9307010D1307C10C93060B00EE
:10BE3800130620009385090013050A0023226104D4
:10BE48002328510A23225102232AE10B2320E1034C
:10BE5800232CF10B232EF101232ED10B232CD101FE
:10BE6800EFA05FAB832E8101832FC101032F010255
:10BE78008322410203234104930C0500338B6C0198
:10BE8800930B010A6FF05F999305130013050A00DD
:10BE980023286100EF409FDD930C05000323010177
:10BEA800630205302328A1006FF01FB43307670130
:10BEB8009386160023A0880123A268012326E10E99
:10BEC8002324D10E1306700093888800635AD6A8DD
:10BED800832581001306410E13050A00EF209028E0
:10BEE800630405006FD05FA20327C10E8326810E6D
:10BEF8009308C1106FF0CFA6338B6C00930B010A27
:10BF08006FF09F91930700032304F10C93078007B8
:10BF18006FF0DFAB9307F0FF2322F1006FD05FA132
:10BF2800630403006FD0DFD8130310006FD05FD80D
:10BF38009309010B13850900232A61042328510A58
:10BF4800232AE10B232CF10B232ED10BEF80801E2B
:10BF58001306C10CEFD0CF91138605009305050099
:10BF680013850900EF70507C0327010B9307010923
:10BF7800930B010A2328E1080327410B1306010844
:10BF880093850700232AE1080327810B13850B00FB
:10BF9800232EF100232CE1080327C10B2328C10419
:10BFA80023200108232EE1083707FC3F2326E10858
:10BFB8002322010823240108EF5000778327010A70
:10BFC8000328410A832E810A032FC10A93850B0097
:10BFD800138509002328F10A2322F104232A010BDF
:10BFE80023220103232CD10B2320D103232EE10B81
:10BFF800232CE1012320010A2322010A2324010A18
:10C008002326010AEF50003D032F8101832E0102F0
:10C0180003284102832741040323410563160500D1
:10C02800130710002326E10C374701801307077E0A
:10C038002322E1046FF01FAF9306610D6318060019
:10C0480093060003230BD10C9306710D9307011B74
:10C058003386F640130707039307D60D2380E600BF
:10C06800232CF1026FD09FE1930A70068325010407
:10C07800832781012322010203C70500232001022F
:10C088001306F00F630EC702635CF70283C6150040
:10C09800B387E740638E06000327010293851500E6
:10C0A800130717002320E102138706006FF09FFD96
:10C0B80083264102938616002322D1026FF09FFC4B
:10C0C800232CF10003274102832701022320B10416
:10C0D8003387E700832781043307F702330B6701AF
:10C0E8009349FBFF93D9F941B3793B016FD05FDDE9
:10C0F8000327C102930A6006338BE700330B6B00FA
:10C108006FF09F8383278101130710009306D002E5
:10C118003307F740A30AD10C6FD05FCD8327810581
:10C1280013F71700631407006FD05FD76FD09FD63F
:10C13800631A070093091000930A6006130B100096
:10C148006FF0CFD88327C102930A6006138B1700BC
:10C15800330B6B009349FBFF93D9F941B3793B014A
:10C168006FF0CFD693070D006FF04FAD0327410155
:10C17800832D07001307470063D40D00930DF0FFCC
:10C1880003CE1400232AE100938407006FD00FED3B
:10C1980093072000232CF1026FD05FCE130B03000E
:10C1A8006FF0DFCD8326810083D7C60013E707042D
:10C1B800930707002396E6006FD0CFF60327810286
:10C1C8009307C0002320F7009307F0FF2322F10014
:10C1D8006FD00FF6930909006FD01FD29309090099
:10C1E8006FD0DFDF83A74506130101FD2328610116
:10C1F80023261102232481022322910223202103D2
:10C20800232E3101232C4101232A510123267101B8
:10C218002324810113972701130B06006358070A8B
:10C228008327860013890500130A0500832B06005F
:10C23800930AF0FF6388070803AC4B0003A40B00C4
:10C2480093592C0063860906930400006F00C00010
:10C2580013044400638C9904832504001306090021
:10C2680013050A00EF10900093841400E31255FFA1
:10C278001305F0FF8320C1020324810223240B004D
:10C2880023220B0083244102032901028329C101CF
:10C29800032A8101832A4101032B0101832BC10059
:10C2A800032C8100130101036780000083278B00A2
:10C2B800137CCCFFB38787412324FB00938B8B002F
:10C2C800E39C07F6130500006FF0DFFAEF10100B80
:10C2D8006FF05FFA03278600630407006FF09FF092
:10C2E800232206001305000067800000130101EDFA
:10C2F800232E3111232C41112324811123261112BD
:10C30800232481122322911223202113232A51113D
:10C318002328611123267111232291112320A111B1
:10C32800232EB10F2328D100130A05009389050095
:10C33800130C06006306050083278503E384071AA8
:10C348000397C9009317070193D70701939627010D
:10C3580063C6060283A64906B7270000B367F7003D
:10C3680037E7FFFF1307F7FF33F7E6002396F900D7
:10C378009397070123A2E90693D7070113F78700CC
:10C388006302071803A70901630E071693F7A701AD
:10C398001307A000638AE718B7570180938747D52A
:10C3A800375B01809304C104232AF10037590180C7
:10C3B80093070BEC930B0C00232091042324010416
:10C3C80023220104232C0100232E01002322010231
:10C3D80023200102232601002322F100130909ED7D
:10C3E800138C040083C70B006388071613075002D9
:10C3F800E38AE75A13840B006F00C0006388E714D0
:10C4080013840C0083471400930C1400E39807FE70
:10C41800338D7C4163020D14032781048327410473
:10C4280023207C013307ED00938717002322AC01FA
:10C438002324E1042322F10493067000130C8C00DA
:10C4480063D0F602E30C0750130601049385090034
:10C4580013050A00EFF01FD9631C0510138C0400A4
:10C468000327C100834714003307A7012326E100EF
:10C478006384070E938B1C0003C71C00A30D0102E5
:10C48800930AF0FF13040000130B0000930CA0059F
:10C49800130D90001306A002938B1B00930707FE51
:10C4A80063E4FC1E8326410193972700B387D700D6
:10C4B80083A707006780070013050A00EFB08FFD08
:10C4C80083274500138507002320F102EFD0CF8B87
:10C4D8002322A102930D050013050A00EFB08FFB7C
:10C4E800832785001306A002232EF100E3960D543E
:10C4F80003C70B006FF05FFA136B0B0203C70B0047
:10C508006FF09FF99385090013050A00EF70DFD1DA
:10C51800630405006F10C00383D7C9001307A00088
:10C5280093F7A701E39AE7E68397E900E3C607E6EE
:10C538008326010113060C009385090013050A00E0
:10C54800EF1080072326A1006F008003338D7C4104
:10C55800E3020DF26FF05FEC83278104638A070022
:10C56800130601049385090013050A00EFF09FC71D
:10C5780083D7C90093F70704638407006F00507DD1
:10C588008320C112032481120325C1008324411290
:10C59800032901128329C111032A8111832A411118
:10C5A800032B0111832BC110032C8110832C411004
:10C5B800032D0110832DC10F1301011367800000A3
:10C5C800B74701809387477F232CF10093770B02AD
:10C5D80063880752832701019386770093F686FFC5
:10C5E80083AD060083AE4600938786002328F100BA
:10C5F80093761B0063860600B3E6DD01E3900642EE
:10C60800937CFBBF13072000A30D01029306F0FFE4
:10C618006380DA66B3E6DD0113FBFCF7E398061ED8
:10C6280063940A74E314073493F71C002324F1007D
:10C63800130D010FE396073883278100938C0A00B6
:10C6480063D4FA00938C07008347B103B337F00033
:10C65800B38CFC006F00400513040000930607FD2F
:10C66800938B1B009317240003C7FBFF33848700B9
:10C678001314140033848600930607FDE372DDFE6D
:10C68800930707FEE3F0FCE2E30807EC93071000CA
:10C698002306E108A30D0102930C10002324F100E6
:10C6A800130DC108930A0000937F2B0063840F00C9
:10C6B800938C2C0003274104137F4B0883278104A4
:10C6C800930617001386060063160F00B30D9441F6
:10C6D800E342B0158345B10393068C00638C0502D1
:10C6E8001307B103938717002320EC0013071000EA
:10C6F8002322EC002324F1042322C1041307700031
:10C70800E346C70C13070600138C06001306160031
:10C7180093868600638E0F041307C103938727004F
:10C728002320EC00130720002322EC002324F1042B
:10C738002322C10413077000E350C708E38A0724C3
:10C74800130601049385090013050A002324E10355
:10C75800EFF05FA9E31E05E0032741048327810466
:10C76800032F81029306410513061700138C04005A
:10C77800930500086300BF6683258100B38ABA4029
:10C7880063485073032781002320AC012322C1048E
:10C79800B307F7002322EC002324F10413077000E9
:10C7A8006352C702638807181306010493850900BA
:10C7B80013050A00EFF01FA3E31C05DA83278104A1
:10C7C8009386040013734B0063060300330C9441F3
:10C7D800634E80176354940113840C000327C1002F
:10C7E800330787002326E10063900778232201049A
:10C7F800138C04006FF01FBF93770B02936C0B012F
:10C808006392075483270101138747008327010197
:10C81800930E00002328E10083AD070013071000E2
:10C828006FF09FDE136B0B0803C70B006FF0DFC6BA
:10C8380083270101A30D010203AD0700938D470073
:10C84800E3080D369307F0FFE384FA2213860A0003
:10C858009305000013050D00EFB00FF4E30A054C33
:10C86800B307A5412324F1002328B101930A00004E
:10C878006FF09FDC93770B0213630B01639A0746F3
:10C88800832701011387470083270101930E0000C6
:10C898002328E10083AD07006F00404793770B0220
:10C8A800936C0B01639C074683270101138747009C
:10C8B800832701012328E10083AD070093DEFD41B2
:10C8C80013870E00634207381307F0FF638AEA00F4
:10C8D80033E7DD0113FBFCF7E3080708930C0B00B3
:10C8E800E3940E1C13079000E360B71D93870D03B4
:10C8F800A307F10E93071000138B0C002324F100FB
:10C90800130DF10E6FF05FD303270101A30D010290
:10C91800930C100083270700130747002328E10022
:10C928002306F108930710002324F100130DC10812
:10C938006FF05FD72322010413734B00630C037C51
:10C94800330C94416358807D9386040013070001DB
:10C9580003264104E35A873F130D0001930D70002D
:10C968006F00800193052600938686001306070052
:10C97800130C0CFF635A8D0583254100938707012B
:10C988001307160023A0B60023A2A6012324F1044E
:10C998002322E104E3D8EDFC638607421306010471
:10C9A8009385090013050A00EFF0DF83E31205BC45
:10C9B80003264104130C0CFF83278104938604008B
:10C9C80093051600E34A8DFB03274100B3878701CF
:10C9D80023A2860123A0E6002324F1042322B10424
:10C9E80013077000E358B7DE638607721306010465
:10C9F8009385090013050A00EFF0CFFEE31A05B688
:10CA0800832781046FF01FDD8347B10303C70B0041
:10CA1800E39407A893070002A30DF1026FF0DFA7C4
:10CA28009307B002A30DF10203C70B006FF0DFA656
:10CA38008327010103C70B0003A40700938747005E
:10CA48002328F100E35A04A433048040136B4B00FD
:10CA58006FF09FA4136B1B0003C70B006FF0DFA3DD
:10CA680003C70B0093871B00E300C730930607FD3D
:10CA7800938B0700930A0000E362DDA2938B1B00EF
:10CA880093972A0003C7FBFFB38A5701939A1A00AA
:10CA9800B38ADA00930607FDE372DDFE6FF01FA08C
:10CAA80003C70B00136B4B006FF01F9F93770B02AC
:10CAB800639807288327010193760B0113874700A2
:10CAC80083A70700E394062C93760B04E3820610F1
:10CAD800939D07012328E10093DD0D01930E0000CB
:10CAE800930C0B00130710006FF01FB2B7470180BB
:10CAF8009387077E232CF10093770B02E39C07AC06
:10CB08000326010193760B018327060013064600CE
:10CB18002328C1006398066693760B046380066633
:10CB2800939D070193DD0D01930E00006FF05FAC3C
:10CB3800832701013787FFFF1347078383AD07006A
:10CB4800938747002328F100B74701809387077E22
:10CB5800231EE102930E0000936C2B00232CF1009E
:10CB6800130720006FF05FAA93770B0263900718F2
:10CB78008327010193760B011387470083A70700DA
:10CB8800E39A062093760B04E3840606939D070137
:10CB980093DD0D01930E000013030B002328E10021
:10CBA8006F00C0168326010193770B021387460096
:10CBB8006392076A93770B016390077E93770B0460
:10CBC800E398070E13730B206308037C8327010186
:10CBD8002328E1000327C10083A707002380E7007B
:10CBE8006FF05F8003C70B009307C006630EF778EA
:10CBF800136B0B016FF05F8A03C70B009307800666
:10CC0800630CF776136B0B046FF01F8993770B0295
:10CC1800639407100327010193770B01130747005B
:10CC2800E39E071693770B046382077E832701012F
:10CC38002328E100930C0B00839D070093DEFD4140
:10CC480013870E00E35207C8B307B0413337F0002B
:10CC5800B30ED041B38EEE401307D002A30DE1020C
:10CC68009306F0FF938D070013071000E394DA9AF8
:10CC780093061000E306D7C6930620006300D7107A
:10CC88009306010F6F00800093060D009397DE0155
:10CC980013F77D0093DD3D0013070703B3EDB701DC
:10CCA80093DE3E00A38FE6FEB3E7DD01138DF6FFAA
:10CCB800E39C07FC93F71C00638C070E93070003A3
:10CCC8006308F70E9386E6FFA30FFDFE9307010F97
:10CCD800B387D7402324F100138B0C00138D060073
:10CCE8006FF09F95EF701FE56FF08FE513030B0052
:10CCF8008327010113877700137787FF832D0700A8
:10CD0800832E4700930787002328F100937CF3BF05
:10CD1800130700006FF05F8F930C0B00832701014E
:10CD28009387770093F787FF03A7470093868700C9
:10CD38002328D10083AD0700930E07006FF09FB83A
:10CD4800930C0B008327010113877700137787FF64
:10CD580093078700832D0700832E47002328F100BF
:10CD6800130710006FF05F8A930610006308D77AE4
:10CD780093062000930C0B00E314D7F0832681015F
:10CD8800130D010F93F7FD00B387F60083C7070063
:10CD98001397CE0193DD4D00130DFDFFB36DB70161
:10CDA80093DE4E002300FD00B3E7DD01E39C07FCA2
:10CDB8009307010FB387A7412324F100138B0C00BD
:10CDC8006FF09F87930510001306000093860400F8
:10CDD8006FF01FBAB30D9441E350B09B9305000167
:10CDE80063DEB577930E0001130F70006F008001AA
:10CDF80093052700130C8C0013870600938D0DFFF5
:10CE080063DCBE05938707019306170023202C01D6
:10CE18002322DC012324F1042322D104E35ADFFC7A
:10CE280063800716130601049385090013050A0099
:10CE3800EFF04FBB631E05F203274104930E000178
:10CE4800938D0DFF83278104138C0400930517002D
:10CE5800130F7000E3C8BEFB13058C00B387B7013E
:10CE680023202C012322BC012324F1042322B10412
:10CE780013077000635AB7386380075C1306010410
:10CE88009385090013050A00EFF0CFB5631205EE8C
:10CE9800832581000327410483278104B38ABA408C
:10CEA8009306410513061700138C0400E35C508DAC
:10CEB8009305000163DE555793080001930D700038
:10CEC8006F00800113062700130C8C0013870600DF
:10CED800938A0AFF63DA58059387070193061700B8
:10CEE80023202C0123221C012324F1042322D10412
:10CEF800E3DADDFC63820706130601049385090063
:10CF080013050A00EFF00FAE631405E6032741048A
:10CF180093080001938A0AFF83278104138C040075
:10CF280013061700E3CA58FB93058C00B387570113
:10CF380023202C0123225C012324F1042322C10491
:10CF4800130770006344C71E1306160093868500F6
:10CF5800138C05006FF01F831306100013070000E1
:10CF6800138C04006FF0DFF61306010493850900A3
:10CF780013050A00EFF00FA7E30A05866FF04FDFED
:10CF88009305100013070000138C04006FF01FE7CF
:10CF9800639007240347B103631E074E63880F207D
:10CFA8009307C1032326F104930720002328F104E3
:10CFB800130610009306410513070600138C06009C
:10CFC80013061600938686006FF08FFAE38807FC35
:10CFD800130601049385090013050A002326E103BB
:10CFE8002324F103EFF00FA0631405D803274104AD
:10CFF800832781049306410513061700138C040048
:10D00800032FC102832F81026FF0CFF0930C0B0026
:10D018006FF01FC6130600016354B65393850B00C7
:10D0280013060C00930B0400138C0A0013840D00E4
:10D03800930E0001930270002324F103930A0F005A
:10D04800938D05006F00C001930527001306860025
:10D0580013870600130404FF63DE8E04930617008B
:10D0680083254100938707012322D6012320B60098
:10D078002324F1042322D104E3D8D2FC63840708D3
:10D08800130601049385090013050A00EFF08F9534
:10D09800631005CE03274104930E0001130404FF17
:10D0A80083278104138604009305170093027000F8
:10D0B800E3C68EFA832F810213870D00138F0A00AF
:10D0C800930D0400930A0C0013840B00130C060044
:10D0D800930B070003274100B387B7012322BC0144
:10D0E8002320EC002324F1042322B1041307700049
:10D0F800E340B7EA130C8C0013861500138705006C
:10D108006FF04FDD1307000093051000138604002D
:10D118006FF05FF46354940113840C008327C100FB
:10D12800B38787002326F1006FF04FEC638E071456
:10D13800130601049385090013050A00EFF08F8A8E
:10D14800631805C203264104832781049306410519
:10D1580013061600138C04006FF0CFE2232201049B
:10D16800138C04006FF0CFAF639A0A3A930A000059
:10D1780023240100130D010F6FF00FCC93760B20C1
:10D1880063980638938D0700930E00006FF04FC622
:10D19800930641051306100013070000138C0400C2
:10D1A8006FF00FDD938C0B006FF0CFAC130700000E
:10D1B8009306410513061000138C04006FF04FDB33
:10D1C80093070003A307F10E130DF10E6FF0CFC6FE
:10D1D800130601049385090013050A002326E103B9
:10D1E8002324F103EFF00F80631405B803274104EB
:10D1F80083278104138C040013061700032FC10230
:10D20800832F81026FF00FCD1386150093068500DA
:10D2180013870500130C05006FF00FD69306000363
:10D22800136B2B00A30EE102230ED102937CFBBFEC
:10D23800130720006FF04FBD8327C10103C70B0000
:10D24800638C07A483C70700638807A4136B0B408C
:10D258006FF08FA40326C10083A706002328E100EE
:10D268009356F64123A0C70023A2D7006FF08F97EB
:10D2780013050D00EFC04FB12324A1002328B101ED
:10D28800930A00006FF04FBB83278100130710003B
:10D298002326A1052328F1042324F1042322E104F1
:10D2A800930641056FF00FD293F70C40130D010F51
:10D2B80023248101138C070093870B002324810208
:10D2C80023264103938B0900130B000093090D00DB
:10D2D8000324C101138A0E00138D07006F0040025A
:10D2E8001306A0009306000013850D0093050A009D
:10D2F800EF20104263080A22930D0500138A0500E7
:10D308001306A0009306000013850D0093050A007C
:10D31800EF30400313050503A38FA9FE130B1B0071
:10D328009389F9FFE30E0CFA03470400E31A67FB3D
:10D338009307F00FE306FBFA631A0A1093079000AD
:10D3480063E6B71193070D00138D090093890B004D
:10D35800938B07009307010FB387A741232E810002
:10D36800032C810003248102032AC1022324F10033
:10D37800138B0C006FF04FAC03C71B00136B0B2013
:10D38800938B1B006FF04F9103C71B00136B0B02AD
:10D39800938B1B006FF04F908327010183A7070031
:10D3A8002328E1000327C10023A0E7006FF08F8343
:10D3B800232451019307600063EA570D375E01800B
:10D3C800832C81002328B101130D8E806FF08FAD5F
:10D3D80093760B20638206122328E10093FDF70F52
:10D3E800930E0000930C0B00130710006FF0CFA1F1
:10D3F80093760B206388060E93FDF70F930E0000BB
:10D4080013030B002328E1006FF05F9093770B2044
:10D41800638C070A83270101930C0B002328E10082
:10D42800838D070093DEFD4113870E006FF08FC9CF
:10D43800938506006FF09FAF930641051306100011
:10D4480013070000138C04006FF00FB38327410209
:10D4580083250102130B0000B389F94013860700E6
:10D4680013850900EFC00F9B034714001306A000A3
:10D47800930600003337E00013850D0093050A007A
:10D488003304E400EF20D0286FF01FE72324F100D5
:10D498006FF0DFF29307B1032326F104930710001E
:10D4A8002328F10413061000930641056FF08FA599
:10D4B800832701012328E1000327C10083A7070070
:10D4C8002390E7006FE01FF283270101930C0B0004
:10D4D8002328E10083AD070093DEFD4113870E008A
:10D4E8006FF04FBE938D0700930E000013030B00DF
:10D4F8002328E1006FF09F812328E100938D070026
:10D50800930E0000930C0B00130710006FF0CF8FE1
:10D5180093FDF70F930E00006FF08F8D930C0B00A7
:10D528006FF0CFBC93079000E3E8B7DD6FF09FE1A1
:10D53800232451012328B101930A00006FF0CF8FF3
:10D54800938506006FF01FB9930516006FF0CFC7DB
:10D558009307F0FF2326F1006FF08F8213850600F2
:10D56800930506006FF09F8F03270101832A0700A8
:10D578009306470063D40A00930AF0FF03C71B0011
:10D588002328D100938B07006FE01FF1930C0B0049
:10D598006FF0CFA713030B006FF00FAF930C0B00C6
:10D5A8006FF00FB19306060013860500930505007A
:10D5B80003A5811C6FE09FD383D7C50003AE450642
:10D5C80003D3E50083A8C50103A84502130101B8E8
:10D5D80093F7D7FF13070040232C8146231AF10045
:10D5E800138405009307010793058100232A9146B8
:10D5F80023282147232E1146130905002326C10796
:10D60800231B610023221103232601032324F10095
:10D61800232CF1002328E100232EE100232001021E
:10D62800EFE0DFCC93040500635C050283574101FA
:10D6380093F70704638807008357C40093E7070438
:10D648002316F4008320C14703248147138504006F
:10D6580003290147832441471301014867800000DB
:10D668009305810013050900EF700F93E30005FC93
:10D678009304F0FF6FF09FFB03A301116700030001
:10D68800638405029307F00F63E8C7002380C50091
:10D6980013051000678000009307A0082320F500F9
:10D6A8001305F0FF67800000130500006780000085
:10D6B800130101FF93870500232481002322910091
:10D6C80093050600930405001385070013860600DA
:10D6D8002326110023A60120EF20DFE09307F0FFA7
:10D6E800630CF5008320C1000324810083244100DA
:10D6F800130101016780000083A7C120E38407FEAE
:10D708008320C1000324810023A0F4008324410066
:10D718001301010167800000B385C502130101FFF1
:10D728002324810023261100EF304FD41304050071
:10D73800630805020326C5FF130740021376C6FFD8
:10D748001306C6FF6360C7069306300193070500FA
:10D7580063E2C60223A0070023A2070023A4070050
:10D76800130504008320C100032481001301010173
:10D778006780000023200500232205009307B001DD
:10D7880063F0C70423240500232605009307050139
:10D79800E312E6FC2328050093078501232A0500E8
:10D7A8006FF05FFB93050000EF301FC813050400FE
:10D7B8008320C10003248100130101016780000058
:10D7C800930785006FF01FF9130101FF23248100DF
:10D7D80023229100930405001385050023261100D8
:10D7E80023A60120EF20DFAF9307F0FF630CF500BD
:10D7F8008320C10003248100832441001301010117
:10D808006780000083A7C120E38407FE8320C1004E
:10D818000324810023A0F4008324410013010101A3
:10D8280067800000130101FF2326110023248100D3
:10D83800232291002320210163800502930405001F
:10D84800138405006306050083278503638C070A94
:10D858008317C400639207028320C1000324810058
:10D86800130900001305090083244100032901005E
:10D87800130101016780000093050400138504006B
:10D88800EF60DFCB8327C40213090500638A070012
:10D898008325C40113850400E7800700634C05064F
:10D8A8008357C40093F70708639E0706832504037C
:10D8B800638C0500930704046386F5001385040050
:10D8C800EF704FBD232804028325440463880500B4
:10D8D80013850400EF700FBC23220404EF708FA699
:10D8E80023160400EF704FA68320C1000324810093
:10D8F80013050900832441000329010013010101D4
:10D9080067800000EF700FA38317C400E38607F455
:10D918006FF09FF68357C4001309F0FF93F70708C9
:10D92800E38607F88325040113850400EF708FB69A
:10D938006FF0DFF79305050003A5811C6FF09FEEDC
:10D94800130101FD23248102232E3101232A5101D1
:10D95800232611022322910223202103232C410193
:10D968002328610193090500938A05001304060022
:10D97800EFA00FBB930710006310F5029387FAFF1F
:10D988001307E00F636AF70013F7FA0F2306E100A5
:10D99800130910006F00C0029306C40513860A001D
:10D9A8009305C10013850900EF20C0469307F0FFD7
:10D9B800130905006304F50A630E05080347C1004F
:10D9C80093040000130AF0FF130BA0006F008002FD
:10D9D80083270400938617002320D4002380E700C0
:10D9E800938414009307C100B387970063F4240756
:10D9F80003C70700832784009387F7FF2324F400D5
:10DA0800E3D807FC83268401930507001306040066
:10DA18001385090063C4D700E31C67FBEF20402689
:10DA2800E31045FD1309F0FF8320C102032481029E
:10DA38001305090083244102032901028329C10136
:10DA4800032A8101832A4101032B010113010103E8
:10DA58006780000013890A006FF01FFD8357C40018
:10DA680093E707042316F4006FF01FFC8317C60022
:10DA7800139727016340070203274606B7260000CD
:10DA8800B3E7D700B72600003367D7002316F600A0
:10DA98002322E6066FF0DFEA130101FE232C810042
:10DAA80003A4811C232A9100232E1100930405004E
:10DAB8001386050063060400832784036384070430
:10DAC8008317C600139727016340070203274606FA
:10DAD800B7260000B3E7D700B72600003367D700A2
:10DAE8002316F6002322E606130504000324810109
:10DAF8008320C1019385040083244101130101029D
:10DB08006FF01FE4130504002326B100EF708F8225
:10DB18000326C1006FF0DFFA130101FF93870500A8
:10DB28002324810023229100930405009305060015
:10DB3800138507002326110023A60120EF200FFCE0
:10DB48009307F0FF630CF5008320C10003248100D4
:10DB580083244100130101016780000083A7C120CD
:10DB6800E38407FE8320C1000324810023A0F4007E
:10DB78008324410013010101678000008327860088
:10DB88006382073483D7C500130101FD2324810272
:10DB9800232C4101232A5101232611022322910219
:10DBA80023202103232E310123286101232671011B
:10DBB80023248101232291012320A10113F7870047
:10DBC80013840500930A0500130A0600630A070870
:10DBD80003A705016306070813F7270083240A0033
:10DBE8006300070A032744028327C401370B008018
:10DBF8009309000013090000134B0BC0138609009A
:10DC08009385070013850A00630409049306090035
:10DC180063742B0193060B00E7000700635AA028E2
:10DC280083278A00B389A9003309A9403385A7400F
:10DC38002324AA00630C05208327C4010327440278
:10DC4800138609009385070013850A00E31009FC71
:10DC580083A9040003A94400938484006FF01FFA89
:10DC68009305040013850A00EF600FDC631C053A76
:10DC78008357C40083240A0013F72700E31407F628
:10DC880013F7170063140724832C8400032504006A
:10DC9800B70B008013CCEBFF130B00001309000037
:10DCA80093CBFBFF630E090E13F70720630C0724C1
:10DCB800138D0C006362992F13F70748630A07084E
:10DCC800832644018325040113071900939916003C
:10DCD800B386D90093D9F601B30CB540B389D900FE
:10DCE80093D91940330797011386090063F6E900B1
:10DCF800930907001306070093F707406384072E6C
:10DD08009305060013850A00EF205FF6130D050042
:10DD1800630205308325040113860C00EF00403DA3
:10DD28008357C40093F7F7B793E707082316F4005F
:10DD380033059D01B38799412328A4012320A4001A
:10DD4800232A3401930C09002324F400130D09003D
:10DD580013060D0093050B00EF00404B832784004A
:10DD68000326040093090900B38C97413306A601E2
:10DD7800232494012320C4001309000083278A0068
:10DD8800330B3B01B389374123243A016380090CE3
:10DD9800832C8400032504008357C400E31609F08C
:10DDA80003AB040003A94400938484006FF09FEF41
:10DDB80083A9440083AB040093848400E38A09FEAA
:10DDC800138609009305A00013850B00EFA0CF9CD4
:10DDD8006304051213051500330B754193070B00F7
:10DDE800138C090063F43701138C07000325040022
:10DDF800832704018326440163F8A70003298400CC
:10DE080033892601634289096348DC1A832744025F
:10DE18008325C40113860B0013850A00E7800700D9
:10DE2800130905006356A008330B2B411305100096
:10DE3800630A0B1683278A00B38B2B01B389294108
:10DE48003389274123242A01631A0908130500008E
:10DE58008320C10203248102832441020329010291
:10DE68008329C101032A8101832A4101032B01016E
:10DE7800832BC100032C8100832C4100032D01005A
:10DE8800130101036780000093850B001306090046
:10DE9800EF00C037832704009305040013850A00A8
:10DEA800B38727012320F400EF601F8FE30E05F6E8
:10DEB8008317C40093E707042316F4001305F0FF43
:10DEC8006FF01FF91305000067800000130B0000B6
:10DED80013050000930B000093090000E38A09EC86
:10DEE800E31E05EE138609009305A00013850B00B9
:10DEF800EFA08F8AE31005EE93871900138B0700B4
:10DF08006FF01FEE8327040163E2A704832744010F
:10DF1800636EF9029306090063742C0193860B0063
:10DF2800B3C6F602032744028325C40113060B0077
:10DF380013850A00B386F602E7000700E35AA0F645
:10DF480093090500330939416FF05FE393890C00A9
:10DF580063749901930909001386090093050B005E
:10DF6800EF00C02A8327840003270400B3873741C2
:10DF7800330737012324F4002320E400E39407FC4B
:10DF88009305040013850A00EF601F81E31205F270
:10DF9800330939416FF09FDE930C0900130D090016
:10DFA8006FF01FDB9305040013850A00EF60CFFEB6
:10DFB800E30205E86FF0DFEF13060C0093850B0012
:10DFC800EF00C024032784008327040013090C00F2
:10DFD80033078741338C87012324E40023208401FD
:10DFE8006FF09FE413850A00EF00C03A130D050097
:10DFF800E31005D48325040113850A00EF609FC947
:10E008008317C4001307C00023A0EA0093F7F7F7AB
:10E018006FF05FEA9307C00023A0FA008317C400DB
:10E028006FF05FE91305F0FF6FF09FE2130101FF46
:10E038002324810023229100930405001385050001
:10E048002326110023A60120EF208FAE9307F0FFAF
:10E05800630CF5008320C100032481008324410060
:10E06800130101016780000083A7C120E38407FE34
:10E078008320C1000324810023A0F40083244100ED
:10E088001301010167800000130101FF9387050058
:10E0980023248100232291009305060093040500A0
:10E0A80013850700138606002326110023A60120E6
:10E0B800EF208FAB9307F0FF630CF5008320C100BE
:10E0C80003248100832441001301010167800000BB
:10E0D80083A7C120E38407FE8320C10003248100B5
:10E0E80023A0F4008324410013010101678000008C
:10E0F800B3C7A50093F73700B308C50063920706B6
:10E108009307300063FEC7049377350013070500B3
:10E118006398070613F6C8FF930706FE636CF708B3
:10E12800637CC702938605009307070003A80600CF
:10E13800938747009386460023AE07FFE3E8C7FEB0
:10E148009307F6FFB387E74093F7C7FF9387470026
:10E158003307F700B385F50063681701678000008F
:10E1680013070500E37C15FF83C705001307170095
:10E1780093851500A30FF7FEE36817FF678000007B
:10E1880083C605001307170093773700A30FD7FE40
:10E1980093851500E38007F883C605001307170069
:10E1A80093773700A30FD7FE93851500E39A07FCF2
:10E1B8006FF05FF683A6050083A2450083AF850054
:10E1C80003AFC50083AE050103AE450103A3850176
:10E1D80003A8C501938545022320D70083A6C5FF60
:10E1E800232257002324F7012326E7012328D701F8
:10E1F800232AC701232C6700232E07011307470290
:10E20800232ED7FEE368F7FA6FF09FF163F6A502B5
:10E21800B387C5006372F5023307C500630A060EAB
:10E228009387F7FF83C607001307F7FF2300D7007C
:10E23800E398F5FE678000009307F00063E8C702E3
:10E24800930705009306F6FF630C060C93861600E9
:10E25800B386D7009385150003C7F5FF938717008A
:10E26800A38FE7FEE398D7FE67800000B3E7A50019
:10E2780093F737006390070A930806FF93F808FF9F
:10E2880093880801330815011387050093070500D3
:10E2980083260700938707011307070123A8D7FEE2
:10E2A800832647FF23AAD7FE832687FF23ACD7FE02
:10E2B8008326C7FF23AED7FEE31CF8FC1377C600FE
:10E2C800B38515011378F600630E0704138705005C
:10E2D80093880700130E3000130747000323C7FF76
:10E2E80093884800B306E84023AE68FEB386D5009D
:10E2F800E364DEFE1307C8FF1377C7FF1307470061
:10E3080013763600B387E700B385E5006FF09FF317
:10E31800678000009306F6FF930705006FF01FF370
:10E3280067800000130608006FF0DFF1130101FF9A
:10E33800938705002324810023229100930506007A
:10E348009304050013850700138606002326110091
:10E3580023A60120EF20CF8D9307F0FF630CF50073
:10E368008320C1000324810083244100130101019B
:10E378006780000083A7C120E38407FE8320C100D3
:10E388000324810023A0F400832441001301010128
:10E3980067800000130101FD232E3101232611029D
:10E3A800232481022322910223202103232C4101CB
:10E3B800232A510123286101232671012324810185
:10E3C80093090600638A0522138B0500930A05004A
:10E3D800EF304F931384B9009307600163FC870EF5
:10E3E800137484FF13070400634C040E636A340F2C
:10E3F8008327CBFF13098BFF93F4C7FF330A9900D8
:10E4080063D2E41A938B81C203A68B0083264A0049
:10E418006306462513F6E6FF3306CA0003264600C0
:10E4280013761600631C061A93F6C6FF3386D400CB
:10E438006356E63493F7170063940702032C8BFFA7
:10E44800330C894183274C0093F7C7FFB386D70065
:10E45800B38B960063D6EB0CB38BF40063D8EB3424
:10E468009385090013850A00EF205F809309050052
:10E47800630C05048327CBFF130785FF93F7E7FF9A
:10E48800B307F900638AE7301386C4FF9307400295
:10E4980063EAC7381307300183260B006364C72873
:10E4A8009307050013070B0023A0D7008326470016
:10E4B80023A2D7000327870023A4E70093050B00B6
:10E4C80013850A00EF600FFD13850A00EF30CF8334
:10E4D8006F00C0011304000113070001E37A34F14F
:10E4E8009307C00023A0FA00930900008320C1020B
:10E4F80003248102138509008324410203290102B0
:10E508008329C101032A8101832A4101032B0101C7
:10E51800832BC100032C81001301010367800000D5
:10E528008327CA0003278A001386C4FF9306400284
:10E538002326F70023A4E70003278C008327CC00B9
:10E5480093098C00330A7C012326F70023A4E700F3
:10E5580063E0C62E9306300103270B00938709005A
:10E5680063F2C6022324EC0003274B009307B00193
:10E578002326EC0003278B0063EEC73293070C01B8
:10E58800130B8B0023A0E70003274B0093840B0099
:10E5980013090C0023A2E70003278B00138B090043
:10E5A80023A4E70003264900B38784401307F0003B
:10E5B80013761600636CF70633E6C4002322C900FD
:10E5C80083274A0093E717002322FA0013850A00DD
:10E5D800EF209FF393090B006FF05FF193F717009B
:10E5E800E39007E8032C8BFF330C894183274C0009
:10E5F80093F7C7FF6FF05FE6032481028320C1020F
:10E6080083244102032901028329C101032A8101CC
:10E61800832A4101032B0101832BC100032C8100B4
:10E6280093050600130101036F204FE4336686004B
:10E638002322C900B305890093E7170023A2F50038
:10E6480083274A009385850013850A0093E71700FE
:10E658002322FA00EF600FE46FF05FF793F6C6FF2E
:10E668003386D400930504016350B60E93F7170060
:10E67800E39807DE032C8BFF330C894183274C007A
:10E6880093F7C7FFB386D700338A9600E346BADC10
:10E698008327CC0003278C001386C4FF930640020F
:10E6A8002326F70023A4E70093098C0063E6C6221B
:10E6B8009305300103270B009387090063F2C50215
:10E6C8002324EC0003274B009307B0012326EC001A
:10E6D80063EAC72403278B0093070C01130B8B00F5
:10E6E80023A0E70003274B0023A2E70003278B00A2
:10E6F80023A4E70033078C00B3078A4023A4EB0068
:10E7080093E717002322F70083274C0013850A009C
:10E7180093F7170033E4870023228C00EF20DFDE15
:10E728006FF0DFDC2320D50083264B001307B001F0
:10E738002322D500636CC71013078B00930785004D
:10E7480083268B006FF05FD633098900B3078640B4
:10E7580023A42B0193E717002322F9008327CBFF7B
:10E7680013850A0093090B0093F7170033E4870019
:10E77800232E8BFEEF205FD96FF05FD78327CA0067
:10E7880003278A0093040600330AC9002326F700EA
:10E7980023A4E7006FF01FE18327C5FF93F7C7FFA6
:10E7A800B384F400330A99006FF0DFDF0327CC004D
:10E7B80083268C001386C4FF9305400223A6E60037
:10E7C8002324D70093098C00330A7C0163E2C50631
:10E7D8001305300183260B00138709006372C502F5
:10E7E8002324DC0003274B009307B0012326EC0009
:10E7F80063E0C70A83268B0013070C01130B8B00F9
:10E808002320D70083264B0093840B0013090C00A8
:10E818002322D70083278B00138B09002324F700BA
:10E828006FF05FD893050B00EFF05F9E6FF01FC984
:10E8380093050B0013850900EFF05F9D138B09000A
:10E8480093840B0013090C006FF0DFD503278B00AE
:10E858002324E5000327CB002326E500630AF600FE
:10E8680013070B019307050183260B016FF0DFC324
:10E8780083260B0113078B01930785012328D500F5
:10E8880083264B01232AD50083268B016FF0DFC135
:10E8980083278B002328FC008327CB00232AFC0036
:10E8A8006304B60483260B0113078C01130B0B01B9
:10E8B8006FF01FF52328EC000327CB0093074002D5
:10E8C800232AEC0003270B016300F60493078C014D
:10E8D800130B0B016FF01FCB93050B001385090079
:10E8E800EFF0DF926FF01FE183270B0113070C0293
:10E8F800130B8B01232CFC008327CBFF232EFC005A
:10E9080083260B006FF0DFEF232CEC0003274B016D
:10E9180093070C02130B8B01232EEC0003270B002B
:10E928006FF05FC683278B002328FC008327CB006A
:10E93800232AFC0003270B016308D60093078C01E8
:10E94800130B0B016FF0DFD9232CEC0003274B01CD
:10E9580093070C02130B8B01232EEC0003270B00EB
:10E968006FF01FD883278600130101FD232A510168
:10E97800232611022324810223229102232021032A
:10E98800232E3101232C4101232861012326710103
:10E9980023248101930A060063880714130B0500DA
:10E9A800138405008329060003A5050083A48500B8
:10E9B8006F00400D8357C40013F70748630A070820
:10E9C8008326440183250401130719009394160034
:10E9D800B386D40093D4F601330AB540B384D40087
:10E9E80093D41440330747011386040063F6E40008
:10E9F800930407001306070093F707406386070A86
:10EA08009305060013050B00EF204FA6130C050015
:10EA1800630A050A8325040113060A00EFF04FED87
:10EA28008357C40093F7F7B793E707082316F40052
:10EA380033054C01338A4441232A9400232444019A
:10EA4800232884012320A40093040900130A090041
:10EA580013060A0093850B00EFF04FFB0327840091
:10EA68000325040083A78A00B304974033054501B2
:10EA7800232494002320A4003389274123A42A01B6
:10EA88006304090603A9490083AB0900138A04003B
:10EA980093898900E30809FEE37E99F0930409004D
:10EAA800130A09006FF0DFFA13050B00EFF09F8ED1
:10EAB800130C0500E31E05F68325040113050B005E
:10EAC800EF604F9D9307C0002320FB008357C400CD
:10EAD8001305F0FF93E707042316F40023A40A00A4
:10EAE80023A20A006F00C00023A20A001305000039
:10EAF8008320C102032481028324410203290102E5
:10EB08008329C101032A8101832A4101032B0101C1
:10EB1800832BC100032C81001301010367800000CF
:10EB280083D7C500130101ED232A51112326711142
:10EB3800232EB10F2326111223248112232291128E
:10EB480023202113232E3111232C41112328611155
:10EB580023248111232291112320A11193F707085F
:10EB68002324D100938A0500930B0500930D06001A
:10EB78006386070083A70501E38C075E375D018084
:10EB88009309C10493074DFE375B0180B754018098
:10EB9800138A0D00232031052324010423220104B4
:10EBA800232A0100232E010023200102232201022F
:10EBB800232201002326F100130B0B15938404165E
:10EBC80023287101938D090083470A006384071283
:10EBD80093065002E384D75213040A006F00C00062
:10EBE8006386D70E13040C0083471400130C14001B
:10EBF800E39807FEB30C4C41638E0C0E0327810487
:10EC08008327410423A04D013307970193871700F9
:10EC180023A29D012324E1042322F1041307700099
:10EC2800938D8D00634AF70A032741008347140038
:10EC3800330797012322E100638E070A1308F0FFC8
:10EC4800130A1C0083461C00A30D010213040000D4
:10EC580013090000130CA005930C9000130DA002DB
:10EC6800930B0800130A1A00938706FE6360FC1CC6
:10EC78000327C10093972700B387E70083A70700FE
:10EC88006780070003250101EF90CF8083274500A7
:10EC9800138507002322F102EFA01F8F2320A10272
:10ECA80003250101EF801FFF032785008327010249
:10ECB800232EE100E398074483460A006FF09FFA89
:10ECC8001369090283460A006FF0DFF9B30C4C415F
:10ECD800E3860CF66FF09FF2032501011306010489
:10ECE80093850A00EFF01FC863140502938D09008D
:10ECF8006FF09FF383278104832B0101638A070048
:10ED08001306010493850A0013850B00EFF09FC5D5
:10ED180083D7CA0093F70704E39607708320C112CC
:10ED2800032481120325410083244112032901127F
:10ED38008329C111032A8111832A4111032B01114F
:10ED4800832BC110032C8110832C4110032D01103B
:10ED5800832DC10F1301011367800000B74701809D
:10ED68009387477F232AF1009377090213880B00C2
:10ED78006388074C8327810013867700137686FF04
:10ED8800032D0600832C4600930786002324F100F8
:10ED9800137619006306060033669D01E3120638F0
:10EDA800137CF9BF93062000A30D01021306F0FFA0
:10EDB8006306C86033669D011379FCF7E3140614F3
:10EDC8006314086EE394062E937C1C00930B010FCA
:10EDD80063880C0093070003A307F10E930BF10E51
:10EDE800130C080063549801138C0C008347B1037B
:10EDF800B337F000330CFC006F000005130400006B
:10EE0800138706FD130A1A00931724008346FAFF96
:10EE1800338487001314140033048700138706FD16
:10EE2800E3F2ECFE938706FEE374FCE4E38406EC6D
:10EE38002306D108A30D0102130C1000930C100037
:10EE4800930BC10813080000937E290063840E0009
:10EE5800130C2C00137E49088327810403264104E0
:10EE680063160E00330D8441E342A00B0345B10342
:10EE78009305160093868D00630005041305B103FE
:10EE88009387170023A0AD001305100023A2AD003F
:10EE98002324F1042322B10413057000E346B518B6
:10EEA800130F260013850D0113860500938D0600A8
:10EEB80093050F0093060500638C0E021306C10329
:10EEC8009387270023A0CD001306200023A2CD009E
:10EED8002324F1042322B10413067000E348B61872
:10EEE80013860500938D060093851500938686008A
:10EEF800130500086306AE60330D9841634AA06F9E
:10EF0800B387FC0023A07D0123A29D012324F104E3
:10EF18002322B10413067000634AB67A9378490035
:10EF280063860800B30C84416348901F63548401CE
:10EF380013040C0003274100330787002322E10054
:10EF48006396077A23220104938D09006FF0DFC7C7
:10EF58008327810013880B00A30D010283AB0700F0
:10EF6800138D4700E38C0B349307F0FFE306F81E7C
:10EF7800130608009305000013850B0023240101E4
:10EF8800EF908F8103288100E3000548B30C754199
:10EF98002324A101130800006FF09FE4937709026E
:10EFA80013880B009368090163940748832781003D
:10EFB8009386470083278100930C00002324D10007
:10EFC80003AD07006F0080489377090213880B0090
:10EFD800136C0901639407488327810093864700CF
:10EFE80083278100930C00002324D10003AD070080
:10EFF800930610006FF05FDB1369090883460A0067
:10F008006FF05FC683460A0093071A00E382A6439F
:10F01800138706FD138A0700930B0000E3E6ECC490
:10F02800130A1A0093972B008346FAFF3388770157
:10F0380013181800B30BE800138706FDE3F2ECFE83
:10F048006FF09FC283460A00136949006FF09FC1A1
:10F058009307B002A30DF10283460A006FF09FC028
:10F068008327810083460A0003A40700938747008B
:10F078002324F100E35804BE330480401369490097
:10F088006FF05FBE9377090213880B00136C0901B8
:10F09800639A073E83278100938647008327810070
:10F0A8002324D10003AD0700935CFD4193860C0037
:10F0B80063C2062E9306F0FF630AD800B3669D016B
:10F0C8001379FCF76382067E130C0900E3920C0C9B
:10F0D80093069000E3EEA60B93070D03A307F10E2A
:10F0E80013090C00930C1000930BF10E6FF05FCF17
:10F0F80003278100A30D0102130C100083270700CA
:10F10800130747002324E1002306F108930C10009D
:10F11800930BC1086FF01FD3930500010326410428
:10F1280063D29507130D0001930D700003290101A7
:10F138006F00C000938C0CFF63569D0593870701F1
:10F148001306160023A0660123A2A6012324F104B6
:10F158002322C10493868600E3DECDFC1306010456
:10F1680093850A0013050900EFF0CFFFE31205BAF3
:10F17800938C0CFF8327810403264104938609009E
:10F18800E34E9DFBB38797011306160023A0660183
:10F1980023A296012324F1042322C10493067000BC
:10F1A800E3D6C6D8032501011306010493850A0096
:10F1B800EFF04FFBE31E05B4832781046FF01FD7E0
:10F1C8001369190083460A006FF0DFA98347B1036A
:10F1D80083460A00E39807A893070002A30DF102EB
:10F1E8006FF05FA89377090213880B0063960726D0
:10F1F80083278100137609019386470083A70700B8
:10F20800E318062613760904E30A060E139D070180
:10F218002324D100135D0D01930C0000130C090089
:10F22800930610006FF05FB8B74701809387077E99
:10F23800232AF1009377090213880B00E39C07B295
:10F248000327810013760901832707001307470066
:10F258002324E10063180666137609046300066632
:10F26800139D0701135D0D01930C00006FF05FB251
:10F2780083278100B786FFFF93C6068303AD070087
:10F28800231ED10293874700B74601802324F1004B
:10F298009387067E13880B00930C0000136C2900DB
:10F2A800232AF100930620006FF01FB0937709021C
:10F2B80013880B00639C07168327810013760901C6
:10F2C8009386470083A70700E318061A13760904F4
:10F2D800E3080600139D0701135D0D01930C000060
:10F2E800930809002324D1006F00401603278100EA
:10F2F800937709029306470063920764937709019D
:10F308006392077A93770904E396070893780920AC
:10F31800638A087883278100032741002324D100CA
:10F3280083A707002380E7006FF01F8A83460A003F
:10F338009307C0066380F676136909016FF09F9200
:10F3480083460A00930780066384F67013690904EC
:10F358006FF05F919377090213880B00639207128D
:10F36800032781009377090193064700E39E070E60
:10F37800937709046384077A832781002324D100C3
:10F38800130C0900039D0700935CFD4193860C0054
:10F39800E3D206D2B307A041B336F000330E904152
:10F3A800B30CDE409306D002A30DD1021306F0FF82
:10F3B800138D070093061000E31EC89E1306100065
:10F3C800E386C6D013062000638AC60E1306010F13
:10F3D8006F00800013860B009397DC0193767D0005
:10F3E800135D3D009386060333EDA70193DC3C00D3
:10F3F800A30FD6FEB3679D01930BF6FFE39C07FCB2
:10F4080093771C006386070E930700036382F60E4A
:10F418001306E6FFA38FFBFE9307010FB38CC740CB
:10F4280013090C00930B06006FF09F9B93080900CB
:10F43800832781009386770093F686FF03AD060045
:10F4480083AC4600938786002324F10013FCF8BFA1
:10F45800930600006FF05F95130C09008327810065
:10F468009386770093F686FF9387860003AD0600A0
:10F4780083AC46002324F100930610006FF0DF925E
:10F48800130C0900832781009387770093F787FF80
:10F4980083A64700138787002324E10003AD0700F4
:10F4A800938C06006FF0DFC013061000638AC674E1
:10F4B80013062000130C0900E39AC6F083264101C5
:10F4C800930B010F9377FD00B387F60083C70700FE
:10F4D8001397CC01135D4D00938BFBFF336DA70190
:10F4E80093DC4C002380FB00B3679D01E39C07FC81
:10F4F8009307010FB38C774113090C006FF05F8EEF
:10F50800330D8441E35AA09F130500016356A5718A
:10F5180013870D00232C2101930D0A0013090D00F8
:10F52800130A0400138D0C0093060001930C0C00C1
:10F53800130E7000130C0800032401016F00C000B3
:10F54800130909FF63DA26059387070113061600D6
:10F55800232097002322D7002324F1042322C10467
:10F5680013078700E35ECEFC1306010493850A00A7
:10F5780013050400EFF00FBF631C05F893060001A4
:10F58800130909FF8327810403264104138709000F
:10F59800130E7000E3CA26FB13080C00138C0C0032
:10F5A800930C0D00130D09000329810113040A00AF
:10F5B80013061600138A0D0013058700930D070024
:10F5C800B387A70123A09D0023A2AD012324F10442
:10F5D8002322C1049306700063C4C648330D9841C2
:10F5E8009305160093068500930D0500E35AA09134
:10F5F800130500016356A555232C2101930600012C
:10F6080013090D0013087000130D0A00130A0400F3
:10F61800032401016F00C000130909FF63DA2605FE
:10F62800938707011306160023A09D0023A2DD007F
:10F638002324F1042322C104938D8D00E35EC8FCCA
:10F648001306010493850A0013050400EFF08FB137
:10F65800631005EC93060001130909FF8327810451
:10F6680003264104938D090013087000E3CA26FBA2
:10F6780013040A00130A0D00130D09000329810160
:10F688009305160013868D00B387A70123A09D005C
:10F6980023A2AD012324F1042322B10493067000B0
:10F6A80063C8B622930D060093851500B387FC0046
:10F6B8009306860023A07D0123A29D012324F10443
:10F6C8002322B10413067000E35AB684032501010E
:10F6D8001306010493850A00EFF0CFA8631A05E228
:10F6E80083278104938609006FF05F830325010156
:10F6F8001306010493850A00EFF0CFA6E3040584FE
:10F708006FF00FE1130C09006FF05FCB9306000157
:10F7180063DCA60B13870D0023262103930D0A0033
:10F72800130F7000130A0400232CD10113040D00D9
:10F738002324C103138D0C0003290101930C0C0031
:10F74800130C08006F00C000130404FF63DA86047A
:10F758009387070113061600232067012322D70089
:10F768002324F1042322C10413078700E35ECFFC9E
:10F778001306010493850A0013050900EFF08F9E14
:10F78800631805D893060001130404FF8327810436
:10F798000326410413870900130F7000E3CA86FA91
:10F7A800832E8101032E81020329C10213080C0054
:10F7B800138C0C00930C0D00130D040013040A00A5
:10F7C800138A0D00930D0700B387A70113061600CF
:10F7D80023A06D0123A2AD012324F1042322C10437
:10F7E80093067000938D8D0063D2C6E8032501014E
:10F7F8001306010493850A00232601032324C10369
:10F80800232CD101EFF00F96631405D083278104D0
:10F8180003264104938D09000328C102032E8102A7
:10F82800832E81016FF08FE4032501011306010483
:10F8380093850A00232601032324C103232CD10125
:10F84800EFF04F92631605CC032641048327810409
:10F858009306410593051600938D09000328C102FC
:10F86800032E8102832E81016FF00FE5032501012C
:10F878001306010493850A0023240103232CC101E4
:10F88800EFF04F8E631605C80326410483278104D1
:10F898009306410593051600938D090003288102FC
:10F8A800032E81016FF0CFE4631C083413080000B5
:10F8B800930C0000930B010F6FF08FD21376092081
:10F8C8006316062E138D0700930C00006FF04FCCC3
:10F8D800032501011306010493850A00EFF08F88C0
:10F8E800631805C2832541048327810493064105D3
:10F8F80093851500938D09006FF08FE0130C0A00B3
:10F908006FF0CFB38327C10183460A00638C07B425
:10F9180083C70700638807B4136909406FF08FB481
:10F928001306000313692900A30ED102230EC10296
:10F93800137CF9BF930620006FF00FC783270700D9
:10F94800032741002324D1001356F74123A0E700E1
:10F9580023A2C7006FF04FA713850B00EF90DFC2FB
:10F96800930C05002324A101130800006FF04FC772
:10F9780093050004EF108FAF23A0AA0023A8AA00C4
:10F98800630A052C9307000423AAFA006FF00F9F5F
:10F9980093770C40930B010F232C810013840700ED
:10F9A80093870C0023264103938C0A001309000057
:10F9B800938A0B0023240103032AC101938B0700B8
:10F9C8006F0040021306A0009306000013050D0007
:10F9D80093850B00EF00C05363880B1A130D0500C5
:10F9E800938B05001306A0009306000013050D0075
:10F9F80093850B00EF00101513050503A38FAAFECE
:10FA080013091900938AFAFFE30E04FA83460A00E1
:10FA1800E39A26FB9307F00FE306F9FA63960B12B5
:10FA28009307900063E2A713938B0A009307010FD3
:10FA3800232E4101938A0C000324810103288102AB
:10FA4800032AC102B38C774113090C006FF04FB938
:10FA580083461A0013690920130A1A006FF08FA051
:10FA6800032501011306010493850A00232C0101D3
:10FA7800EFE05FEF631E05A8032641048327810496
:10FA88009306410593051600938D0900032881010B
:10FA98006FF08FC683461A0013690902130A1A0009
:10FAA8006FF04F9C832781000327410083A707003D
:10FAB8002324D10023A0E7006FF00F919307600083
:10FAC800930C080063F40701930C6000375301801E
:10FAD800138C0C002324A101930B83806FF08FB645
:10FAE800137609206304061013FDF70F930C00002A
:10FAF800930809002324D1006FF05F95137609203D
:10FB0800630A060C2324D10013FDF70F930C0000A1
:10FB1800130C0900930610006FF00FA993770920C2
:10FB2800638C070883278100130C09002324D10064
:10FB3800038D0700935CFD4193860C006FF04FD74F
:10FB4800138606006FF05FB4832701028325410204
:10FB580013090000B38AFA401386070013850A00C8
:10FB6800EF905FAB03481A001306A000930600004D
:10FB78003338000113050D0093850B00330A0A0181
:10FB8800EF0000396FF09FE593079000E3E8A7E5E1
:10FB98006FF09FE983278100032741002324D100C8
:10FBA80083A707002390E7006FF00F8213FDF70F7C
:10FBB800930C00006FF0CF9D83278100130C090080
:10FBC8002324D10003AD0700935CFD4193860C000C
:10FBD8006FF00FCE2324D100138D0700930C000083
:10FBE800130C0900930610006FF00F9C138D07008B
:10FBF800930C0000930809002324D1006FF01F859F
:10FC0800130C09006FF04FCD930C08002324A101B9
:10FC1800130800006FF0CF9C1385060013860500BB
:10FC28006FF01F9A9307F0FF2322F1006FF00F8FF8
:10FC380003278100832B07001307470063D40B00B9
:10FC4800930BF0FF83461A002324E100138A070070
:10FC58006FF04F819307C00023A0FB009307F0FFCC
:10FC68002322F1006FF08F8B130C09006FF00FC384
:10FC7800130C09006FF0CFB6930809006FF08FB32B
:10FC8800130101FE232C8100232A9100232821013E
:10FC9800232E110023263101130905009384050042
:10FCA8001304060063060500832785036388071489
:10FCB8000317C400832784019316070193D606010E
:10FCC8002324F40093F7860063820708832704013E
:10FCD800638E07061396260193F9F40F93F4F40F35
:10FCE800635E06080327040083264401B307F74030
:10FCF80063DED70A83268400130617002320C40076
:10FD08009386F6FF2324D4002300370103274401F8
:10FD1800938717006308F70C8357C40093F71700FD
:10FD2800638607009307A000638EF40A8320C1014D
:10FD3800032481011385040003290101832441015F
:10FD48008329C100130101026780000093050400A4
:10FD580013050900EF404FCD631E05080317C400C3
:10FD680093F9F40F832704019316070193D606012C
:10FD78001396260193F4F40FE34606F68326440609
:10FD8800372600003367C70037E6FFFF1306F6FF84
:10FD9800B3F6C6002316E400032704002322D40682
:10FDA80083264401B307F740E3C6D7F4930504005C
:10FDB80013050900EF405F9E631E05020327040038
:10FDC8008326840093071000130617009386F6FF16
:10FDD8002320C4002324D40023003701032744012F
:10FDE800E31CF7F29305040013050900EF40DF9ABE
:10FDF800E30E05F29304F0FF6FF05FF3EF409FD33B
:10FE08006FF01FEB138605009305050003A5811C01
:10FE18006FF01FE7130101FE232C8100232A9100B4
:10FE2800232E1100130405009384060083A70111F3
:10FE380063820502E78007009307F0FF6306F50277
:10FE48008320C1010324810183244101130101029C
:10FE5800678000001306000093054100E780070053
:10FE68009307F0FFE31EF5FC23A004009307A00806
:10FE78002320F4008320C10103248101832441014C
:10FE88001301010267800000130101FE232C810089
:10FE9800232A910003A4811C232E11009304060039
:10FEA80083A701119306060063080502138605005F
:10FEB8009305050013050400E78007009307F0FF8A
:10FEC8006308F5028320C1010324810183244101D1
:10FED800130101026780000013060000930541002A
:10FEE80013050400E78007009307F0FFE31CF5FC07
:10FEF80023A004009307A0082320F4008320C10155
:10FF08000324810183244101130101026780000059
:10FF1800938705001308060093880600130305005D
:10FF280063960628375701801307472263F6C50EE4
:10FF3800B70601006378D60C9306F00FB3B6C60077
:10FF480093963600B358D6003307170103470700C6
:10FF5800B306D700130700023307D740630C070026
:10FF6800B397E700B356D5003318E600B3E5F600BB
:10FF78003313E5001355080133F7A50213160801DA
:10FF88001356060193560301B3D5A50213170701AB
:10FF9800B366D700B307B6021387050063FEF60001
:10FFA800B38606011387F5FF63E8060163F6F600DA
:10FFB8001387E5FFB3860601B386F640B3F7A602BA
:10FFC8001313030113530301B3D6A6029397070132
:10FFD80033E36700B305D60213850600637CB300DC
:10FFE800330368001385F6FF636603016374B30087
:08FFF8001385E6FF1317070152
:02000004800179
:100000003367A700930500006F00400EB70800019A
:1000100093060001E36C16F3930680016FF01FF363
:10002000631606009306100033D8C602B706010017
:100030006372D80C9306F00F63F4060193088000F6
:10004000B35618013307D700834607001307000291
:10005000B38616013307D7406318070AB3870741F1
:1000600093051000135608019318080193D808014E
:100070009356030133F7C702B3D7C702131707011B
:10008000B366D7003385F8021387070063FEA60026
:10009000B38606011387F7FF63E8060163F6A6003F
:1000A0001387E7FFB3860601B386A640B3F7C602FF
:1000B0001313030113530301B3D6C6029397070129
:1000C00033E36700B388D80213850600637C13010D
:1000D000330368001385F6FF63660301637413013D
:1000E0001385E6FF131707013367A7001305070001
:1000F00067800000B706000193080001E362D8F4AE
:10010000930880016FF0DFF33318E800B3D5D70010
:100110003313E500B356D50013550801B397E70034
:1001200033F7A502B3E8F6009317080193D7070148
:1001300013D60801B3D5A502131707013367C7000B
:10014000B386B70213860500637ED7003307070125
:100150001386F5FF636807016376D7001386E5FF12
:1001600033070701B306D74033F7A6029398080177
:1001700093D80801B3D6A60213170701B385D70297
:10018000B36717011387060063FEB700B387070143
:100190001387F6FF63E8070163F6B7001387E6FFEE
:1001A000B3870701B387B74093150601B3E5E500B0
:1001B0006FF05FEB63E6D5183707010063F4E604E0
:1001C0001308F00F3337D800131737003758018062
:1001D00013084822B3D5E600B385050103C805001E
:1001E000930500023308E800B385054163960502D4
:1001F00013071000E3ECF6EE3335C5001347150086
:100200006FF0DFEEB705000113070001E3E0B6FC75
:10021000130780016FF09FFB33570601B396B600BA
:10022000B366D70093DE060133D70701B378D7034F
:10023000B397B700335805013363F800939706016D
:1002400093D70701135803013316B6003357D7036A
:100250009398080133E80801338FE702130E070073
:10026000637EE8013308D800130EF7FF6368D800F7
:100270006376E801130EE7FF3308D8003308E8413E
:10028000B378D8033358D80393980801B38E070383
:100290009317030193D70701B3E7F800130708008A
:1002A00063FED701B387D7001307F8FF63E8D700D1
:1002B00063F6D7011307E8FFB387D700131E0E01BB
:1002C000B387D741B70E01003367EE001388FEFFF6
:1002D000337307019358070133780601135606015B
:1002E000330E03033388080393560E013303C3020E
:1002F00033030301B3866600B388C80263F40601C2
:10030000B388D80113D60601B308160163E61703B4
:10031000E39A17CFB70701009387F7FFB3F6F6000C
:1003200093960601337EFE003315B500B386C601F1
:1003300093050000E37CD5DA1307F7FF6FF09FCC3D
:1003400093050000130700006FF05FDA93080600C2
:10035000138706009307050013880500639C062297
:10036000B75601809386462263FCC50C3703010013
:10037000637E660A1303F00F6374C30013078000E3
:100380003353E600B386660003CE06001303000273
:10039000330EEE003303C341630C0300B3956500D5
:1003A000335EC501B31866003368BE00B31765003D
:1003B00013D608013377C8021395080113550501B8
:1003C00093D607013358C80213170701B366D70045
:1003D0003308050363FA0601B386160163E61601C6
:1003E00063F40601B3861601B386064133F7C602ED
:1003F0009397070193D70701B3D6C602B306D50278
:1004000013150701B367F50063FAD700B387170127
:1004100063E6170163F4D700B3871701B387D740AA
:1004200033D56700930500006780000037030001A3
:1004300013070001E36666F4130780016FF05FF4B1
:100440006316060013061000B358160337060100A2
:1004500063F2C80A1306F00F6374160113078000D5
:1004600033D6E800B386C60003CE060013030002AD
:10047000330EEE003303C34163180308B3851541FF
:1004800013D70801139508011355050113D6070169
:10049000B3F6E502B3D5E50293960601B3E6C600CE
:1004A000B305B50263FAB600B386160163E616011A
:1004B00063F4B600B3861601B385B640B3F6E50221
:1004C0009397070193D70701B3D5E502B305B502AA
:1004D00013950601B367F50063FAB700B3871701F8
:1004E00063E6170163F4B700B3871701B387B7401A
:1004F0006FF01FF33706000113070001E3E2C8F6AF
:10050000130780016FF0DFF5B398680033D7C5019A
:10051000B3176500335EC50113D50801B376A70292
:10052000B3956500336EBE009395080193D5050120
:1005300013560E013357A70293960601B3E6C60081
:100540003387E50263FAE600B386160163E6160117
:1005500063F4E600B38616013386E640B376A6025E
:10056000131E0E01135E0E013356A602939606016A
:100570003386C502B3E5C60163FAC500B38515012C
:1005800063E6150163F4C500B3851501B385C54065
:100590006FF01FEFE3EAD5E83707010063FCE604DC
:1005A000930EF00F33B7DE00131737003753018077
:1005B000B3D8E60013034322B388680083CE080053
:1005C000130E0002B38EEE00330EDE41631E0E02E8
:1005D00063E4B600636AC500B307C540B385D54080
:1005E0003335F5003388A5401385070093050800CF
:1005F0006FF09FE3B708000113070001E3E816FB63
:10060000130780016FF09FFA3357D601B396C601E6
:10061000B366D70013D8060133D7D5013373070368
:10062000B395C501B357D501B3E7B700939506015C
:1006300093D5050193D807013316C6013315C501BB
:100640003357070313130301B3681301338FE50214
:100650001303070063FEE801B388D8001303F7FF14
:1006600063E8D80063F6E8011303E7FFB388D80016
:10067000B388E84133FF0803B3D80803131F0F0101
:10068000338815039395070193D50501B365BF0022
:100690009387080063FE0501B385D5009387F8FFB3
:1006A00063E8D50063F605019387E8FFB385D500BD
:1006B00013130301370F01003363F3009307FFFFA8
:1006C000B378F300B38505411353030113580601B2
:1006D000B377F6003387F802B307F302B388080351
:1006E00033030303B388F8001358070133081801D4
:1006F0006374F8003303E301935708013383670001
:10070000B70701009387F7FF3378F8001318080143
:100710003377F7003307E80063E66500639E650002
:10072000637CE5003306C7403337C7003307D70083
:100730003303E340130706003307E5403335E50094
:10074000B3856540B385A540B397D5013357C7013D
:1007500033E5E700B3D5C5016FF01FCD130101FDEF
:1007600013D8450123229102232E3101232C41016C
:1007700023286101232671019394C50023261102C9
:100780002324810223202103232A51011378F87F97
:10079000130B0500930B0600138A060093D4C400C4
:1007A00093D9F5016300080A9307F07F630EF80EF2
:1007B000935AD50193943400B3E49A00B70A8000A9
:1007C000B3EA540113143500130918C0130B0000C9
:1007D00013554A019314CA001378F57F93D4C400CB
:1007E000135AFA01630008109307F07F6300F816AC
:1007F0001395340093D7DB0133E5A700B7048000DD
:10080000B3649500139F3B00130518C093070000C5
:1008100013172B003367F7001307F7FF9306E00069
:1008200033C649013308A94063EEE614B756018088
:1008300013172700938606173307D70003270700EF
:1008400067000700B3EAA400638E0A06638004040D
:1008500013850400EF30D041930755FF1307C00103
:10086000634CF702930AD001130485FFB38AFA4060
:10087000B3948400B35A5B01B3EA9A0033148B003B
:100880001308D0C03309A8406FF05FF4EF30503E3A
:10089000130505026FF05FFC930485FDB31A9B00FE
:1008A000130400006FF0DFFDB3EAA40063840A02C2
:1008B00013040500938A04001309F07F130B300022
:1008C0006FF01FF11304000013090000130B100058
:1008D0006FF01FF0130400001309F07F130B2000CA
:1008E0006FF01FEF33EF7401630E0F066380040493
:1008F00013850400EF30D037930755FF1307C0016D
:10090000634EF7021307D001130F85FF3307F7403B
:10091000B394E40133D7EB00B3649700339FEB014A
:100920001306D0C03305A6406FF05FEE13850B00B1
:10093000EF301034130505026FF01FFC930485FDA2
:10094000B3949B00130F00006FF09FFD33EF740111
:1009500063020F02138F0B001305F07F9307300023
:100960006FF01FEB930400001305000093071000C5
:100970006FF01FEA930400001305F07F9307200037
:100980006FF01FE963E6540163989A346366E435B7
:100990009396FA01135714009317F40193DA1A008F
:1009A00033E4E6001395840093548F0133E5A400EB
:1009B000135E0501B3D8CA031313050113530301D2
:1009C0001357040193158F00B3F4CA03938F0800E3
:1009D000B3061303939A040133675701637ED7006C
:1009E0003307A700938FF8FF6368A7006376D700EB
:1009F000938FE8FF3307A7003307D740B35EC703E1
:100A000013140401135404013377C70393860E00B3
:100A1000B308D303131707013367E400637E17019C
:100A20003307A7009386FEFF6368A700637617016C
:100A30009386EEFF3307A700939F0F01B3EFDF000C
:100A4000B7060100330417419388F6FF13DF0F0147
:100A500033F71F0193DE0501B3F81501B303170344
:100A6000B3041F033387EE02B302DF03330F970093
:100A700013D703013307E70163749700B382D200F1
:100A8000135F0701330F5F00B70201009382F2FF8B
:100A9000B376570093960601B3F35300B3867600FE
:100AA0006368E40193840F006314E40563F2D704E0
:100AB000B387B70033B7B7003307A7003304E400A8
:100AC0009384FFFF636685006314850263E2B702C7
:100AD0006366E401631E8F0063FCD700B387B70031
:100AE00033B7B7003307A7009384EFFF3304E40064
:100AF000B386D7403304E441B3B7D7003304F4409E
:100B0000130FF0FF63048512335FC40313D706018C
:100B10003374C403B307E30313140401336487007D
:100B200013070F00637EF4003304A4001307FFFFD4
:100B30006368A4006376F4001307EFFF3304A40096
:100B40003304F440335FC4039396060193D6060141
:100B50003374C40393070F003303E3031314040136
:100B600033E48600637E64003304A4009307FFFF30
:100B70006368A400637664009307EFFF3304A40066
:100B8000131707013367F7009317070193D707017E
:100B90003304644013530701338E1703B308130360
:100BA00033836E02B38EFE0293570E01B38E1E0185
:100BB000B387D70163F61701B70601003303D300EB
:100BC00093D80701B3886800370301001303F3FFCC
:100BD000B3F6670093960601337E6E00B386C601B6
:100BE00063681401631C1423130F07006380060459
:100BF00033048500130FF7FF6364A40263661401D6
:100C0000631C142163F0D50293971500B3B5B700A8
:100C10003385A500130FE7FF3304A4009385070075
:100C2000631414016384B600136F1F001307F83FA9
:100C30006352E01093777F00638007029377FF0091
:100C400093064000638AD70093064F0033BFE60146
:100C5000B384E401138F06009397740063DA0700EE
:100C6000B70700FF9387F7FFB3F4F40013070840BA
:100C70009307E07F63C2E718135F3F009397D401A7
:100C8000B3E7E70113D534001315C5001377F77FD9
:100C9000131747018320C102032481021355C500A5
:100CA0003365E5001316F6013367C500832441025E
:100CB000032901028329C101032A8101832A4101F9
:100CC000032B0101832BC100138507009305070047
:100CD00013010103678000001308F8FF9307000069
:100CE0006FF05FCC1386090093840A00130F040091
:100CF00093070B00130720006380E71013073000F1
:100D00006382E70E13071000E392E7F21305000079
:100D1000930700006F00400913060A006FF09FFD63
:100D2000B7040800130F00001306000093073000FB
:100D30006FF05FFC130510003305E5409307800357
:100D4000E3C6A7FC9307F00163C4A7061308E841B4
:100D5000B39704013357AF0033180F01B3E7E7002F
:100D600033380001B3E7070133D5A40013F7770048
:100D70006300070213F7F70093064000630AD700E9
:100D800013874700B337F7003305F50093070700D3
:100D900013178500634A07061317D50193D7370049
:100DA000B367F70013553500130700006FF0DFED50
:100DB000930710FEB387E74093060002B3D7F40011
:100DC000130700006306D5001308E84333970401B6
:100DD000336FE701333FE001B3E7E701130500009C
:100DE0006FF0DFF837050800930700001307F07F66
:100DF000130600006FF05FE9130500009307000081
:100E00001307F07F6FF05FE8130500009307000001
:100E1000130710006FF05FE713070F00130F0700B1
:100E20006FF09FE0130101FD232E310193D945019D
:100E30002324810223229102232C4101232A5101E0
:100E4000232861019394C500232611022320210346
:100E50002326710193F9F97F13040500130B060093
:100E6000938A060093D4C40013DAF5016382090A59
:100E70009307F07F6380F9109357D5019394340062
:100E8000B3E49700B7078000B3E4F400131935000A
:100E9000938919C0930B000013D54A011394CA001B
:100EA0001375F57F1354C40093DAFA01630005103B
:100EB0009307F07F6300F5169357DB01131434009A
:100EC00033E48700B70780003364F400130515C0CE
:100ED00093173B001307000093962B00B3E6E60040
:100EE0003385A9009386F6FF9305E00033465A0147
:100EF0001308150063ECD514B755018093962600AE
:100F00009385C51AB386B60083A6060067800600DF
:100F100033E9A400630C090663800404138504000C
:100F2000EF300055130755FF9307C00163CCE7026C
:100F30009307D001130985FFB387E740B3942401D9
:100F4000B357F400B3E49700331924019309D0C0D8
:100F5000B389A9406FF01FF4EF30805113050502EB
:100F60006FF05FFC930485FDB31494001309000037
:100F70006FF0DFFD33E9A4006302090213090500E5
:100F80009309F07F930B30006FF01FF19304000082
:100F900093090000930B10006FF01FF09304000002
:100FA0009309F07F930B20006FF01FEFB36764018C
:100FB000638E07066300040413050400EF30404B02
:100FC000930655FF9307C00163CED7021307D001E4
:100FD000930785FF3307D7403314F4003357EB00F2
:100FE00033648700B317FB001307D0C03305A74055
:100FF0006FF05FEE13050B00EF308047130505021D
:101000006FF01FFC130485FD33148B009307000061
:101010006FF09FFDB36764016382070293070B00C3
:101020001305F07F130730006FF01FEB130400006F
:1010300013050000130710006FF01FEA13040000EF
:101040001305F07F130720006FF01FE9370F010031
:10105000930EFFFF1357090193D807013379D90184
:10106000B3F7D701B3852803B3862703B30FF7027D
:101070003383F50193D50601B3856500330E17035D
:1010800063F4F501330EEE0193D30501B3F5D501F9
:10109000B3F6D601135F0401B372D4019395050131
:1010A000B385D500B30E5702B386220333092F034D
:1010B0003303D90113D90601330969003307E70364
:1010C0006376D9013703010033076700935E090196
:1010D000B7090100B38EEE001387F9FF3379E900F9
:1010E000B3F6E60013D4040113190901B3F4E400C4
:1010F0003309D90033879702B38323013303F40202
:10110000B3869802B3878802B388660093560701B6
:10111000B386160163F46600B387370193D80601DE
:10112000B7090100B38FF8009387F9FFB3F6F60013
:101130003377F700B388920293960601B386E600F0
:10114000B3075402B3049F0233038F02B384F40045
:1011500013D40801B304940063F4F400330333019F
:10116000B70701009387F7FF33F7F400B3F8F800EF
:1011700013170701330E7E003307170133392E0191
:101180003307D70133042701330EDE00B336DE0008
:10119000B308F401338FD8003337D7013334240137
:1011A0003364870093D40401B3B8F801B336DF0089
:1011B00033049400B3E6D8003304D400330464004D
:1011C00093577F01131494003364F40093179E0027
:1011D000B3E7B700B337F000135E7E0113179F002B
:1011E000B3E7C701B3E7E7001317740063520710B2
:1011F00013D7170093F71700B367F7001317F4011D
:10120000B3E7E700135414009306F83F6356D00E7B
:1012100013F777006300070213F7F7009305400008
:10122000630AB70013874700B337F7003304F400AD
:101230009307070013177400635A0700370700FF6E
:101240001307F7FF3374E400930608401307E07FA9
:101250006346D71613D737009317D401B3E7E700D7
:10126000135434001314C40013F7F67F1317470107
:101270001354C4003364E4001316F6013367C4004A
:101280008320C10203248102832441020329010235
:101290008329C101032A8101832A4101032B010112
:1012A000832BC10013850700930507001301010379
:1012B0006780000013060A001384040093070900E6
:1012C00013870B0093062000630AD70E93063000A5
:1012D000630CD70C93061000E318D7F21304000038
:1012E000930700006F00800813860A006FF09FFDCF
:1012F000130805006FF05FF193051000B385D5402A
:1013000013078003E34CB7FC1307F0016344B706EF
:101310001308E84133170401B3D6B700B3970701A8
:101320003367D700B337F000B367F7003354B40026
:1013300013F777006300070213F7F70093064000E6
:10134000630AD70013874700B337F7003304F4006C
:101350009307070013178400634A07061317D40185
:1013600093D73700B367F700135434009306000097
:101370006FF05FEF130710FE3307D740130500022D
:101380003357E400930600006386A5001308E84382
:10139000B3160401B3E7F600B337F000B367F70004
:1013A000130400006FF0DFF8370408009307000013
:1013B0009306F07F130600006FF0DFEA13040000CD
:1013C000930700009306F07F6FF0DFE9130400003D
:1013D00093070000930610006FF0DFE88327C50035
:1013E00003AF050083AF450083A2850083A5C50038
:1013F0003787000093D607011307F7FF13980701FB
:10140000939E050113D6F701B3F6E60093D70501C5
:10141000130101FF8328050003234500032E8500E7
:101420001358080193DE0E01B3F7E70093D5F501D9
:101430006390E60233E768003367C701336707014B
:1014400013051000631A07046398D7046F00800027
:10145000639CE7003367FF01336757003367D701A9
:1014600013051000631A0702130510006396D702D4
:101470006394E8036312F30363105E02631ED801F2
:101480006300B602639A070033E568003365C5015F
:10149000336505013335A0001301010167800000A9
:1014A000130500006FF05FFF832F05000328450040
:1014B000032E85000325C50003A6C500B7870000DD
:1014C000935605019387F7FF13130601135706017F
:1014D00083A2050083A8450083AE8500B3F6F6001D
:1014E00093150501130101FF93D505011355F5016E
:1014F000135303013377F7001356F601639EF6008A
:10150000B367F801B3E7C701B3E7B7006388070C17
:101510001305E0FF6F000006631AF700B3E75800F9
:10152000B3E7D701B3E76700E39407FE639A060ABF
:10153000B367F801B3E7C701B3E7B70093B7170084
:10154000631A070033EF5800336FDF01336F6F000A
:10155000630A0F06639A07006302C502630005066B
:101560001305F0FF6F0000011305F0FF6304060090
:10157000130506001301010167800000E340D7FE58
:1015800063D6E600E31805FE6FF09FFDE368B3FC49
:10159000639E6502E3E4CEFD639ECE03E3E008FDB7
:1015A00063940801E3ECF2FBE36E18FD6394080119
:1015B000E3EA5FFC130500006FF0DFFB130510008A
:1015C0006FF05FFBE39807FE6FF05FF9E3EC65FAFD
:1015D0006FF05FFEE368DEFB6FF0DFFDE300D7F442
:1015E000E31C07F6930700006FF0DFF5832F05007B
:1015F00003284500032E85000325C50003A6C5006A
:10160000B7870000935605019387F7FF1313060170
:101610001357060183A2050083A8450083AE850009
:10162000B3F6F60093150501130101FF93D50501EB
:101630001355F501135303013377F7001356F601E1
:10164000639EF600B367F801B3E7C701B3E7B700DD
:101650006388070C130520006F000006631AF7006B
:10166000B3E75800B3E7D701B3E76700E39407FE99
:10167000639A060AB367F801B3E7C701B3E7B70097
:1016800093B71700631A070033EF5800336FDF0179
:10169000336F6F00630A0F06639A07006302C50287
:1016A000630005061305F0FF6F0000011305F0FF4E
:1016B00063040600130506001301010167800000A2
:1016C000E340D7FE63D6E600E31805FE6FF09FFD0A
:1016D000E368B3FC639E6502E3E4CEFD639ECE0344
:1016E000E3E008FD63940801E3ECF2FBE36E18FD10
:1016F00063940801E3EA5FFC130500006FF0DFFB71
:10170000130510006FF05FFBE39807FE6FF05FF9C1
:10171000E3EC65FA6FF05FFEE368DEFB6FF0DFFD80
:10172000E300D7F4E31C07F6930700006FF0DFF542
:10173000130101F42326310B83A9C50083A60500FC
:1017400083A745002326A10003A58500139709015F
:101750002328210B2324410B2322510B2320610B2F
:10176000032A0600032B4600832A86000329C600AD
:1017700037860000232A910A1357070193D40901E1
:101780001306F6FF23263107232E110A232C810A84
:10179000232E7109232C8109232A91092328A109C9
:1017A0002326B1092320D1062322F1062324A106F2
:1017B0002328D102232AF102232CA102232EE102A5
:1017C000B3F4C40093D9F901638804126386C42476
:1017D000B7070100B367F700232EF10213060103D8
:1017E0009307C10303A7070083A6C7FF9387C7FF1B
:1017F0001317370093D6D6013367D70023A2E7002B
:10180000E312F6FE8327010337C5FFFF130515001A
:10181000939737002328F102B384A400930B0000B0
:101820001315090137870000935709011355050166
:101830001307F7FF232621072320410723226107EF
:101840002324510723204105232261052324510528
:101850002326A104B3F7E7001359F9016382071E99
:101860006380E730B70A0100B36A550123265105AA
:10187000930501041307C104832607000326C7FF4D
:101880001307C7FF939636001356D601B3E6C6007A
:101890002322D700E392E5FE0327010437C5FFFFAB
:1018A00013051500131737002320E104B387A700A1
:1018B00013070000B387F4002320F1029387170079
:1018C000232EF10093972B00B3C62901B3E7E7005D
:1018D0002328D1009387F7FF9306E00063E6F62AFA
:1018E000B7560180939727009386861EB387D7004B
:1018F00083A707006780070033E6D7003366A6009A
:101900003366E60063080612630007061305070046
:10191000EF201036930645FF93D7564093F6F60115
:10192000638E06061307C0FF3387E7021303010324
:1019300013080002939527003308D8401307C70007
:101940003307E3006314E30813070108B305B70086
:10195000032701039387F7FFB316D70023A8D5FA0F
:101960009306F0FF6F00000A63080500EF20503077
:10197000130505026FF01FFA638A0700138507003D
:10198000EF20102F130505046FF0DFF81385060014
:10199000EF20102E130505066FF0DFF71306C0FFCA
:1019A0003386C7021307C10393063000B305C7008F
:1019B00083A505009386F6FF1307C7FF2322B70010
:1019C000E3D6F6FE9387F7FF6FF09FF90326C7FF74
:1019D00083280700330EB70033560601B398D800AA
:1019E000336616012320CE001307C7FF6FF09FF563
:1019F00013972700130601033307E600232007008F
:101A00009387F7FFE396D7FEB7C4FFFF93841401D3
:101A1000B384A4406FF09FE0B3E7D700B3E7A7001B
:101A2000B3E7E700930B3000E39C07DE930B200045
:101A30006FF01FDF93040000930B10006FF05FDE68
:101A4000B3676A01B3E75701B3E7A70063880712DA
:101A5000630E0504EF20D021130645FF13575640AF
:101A60001376F601630006089306C0FFB306D7029B
:101A7000130301049307000213182700B387C7401C
:101A80009386C600B306D3006316D30893070108F4
:101A900033880701832701041307F7FF3396C70034
:101AA0002320C8FC9306F0FF6F00400A638A0A00F7
:101AB00013850A00EF20D01B130505026FF0DFF934
:101AC000630A0B0013050B00EF20901A13050504A1
:101AD0006FF09FF813050A00EF2090191305050613
:101AE0006FF09FF71306C0FF3306C7029306C104C9
:101AF00093073000B385C60083A505009387F7FFE1
:101B00009386C6FF23A2B600E3D6E7FE1307F7FFCE
:101B10006FF05FF983A5C6FF83A80600338E060128
:101B2000B3D5F500B398C800B3E515012320BE0076
:101B30009386C6FF6FF05FF5931727001306010425
:101B4000B307F60023A007001307F7FFE316D7FE3D
:101B5000B7C7FFFF93871701B387A7406FF05FD523
:101B6000336A6A01B36A5A01B3EAAA001307300064
:101B7000E3920AD4130720006FF0DFD3930700002D
:101B8000130710006FF01FD303270103032E010476
:101B9000370501009306F5FF935F0701935A0E0185
:101BA0003377D700337EDE00B387EA023306EE02D6
:101BB0003388CF03B385070193570601B387B70076
:101BC000338B5F0363F40701330BAB00032F410436
:101BD00093D20701B3F7D7003376D6009397070166
:101BE000B387C70093540F01337FDF002322F10234
:101BF0002320F106B306EF02B387E4023386EF0336
